:020000040800F2
:1000000000040020E1010008410E0008450E000830
:10001000990E0008450E00086D0E0008E301000867
:10002000E3010008E3010008E30100086D2F000868
:10003000E3010008E3010008E3010008E301000810
:10004000E3010008E3010008E3010008E301000800
:10005000E3010008E3010008CD310008F931000890
:1000600025320008513200087D320008E301000803
:10007000E3010008E3010008E3010008E3010008D0
:10008000E3010008E3010008E3010008E3010008C0
:10009000E3010008E3010008E3010008A9320008B9
:1000A000E3010008E3010008E3010008E3010008A0
:1000B000E92F0008E3010008E3010008E30100085C
:1000C000E3010008E3010008E3010008E301000880
:1000D000E3010008E3010008E3010008E301000870
:1000E00011330008E3010008E3010008E301000800
:1000F000E3010008E3010008E3010008E301000850
:10010000E3010008E3010008E3010008E30100083F
:10011000E3010008E3010008E3010008E30100082F
:10012000E3010008E3010008E3010008E30100081F
:10013000E3010008E3010008E3010008E30100080F
:10014000E3010008E3010008E3010008C1260008FC
:10015000E3010008E3010008E3010008E3010008EF
:10016000E3010008E3010008E3010008E3010008DF
:10017000E3010008E3010008E3010008E3010008CF
:10018000E3010008E3010008E3010008E3010008BF
:10019000E3010008E3010008E3010008E3010008AF
:1001A000E3010008E3010008E3010008E30100089F
:1001B000E3010008E3010008E3010008E30100088F
:1001C000E3010008E3010008E3010008E30100087F
:1001D000E3010008E3010008E3010008E30100086F
:1001E00002E000F000F8FEE772B6394880F30888B4
:1001F000384880F3098838484EF60851CEF200019D
:10020000086040F20000CCF200004EF63471CEF2ED
:1002100000010860BFF34F8FBFF36F8F40F2000003
:10022000C0F2F0004EF68851CEF200010860BFF334
:100230004F8FBFF36F8F4FF00000E1EE100A4EF6C4
:100240003C71CEF200010860062080F31488BFF3F1
:100250006F8F01F0FDFE02F01FFE4FF055301F4979
:100260001B4A91423CBF41F8040BFAE71C49194A6A
:1002700091423CBF41F8040BFAE71A491A4A1B4B5A
:100280009A423EBF51F8040B42F8040BF8E70020F5
:100290001749184A91423CBF41F8040BFAE701F0B4
:1002A000DBFE02F055FE144C144DAC4203DA54F858
:1002B000041B8847F9E700F03FF8114C114DAC42A0
:1002C00003DA54F8041B8847F9E701F0C3BE0000C5
:1002D000000400200024002000000008000000208E
:1002E00000040020203700080024002028240020DB
:1002F0002824002018300020E0010008E001000858
:10030000E0010008E00100082DE9F04F2DED108A12
:10031000C1F80CD0C3689D46BDEC108ABDE8F08FD3
:10032000002383F311882846A047002001F016FB24
:1003300001F0C6FA00DFFEE71A4B7D2270B50024FB
:100340001A700F225C709C70DC701C715C719C7167
:10035000DC711C725C729A72DC7201F04BFE064614
:1003600001F070FE054650B90F4B9E4217D0013385
:100370009E4241F2883412BF054600240125002028
:1003800001F042FE0DB100F0B5F800F02DFD00F0D7
:10039000F5FB204600F00CF900F0ACF8F9E7044654
:1003A000EDE700BF28240020010007B008B500F0E9
:1003B00087FBA0F120035842584108BD07B5054B03
:1003C00002211B88ADF8043001A800F0C7FB03B080
:1003D0005DF804FBF4330008064991F8243033B18A
:1003E00000230822086A81F8243000F0E9BB0120CC
:1003F000704700BF482400202DE9F84F234C94F8A3
:1004000024300546884617468BBB2E46DFF87C9085
:10041000002F38D094F824A0BAF1000F05D1202283
:10042000FF214846266200F0CDFCCAF10805BD4216
:1004300028BF3D465FFA85FBAD0041462A4604EBE6
:100440008A0000F095FC94F82430A7EB0B079B443E
:100450005FFA8BFBBBF1080F2E44A844FFB284F86F
:1004600024B0D5D1FFF7B8FF0028D1D108E0266A23
:1004700006EB8306B042C9D0FFF7AEFF0028C4D117
:100480000020BDE8F88F0120BDE8F88F4824002047
:1004900010B5202383F311881248C3680BB101F013
:1004A000E3FA0023104A0F484FF47A7101F0A0FAE2
:1004B000002383F311880D4C236813B12368013B9B
:1004C0002360636813B16368013B6360084B1B786A
:1004D00033B9636823B9022000F036FC322363602D
:1004E00010BD00BF342400209104000878250020AE
:1004F0007024002010B5254B254953F8042F0132F4
:1005000000D110BD8B42F8D1224C234B22689A4275
:100510003AD9224B9B6803F1006303F580339A427A
:1005200032D2002000F044FB1D4B0220187000F076
:10053000F9FB1C4B1A6C00221A64196E1A66196EAC
:10054000596C5A64596E5A665A6E5A6942F0800262
:100550005A615A6922F080025A615A691A6942F056
:1005600000521A611A6922F000521A611B6972B6B0
:100570000D4A0E4B13601B682268202181F31188FD
:100580009D4683F30888104710BD00BFFCFF00089C
:100590001C00010804000108FFFF000828240020B7
:1005A000702400200038024008ED00E0000001083F
:1005B0002DE9F04F99B0B34C01902022FF2110A8F3
:1005C000A66800F0FFFBB04A1378A346A3B9AF4872
:1005D0000121C3601170202383F31188C3680BB11C
:1005E00001F042FA0023AA4AA8484FF47A7101F0B8
:1005F000FFF9002383F31188019B13B1A54B019AE6
:100600001A60A54AA349019F0292002313704B6010
:1006100099461C461D469846012000F083FB002F9A
:1006200000F012829B4B1B68002B40F00D8219B02A
:10063000BDE8F08F0220FFF7B9FE002840F0FB81F3
:10064000019BB9F1000F08BF1F46944B1B88ADF802
:100650002C3002210BA800F081FADDE74FF47A700C
:1006600000F02EFA031E0393EADB0220FFF79EFE42
:1006700082460028E4D0039B581E042800F2DD8146
:10068000DFE800F0030E1114170018A8052340F846
:10069000343D042100F062FA54464FF0000856E061
:1006A00004217848F6E704217D48F3E704217D48DA
:1006B000F0E71C24204600F07DFA04340B9004215E
:1006C0000BA800F04BFA2C2CF4D1E5E7002DB7D0A5
:1006D000002CB5D00220FFF769FE0546002800F087
:1006E000AF8101206C4C00F063FA0220207000F012
:1006F00019FB4FF000095FFA89FA504600F068FADA
:10070000074658B1504600F073FA09F10109002874
:10071000F1D12C46A9460027634B97E7012302201D
:10072000237000F0EDFA3E46DBF808309E4206D218
:10073000304600F03FFA0130EBD10436F4E7029B7B
:1007400000261E70534BA9465E602C46374600F0CB
:1007500041FB15B1002C18BF0027FFF72FFE5BE708
:10076000002D3FF46DAF002C3FF46AAF029B0220D6
:10077000187000F0D7FA322000F0A2F9B0F1000AA8
:10078000C0F25E811AF0030540F05A81DBF80820C0
:1007900006EB0A03934200F25381BAF5807F00F220
:1007A0004F8155450DDA4FF47A7000F089F90490C5
:1007B000049B002BC0F244813C4A049BAB5401359E
:1007C000EFE7C820FFF7F2FD0546002800F038816A
:1007D0001F2E11D8C6F12004544528BF544610AB33
:1007E00026F0030022463149184400F0C1FA22469F
:1007F000FF212E4800F0E6FA4FEAAA0A5FFA8AF2D1
:100800002A493046FFF7F8FD0446002800F01A8117
:1008100006EB8A0605469AE70220FFF7C7FD002887
:100820003FF40EAFFFF7D8FD00283FF409AF4FF0BB
:10083000000A5346DBF8082092451CD2BAF11F0F7C
:1008400012D8109A01320FD02AF0030218A90A44D4
:1008500052F8202C0B92184604220BA900F030FB12
:100860000AF1040A0346E5E75046039300F0A2F9B3
:10087000039B0B90EFE718A8042140F84C3D00F0D3
:100880006DF964E72824002074250020342400201A
:10089000910400087825002070240020F633000819
:1008A0002C24002030240020F83300087424002079
:1008B00018A8002340F8343D642100F02BF90028EB
:1008C0007FF4BEAE0220FFF771FD00283FF4B8AE02
:1008D0000B9800F09FF918AB43F8480D0421184617
:1008E000CDE718A8002340F8343D642100F012F948
:1008F00000287FF4A5AE0220FFF758FD00283FF442
:100900009FAE0B9800F094F918AB43F8440DE5E75F
:100910000220FFF74BFD00283FF492AE00F08EF965
:1009200018AB43F8400DD9E70220FFF73FFD002840
:100930003FF486AE0BA9142000F086F9824618A871
:10094000042140F83CAD00F009F951460BA896E7A8
:10095000322000F0B5F8B0F1000AFFF671AE1AF0DF
:10096000030F7FF46DAEDBF808200AEB0803934217
:100970003FF666AE0220FFF719FD00283FF460AE97
:100980002AF0030AC244D0453FF4E1AE404600F0ED
:1009900011F904210A900AA800F0E0F808F104080F
:1009A000F1E74FF47A70FFF701FD00283FF448AEFD
:1009B000FFF712FD00283FF4AFAE109B01330CD0BF
:1009C000082210A90020FFF717FD00283FF4A4AE6D
:1009D0002022FF2110A800F0F5F9FFF7EFFC3748BF
:1009E00000F0C2FF23E6002D3FF42AAE002C3FF4B6
:1009F00027AE18A8002340F8343D642100F08AF89F
:100A0000824600287FF41CAE0220FFF7CFFC0028AE
:100A10003FF416AE0390FFF7D1FC41F2883000F0AE
:100A2000A3FF0B9800F00AFA00F0D4F9039B574695
:100A30001C461D46F0E5054689E64FF00008FFE537
:100A40002546FDE52C4667E6002000F039F80490C5
:100A5000049B002BFFF6E3AD012000F051F9049B4D
:100A6000213B122B3FF6D8AD01A252F823F000BF74
:100A7000350600085D060008CD06000819060008C6
:100A80001906000819060008610700085109000846
:100A900019080008B1080008E30800081109000857
:100AA000190600082909000819060008A30900080A
:100AB0004F07000819060008E7090008A086010092
:100AC00037B5114B1A780132D2B20024012A0146FF
:100AD0008DF8074011D80D4803681D6A4FF47A73EA
:100AE0004B4301220DF10701A847012805D1084B0E
:100AF0009DF807001C7003B030BD4FF4FA7000F091
:100B000033FF4FF0FF30F6E7002400204826002096
:100B10008425002038B50E4B1A780132D2B2012A52
:100B200005460ED80B4803681C6A4FF47A734B4392
:100B300004222946A047042803D1074B002018703F
:100B400038BD4FF4FA7000F00FFF4FF0FF3038BDA2
:100B500000240020482600208425002030B4054CC5
:100B60002368DD69044B0A46AC460146204630BC8A
:100B7000604700BF48260020A086010070B501F044
:100B80003DF9094C094E20700025306823788342D6
:100B900008D901F02DF9336805440133B5F5803FDC
:100BA0003360F2D370BD00BF852500208025002072
:100BB00001F0D2B900F1006000F5803000687047A4
:100BC00000F10060920000F5803001F05DB9000096
:100BD000054B1A68054B1B789B1A834202D91044B7
:100BE00001F006B9002070478025002085250020EF
:100BF00038B5074D04462868204401F001F928B9AA
:100C000028682044BDE8384001F012B938BD00BF63
:100C10008025002010F0030308D1B0F5007F05D82F
:100C200000F10050A0F508400068704700207047B0
:100C3000014BC058704700BF107AFF1F014B186866
:100C4000704700BF002004E070B52A4B1C68C4F355
:100C50000B03240C63B140F21342934231D040F2B3
:100C6000194293422FD040F2214293422DD10323C7
:100C7000214A0C2505FB03235D6893F9082042F205
:100C800001039C4224D0B4F5805F23D041F20103DC
:100C90009C4221D041F203039C421FD041F2070342
:100CA0009C4208BF3122441E0C44013D0B46A34226
:100CB0001ED215F9016F581C96B1034600F8016C5D
:100CC000F5E70123D4E70223D2E73F220B4DD6E715
:100CD0003322E3E74122E1E75A22E4E75922E2E73F
:100CE0002C2584421D7001D9981C5A70401A70BD81
:100CF0001846FBE7002004E008340008FC33000835
:100D0000022804D1054B4FF000729A617047012808
:100D1000FCD14FF08042024BF7E700BF00040240D5
:100D200000000240022804D1054B4FF400729A6182
:100D300070470128FCD14FF48042024BF7E700BF17
:100D40000004024000000240022805D1064A53690F
:100D500083F40073536170470128FCD1034A53693F
:100D600083F48043F6E700BF000402400000024025
:100D700010B50023934203D0CC5CC4540133F9E78F
:100D800010BD000030B5441E14F9010F0B4660B1D0
:100D900093F90050854201F1010106D11AB993F986
:100DA0000020801A30BD013AEEE7002AF7D1104644
:100DB00030BD000002460346981A13F9011B0029B2
:100DC000FAD1704702440346934202D003F8011B54
:100DD000FAE77047024B1A78024B1A70704700BF4F
:100DE000842500200024002038B5104D104C2846E2
:100DF00000F002F92146284600F02AF924680D483F
:100E0000626DD2F8043843F00203C2F8043800F0EF
:100E1000ABFD0949204600F027FA626DD2F804388C
:100E200023F00203C2F8043838BD00BF4826002072
:100E3000D434000840420F00FC3400087047000022
:100E4000FEE7000000B59BB0EFF309816822684619
:100E5000FFF78EFFEFF30583034B9A6B9A6A9A6A4A
:100E60009A6A9A6A9B6AFEE700ED00E000B59BB0C3
:100E7000EFF3098168226846FFF77AFFEFF30583F5
:100E8000044B9A6B9A6A9A6A9A6A9A6A9A6A9B6AF5
:100E9000FEE700BF00ED00E000B59BB0EFF3098175
:100EA00068226846FFF764FFEFF30583034B5A6B34
:100EB0009A6A9A6A9A6A9A6A9B6AFEE700ED00E06B
:100EC00030B5084D0A4491420BD011F8013B09247A
:100ED0005840013CF7D040F300032B4083EA500018
:100EE000F7E730BD2083B8ED002304491A465A5075
:100EF000C8180833802B4260F9D17047882500203C
:100F0000026843681143016003B11847704700004D
:100F100013B5446BD4F894341A681178042915D1A8
:100F2000217C022912D11979128901238B401342A5
:100F30000CD101A904F14C0001F028FED4F894442E
:100F4000019B21790246206800F0DAF902B010BD59
:100F5000143001F0ABBD00004FF0FF33143001F04E
:100F6000A5BD00004C3001F07DBE00004FF0FF3306
:100F70004C3001F077BE0000143001F079BD000064
:100F80004FF0FF31143001F073BD00004C3001F020
:100F900049BE00004FF0FF324C3001F043BE00006C
:100FA000D0F8942438B5136819780429054601D07F
:100FB000012038BD017C0229FAD112795C89012017
:100FC00090400440F4D105F1140001F00BFD0246FD
:100FD0000028EDD0D5F894544FF4807328686979CF
:100FE00000F07CF9204638BD406BFFF7D9BF000008
:100FF00000207047704700007FB5124B036000234C
:1010000043608360C360012502260F4B05740446CC
:101010000290019300F18402294600964FF48073F8
:10102000143001F0BBFC094B0193029400964FF47D
:10103000807304F52372294604F14C0001F082FD0F
:1010400004B070BD58340008E90F0008110F000803
:101050000B68202282F311880A7903EB82029061E7
:101060004A79093243F822008A7912B103EB8203EC
:10107000986102230374C0F89414002383F3118849
:101080007047000038B5037F044613B190F8543020
:10109000ABB9201D01250221FFF732FF04F1140036
:1010A00025776FF0010100F087FC84F8545004F1BB
:1010B0004C006FF00101BDE8384000F07DBC38BD48
:1010C00010B5012104460430FFF71AFF00232377EF
:1010D00084F8543010BD000038B5044600251430A3
:1010E00001F074FC04F14C00257701F043FD201D54
:1010F00084F854500121FFF703FF2046BDE8384033
:10110000FFF74EBF90F8443003F06003202B19D155
:1011100090F84520212A0AD0222A4FF000030ED051
:10112000202A0FD1084A82630722C26304E0064BDB
:1011300083630723C3630023036401207047836331
:10114000C363F9E70020704701240020D0F89434ED
:1011500037B51A681178042904461AD1017C02298E
:1011600017D11979128901238B40134211D100F153
:101170004C05284601F0BEFD58B101A9284601F0F2
:1011800005FDD4F89444019B21790246206800F0C3
:10119000B7F803B030BD000000EB8103F7B59C69E0
:1011A00005460E46F4B1202383F3118805EB86072C
:1011B000201D0821FFF7A4FEFB685B691B684C3407
:1011C00013B1204601F0F0FC01A9204601F0DEFC3D
:1011D000024648B1019B3146284600F091F80023B1
:1011E00083F3118803B0F0BDFB685A691268002AC6
:1011F000F5D01B8A013B1340F1D105F14402EAE727
:10120000093138B550F82140DCB1202383F311882F
:10121000D4F894241368527903EB8203DB689B694A
:101220005D6845B104216018FFF76AFE294604F1A4
:10123000140001F0E1FB2046FFF7B2FE002383F328
:10124000118838BD7047000000F08CBF0123037087
:1012500000234360C36183620362C362436203632A
:10126000038143817047000038B50446202383F38F
:10127000118800254160C56005614561856100F008
:1012800081FF0223237085F3118838BD70B500EB10
:10129000810305465069DA600E46144618B11022E3
:1012A0000021FFF78FFDA06918B110220021FFF780
:1012B00089FD31462846BDE8704001F02DB8000098
:1012C000028902F001020281428902F00102428198
:1012D000002202614261826101F0B2B8F0B400EB19
:1012E00081044789E4680125A4698D403D43458117
:1012F00023600023A2606360F0BC01F0CDB8000061
:10130000F0B400EB81040789E468012564698D402D
:101310003D43058123600023A2606360F0BC01F0BF
:1013200047B9000070B50223002504460370A0F8F9
:101330004C5080F84E5080F84F5005814581C56073
:1013400005614561856180F8345000F081FF636874
:101350001B6823B129462046BDE87040184770BD80
:10136000436802781B6880F85020052202700BB198
:101370000421184770470000436890F850201B680C
:1013800002700BB1052118477047000090F8343007
:1013900070B5044613B1002380F8343004F14402E0
:1013A000204601F06FF863689B6863BB94F8445073
:1013B00015F0600615D194F8453005F07F0545EA33
:1013C000032540F202339D4200F00E815BD8022DCE
:1013D00000F0DC803FD8002D00F08780012D00F068
:1013E000CF800021204601F0A5FA0021204601F01F
:1013F00097FA63681B6813B10621204698470623B5
:1014000084F8343070BD204698470028CED094F838
:101410004B2094F84A3043EA0223E26B934238BFF0
:10142000E36394F94430E56B002B4FF0200380F226
:10143000FD80002D00F0EC80092284F8342083F335
:1014400011880021E36BA26B2046FFF759FF0023B0
:1014500083F3118870BDB5F5817F00F0B180B5F5DB
:10146000407F49D0B5F5807FBBD194F84630012B41
:10147000B7D1B4F84C3023F00203A4F84C30A66383
:10148000E6632664C3E740F201639D421ED8B5F5CA
:10149000C06F3BD2B5F5A06FA3D1B4F84430B3F51B
:1014A000A06F0ED194F8463084F84E30204600F0FC
:1014B00027FF63681B6813B1012120469847032367
:1014C00023700023A363E3632364A0E7B5F5106FE3
:1014D00032D040F602439D4252D0B5F5006F80D124
:1014E00004F14F03A363012324E004F14C03A3633D
:1014F0000223E36325648AE794F84630012B7FF4E6
:1015000070AFB4F84C3043F00203B6E794F84920CA
:10151000616894F848304D6894F8471043EA022314
:10152000204694F84620A84700283FF45AAF436865
:10153000A3630368E363A4E72378042B10D120237B
:1015400083F311882046FFF7BBFE86F3118863689A
:1015500084F84F601B68032121700BB12046984727
:1015600094F84630002BACD084F84F30042323701D
:1015700063681B68002BA4D0022120469847A0E78F
:10158000374BA3630223E36300239DE794F84810DD
:1015900011F0800F204601F00F010ED000F064FF23
:1015A000012806D002287FF41CAF2E4BA363E06312
:1015B00067E72D4BA363E56363E700F047FFEFE7C1
:1015C00094F84630002B7FF40CAF94F8483013F0B9
:1015D0000F013FF476AF1A06204602D501F0BEF99E
:1015E0006FE701F0B1F96CE794F84630002B7FF417
:1015F000F8AE94F8483013F00F013FF462AF1B06C9
:10160000204602D501F096F95BE701F089F958E729
:10161000142284F8342083F311882B462A46294665
:101620002046FFF75BFE85F3118870BD5DB1152282
:1016300084F8342083F311880021E36BA26B2046E9
:10164000FFF74CFE03E70B2284F8342083F3118864
:101650002B462A4629462046FFF752FEE3E700BF05
:1016600088340008803400088434000838B590F8C5
:1016700034300446152B29D8DFE803F03E2828280B
:1016800028283E28280B29392828282828282828CF
:101690003E3E90F84B1090F84A20C36B42EA01227C
:1016A0009A4214D9C268128AB3FBF2F502FB1535CF
:1016B0006DB9202383F311882B462A462946FFF76C
:1016C0001FFE85F311880A2384F8343038BD1423B3
:1016D00084F83430202383F3118800231A461946F6
:1016E0002046FFF7FBFD002383F3118838BD036C10
:1016F00003B198470023E7E7002101F01BF900211F
:10170000204601F00DF963681B6813B106212046DD
:1017100098470623D8E7000090F83420152A38B5FA
:10172000044622D80123934040F6416213421DD162
:1017300013F480150FD19B0217D50B2380F834309A
:10174000202383F311882B462A462946FFF7D8FD2C
:1017500085F3118838BDC3689B695B682BB9036C3E
:1017600003B19847002384F8343038BD002101F0DC
:10177000E1F80021204601F0D3F863681B6813B13B
:101780000621204698470623EDE70000024B002281
:101790001B605B609A60704708260020002303747A
:1017A0008268054B1B6899689142FBD25A680360B6
:1017B00042601060586070470826002008B520235A
:1017C00083F31188037C032B05D0042B0DD02BB998
:1017D00083F3118808BD436900221A604FF0FF337C
:1017E0004361FFF7DBFF0023F2E790E80C001A608B
:1017F00002685360F2E70000002303748268054B1F
:101800001B6899689142FBD85A6803604260106077
:101810005860704708260020054B1969087418683D
:1018200002681A605360186101230374FEF76CBDEF
:101830000826002030B54B1C87B005460A4C10D056
:1018400023690A4A01A800F0D3F82846FFF7E4FF0D
:10185000049B13B101A800F007F92369586907B088
:1018600030BDFFF7D9FFF8E708260020BD170008B4
:1018700038B50C4D41612B6981689A6891420446E4
:1018800003D8BDE83840FFF789BF1846FFF786FF49
:1018900001232C61014623742046BDE83840FEF741
:1018A00033BD00BF08260020044B1A681B699068EE
:1018B0009B68984294BF00200120704708260020B2
:1018C00010B5084C236820691A6822605460012210
:1018D00023611A74FFF790FF01462069BDE81040AC
:1018E000FEF712BD08260020826002220274002248
:1018F000427470478368A3F17C0243F80C2C0269A0
:1019000043F83C2C426943F8382C074A43F81C2C16
:10191000C26843F8102C022203F8082C002203F8B6
:10192000072CA3F1180070472103000810B52023ED
:1019300083F31188FFF7DEFF00210446FFF798FFCD
:10194000002383F31188204610BD0000024B1B6961
:1019500058610F20FFF760BF08260020202383F383
:101960001188FFF7F3BF000008B50146202383F379
:1019700011880820FFF75EFF002383F3118808BD5C
:1019800049B1064B42681B6918605A601360436096
:101990000420FFF74FBF4FF0FF30704708260020AC
:1019A0000368984206D01A68026050605961184670
:1019B000FFF7F4BE7047000038B504460D462068B6
:1019C000844200D138BD036823605C604561FFF745
:1019D000E5FEF4E7054B03F114025A619A614FF0FA
:1019E000FF32DA6100221A62704700BF0826002029
:1019F000F8B503614FF08043C2605C6A194B1A4628
:101A0000022952F8145F38BF0221954206461F464C
:101A10000AD1586198611C620560456081600819AF
:101A2000BDE8F84001F088B9186AAB68241A0C19AF
:101A300002D3E41A2D6804E09C4202D2204401F053
:101A400089F9AB689C42F4D86B68736035601E609E
:101A50006E60B460A9684FF0FF33091BA960FB6199
:101A6000F8BD00BF0826002010B41B4C234653F8D5
:101A7000141F814210D0416802680A6002685160F8
:101A80009A424FF00001C16003D0936881680B4413
:101A900093605DF8044B70470A68626100209A42C7
:101AA0005360C86003D15DF8044B01F04DB99368F1
:101AB0008868034493604FF08042206A526A121A89
:101AC0009342E6D9991A012998BF931C18445DF8EE
:101AD000044B01F03FB900BF0826002000207047EA
:101AE000FEE70000704700004FF0FF307047000035
:101AF000022906D0032906D00129064818BF002074
:101B0000704705487047032A9ABF044800EBC2009B
:101B100000207047583500080C35000808240020C4
:101B200070B59AB001AD064608462946144600F045
:101B300095F82846FFF73EF9C0B2431C5B0086E8E3
:101B40001800237003236370002302341946DAB2AD
:101B5000904204F1020401D81AB070BDEA5C04F8A6
:101B6000022C04F8011C0133F1E7000008B5202322
:101B700083F311880348FFF7E9FA002383F3118800
:101B800008BD00BF4826002010B50446052916D818
:101B9000DFE801F016150316161D202383F31188C4
:101BA0000E4A0121FFF772FB20460D4A0221FFF782
:101BB0006DFB0C48FFF790FA002383F3118810BDEA
:101BC000202383F311880748FFF75CFAF4E720230A
:101BD00083F311880348FFF773FAEDE78C340008AC
:101BE000B03400084826002038B50C4D0C4C0D4987
:101BF0002A4604F10800FFF793FF05F1CA0204F139
:101C000010000949FFF78CFF05F5CA7204F11800AE
:101C10000649BDE83840FFF783BF00BF102B002006
:101C200008240020DC340008E6340008F134000801
:101C300070B5044608460D46FFF7BCF8C6B220460C
:101C4000013403780BB9184670BD32462946FFF7B8
:101C500099F80028F3D1012070BD00002DE9F84F5C
:101C600005460C46FFF7A6F82B49C6B22846FFF7F3
:101C7000DFFF08B10236F6B228492846FFF7D8FF41
:101C800008B11036F6B2632E0DD8DFF88C80DFF87D
:101C90008C90234FDFF890A0DFF890B02E7846B9F3
:101CA0002670BDE8F88F29462046BDE8F84F01F0C0
:101CB00099BB252E2CD1072241462846FFF762F812
:101CC00058B9DBF800302360DBF8043063609BF820
:101CD0000830237207350934E0E7082249462846D0
:101CE000FFF750F8A0B90F4BA21C13F8011F090908
:101CF0005345C95D02F8021C197801F00F0102F189
:101D00000202C95D02F8031CEFD118340835C5E79B
:101D1000267001350134C1E778350008F134000838
:101D20008A3500080F7AFF1F1B7AFF1F80350008D5
:101D3000BFF34F8F024AD368DB03FCD4704700BF68
:101D4000003C024008B5094B1B7873B9FFF7F0FF60
:101D5000074B1A69002ABFBF064A5A6002F188324F
:101D60005A601A6822F480621A6008BD6E2D002045
:101D7000003C02402301674508B50B4B1B7893B923
:101D8000FFF7D6FF094B1A6942F000421A611A6840
:101D900042F480521A601A6822F480521A601A685B
:101DA00042F480621A6008BD6E2D0020003C0240A3
:101DB0000B2870B513D80B4A0B4C137863B90B4E34
:101DC0004FF0006144F8231056F8235001330C2BD8
:101DD0002944F7D10123137054F8200070BD00206E
:101DE00070BD00BFA02D0020702D00209C35000884
:101DF000014B53F8200070479C3500080C207047B9
:101E00000B2810B5044601D9002010BDFFF7D0FF04
:101E1000064B53F824301844C21A0BB9012010BDE8
:101E200012680132F0D1043BF6E700BF9C35000890
:101E30000B2810B5044621D8FFF77AFFFFF782FF81
:101E40000F4AF323D360C300DBB243F4007343F0C3
:101E500002031361136943F480331361FFF768FFD2
:101E6000FFF7A6FF074B53F8241000F0DDF8FFF74B
:101E700083FF2046BDE81040FFF7C2BF002010BD21
:101E8000003C02409C3500082DE9F84312F00103A4
:101E9000154640D18218B2F1016F3CD22C4B1B6821
:101EA00013F0010337D02B4CFFF74CFFF323E36013
:101EB000FFF73EFF40F20127032D01D9830713D01E
:101EC000244C0F46401A40F20118EB1B0B44012B27
:101ED00000EB0706236924D823F001032361FFF7F1
:101EE0004BFF0120BDE8F883236923F4407323618D
:101EF00023693B43236151F8046B0660BFF34F8FA6
:101F0000FFF716FF03689E4208D0236923F0010300
:101F10002361FFF731FF0020BDE8F883043D043062
:101F2000CAE723F440732361236943EA080323616A
:101F3000B94637F8023B3380BFF34F8FFFF7F8FE07
:101F40003688B9F80030B6B2B342BED0DDE700BF84
:101F500000380240003C0240084908B50B7828B11F
:101F600053B9FFF7EFFE01230B7008BD23B1BDE8A5
:101F700008400870FFF700BF08BD00BF6E2D0020AD
:101F800010B50244064B0439D2B2904200D110BDC4
:101F9000441C00B253F8200041F8040FE0B2F4E70B
:101FA00050280040104B30B51C6F240407D41C6F20
:101FB00044F400741C671C6F44F400441C670B4C11
:101FC000236843F4807323600244094B0439D2B27E
:101FD000904200D130BD441C00B251F8045F43F878
:101FE0002050E0B2F4E700BF00380240007000402B
:101FF0005028004007B5012201A90020FFF7C0FFCB
:10200000019803B05DF804FB13B50446FFF7F2FF37
:10201000A04206D002A9012241F8044D0020FFF79A
:10202000C1FF02B010BD000070470000034B1B68E9
:102030009B0042BF024B01221A7070477438024065
:10204000A12D0020014B1878704700BFA12D002062
:1020500070470000FEE70000084A094B09498B421F
:1020600004D3094A0021934205D3704752F8040F64
:1020700043F8040BF3E743F8041BF4E74437000884
:10208000183000201830002018300020836D30B543
:1020900000229D68446D11464FF0FF3004EB42135F
:1020A00001329542C3F80019C3F81019C3F80809A2
:1020B000C3F8001BC3F8101BC3F8080BEED24FF097
:1020C0000113C4F81C3830BD890141F020010161C1
:1020D00003699B06FCD4122000F0C4BE204B03EB26
:1020E00080022DE9F047D2F80CE05D6DDEF8142097
:1020F000461CD2F800C005EB063605EB40185168C7
:1021000061450BD3D5F83428012303FA00F022EA05
:102110000000C5F834081846BDE8F087BEF8104046
:10212000ACEB0103A34228BF2346D8F81849A4B258
:10213000B3EB840F10D894681F46A4F1040959F832
:1021400004AFC6F800A0042F01D9043FF7E71C44F0
:102150000B4494605360D2E70020BDE8F08700BFD5
:10216000A42D002010B5054C2046FFF76FF84FF066
:10217000A0436365024BA36510BD00BFA42D0020E2
:10218000F03500080378012B70B5054650D12A4B75
:10219000446D98421BD1294B5A6B42F080025A631E
:1021A0005A6D42F080025A655A6D5A6942F08002B7
:1021B0005A615A6922F080025A610E2143205B69FC
:1021C00000F0D6FB1E4BE3601E4BC4F80038002322
:1021D000C4F8003EC02323606E6D4FF40413A36364
:1021E0003369002BFCDA012333610C2000F03AFE46
:1021F0003369DB07FCD4122000F034FE3369002B76
:10220000FCDA0026A6602846FFF740FF6B68C4F89A
:102210001068DB68C4F81468C4F81C684BB90A4B32
:10222000A3614FF0FF336361A36843F00103A36030
:1022300070BD064BF4E700BFA42D0020003802401B
:102240004014004003002002003C30C0083C30C075
:10225000F8B5446D054600212046FFF735FFA96D0E
:1022600000234FF001128F68C4F834384FF0006635
:10227000C4F81C284FF0FF3004EB431201339F4297
:10228000C2F80069C2F8006BC2F80809C2F8080B6E
:10229000F2D20B686A6DEB656362102313611669F5
:1022A00016F01006FBD1122000F0DCFDD4F8003847
:1022B00023F4FE63C4F80038A36943F4402343F0D9
:1022C0001003A3610923C4F81038C4F814380A4B6A
:1022D000EB604FF0C043C4F8103B084BC4F8003B20
:1022E000C4F81069C4F80039EB6D03F1100243F42F
:1022F0008013EA65A362F8BDCC3500084080001069
:10230000426D90F84E10D2F8003823F4FE6343EA91
:102310000113C2F8003870472DE9F0410EB200EB0E
:1023200086080D46D8F80C100F6807F00303022B3F
:1023300050D0032B50D03D4A3D4F012B18BF1746BC
:10234000446D4FEA451E04EB0E030022C3F8102B28
:102350008A6905F1100C002A40D04A8A05F1580319
:102360005B013A43E2500123D4F81C2803FA0CF332
:102370001343A6444A69C4F81C380023CEF8103928
:1023800005F13F03002A39D00A8A898B9208012976
:1023900088BF4A43C16D04EB8303561841EA0242E9
:1023A000C66529465A602046FFF78EFED8F80C30E5
:1023B0001B8A43EA85531F4305F148035B01E7503D
:1023C0000123D4F81C2803FA05F51543C4F81C585A
:1023D000BDE8F081174FB3E7174FB1E704EB4613A1
:1023E000D3F8002B22F40042C3F8002BD4F81C28A9
:1023F000012303FA0CF322EA0303BAE704EB830395
:102400000E4A5A6004EB461629462046FFF75CFE4A
:10241000D6F8003923F40043C6F80039D4F81C3844
:10242000012202FA05F523EA0505CFE70080001036
:10243000008004100080081000800C1000040002CE
:10244000826D1268C265FFF721BE00005831436DEE
:1024500049015B5813F4004004D013F4001F14BF6B
:1024600001200220704700004831436D49015B584C
:1024700013F4004004D013F4001F14BF0120022005
:102480007047000000EB8101CB68196A0B6813608C
:102490004B6853607047000000EB810330B5DD6886
:1024A000AA691368D36019B9402B84BF4023136015
:1024B0006B8A1468426D1C44013CB4FBF3F4634323
:1024C000033323F0030302EB411043EAC44343F018
:1024D000C043C0F8103B2B6803F00303012B09B283
:1024E0000ED1D2F8083802EB411013F4807FD0F8F7
:1024F000003B14BF43F0805343F00053C0F8003B4F
:1025000002EB4112D2F8003B43F00443C2F8003B17
:1025100030BD00002DE9F041244D6E6D06EB4013F7
:102520000446D3F8087BC3F8087B38070AD5D6F8E9
:102530001438190706D505EB84032146DB682846C5
:102540005B689847FA072FD5D6F81438DB072BD5E8
:1025500005EB8403D968CCB98B69488A5E68B6FB01
:10256000F0F200FB12628AB91868DA6890420DD264
:10257000121A83E81400202383F311880B482146A4
:10258000FFF78AFF84F31188BDE8F081012303FA85
:1025900004F26B8923EA02036B81CB6823B12146E5
:1025A0000248BDE8F0411847BDE8F081A42D0020A5
:1025B00000EB810370B5DD68436D6C692668E660E9
:1025C0004A0156BB1A444FF40020C2F810092A6889
:1025D00002F00302012A0AB20ED1D3F8080803EB75
:1025E000421410F4807FD4F8000914BF40F08050EA
:1025F00040F00050C4F8000903EB4212D2F8000981
:1026000040F00440C2F80009D3F83408012202FA6D
:1026100001F10143C3F8341870BD19B9402E84BFCD
:102620004020206020682E8A841940F00050013C30
:102630001A44B4FBF6F440EAC440C6E7F8B50446D1
:102640001E48456D05EB4413D3F80869C3F80869C3
:10265000F10717D5D5F81038DA0713D500EB840346
:10266000D9684B691F68DA68974218D2D21B0027D5
:102670001A605F60202383F311882146FFF798FFDB
:1026800087F31188330617D5D5F834280123A340E2
:10269000134211D02046BDE8F840FFF71FBD0123CB
:1026A00003FA04F2038923EA020303818B68002BF7
:1026B000E8D021469847E5E7F8BD00BFA42D0020EB
:1026C00096482DE9F84F456D6E69AB691E4016F4CA
:1026D000805F6E61044605D0FEF724FEBDE8F84F2A
:1026E00000F054BC002E12DAD5F8003E8B489B0750
:1026F0001EBFD5F8003E23F00303C5F8003ED5F811
:10270000043823F00103C5F80438FEF735FE370519
:1027100002D58248FEF724FEB0040CD5D5F808385F
:1027200013F0060FEB6823F470530CBF43F41053FF
:1027300043F4A053EB60310704D56368DB680BB149
:1027400076489847F2025AD4B3020CD5D4F8548094
:10275000DFF8C8A100274FF00109A36D9B68F9B20B
:102760008B4280F08780F70619D5616D0A6AC2F343
:102770000A1702F00F0302F4F012B2F5802F00F0F6
:10278000A180B2F5402F0AD104EB830301F58051FB
:10279000DB68186A00231A469F4240F087803003A6
:1027A000D5F8184813D5E10302D50020FFF7B2FE93
:1027B000A20302D50120FFF7ADFE630302D502207C
:1027C000FFF7A8FE270302D50320FFF7A3FE75033A
:1027D00084D5E00702D50020FFF730FFA10702D51E
:1027E0000120FFF72BFF620702D50220FFF726FF2B
:1027F00023077FF573AF0320FFF720FF6EE7D4F8C0
:102800005480DFF818A100274FF00109A36D9B68E1
:102810005FFA87FB5B4597D308EB4B13D3F800298E
:1028200002F44022B2F5802F22D1D3F80029002AE9
:102830001EDAD3F8002942F09042C3F80029D3F8F9
:102840000029002AFBDB5946606DFFF73DFC228919
:1028500009FA0BF322EA0303238104EB8B03DB6801
:102860009B6813B15946504698475846FFF736FCC7
:102870000137CBE708EB4112D2F8003B03F44023C9
:10288000B3F5802F10D1D2F8003B002B0CDA62890F
:1028900009FA01F322EA0303638104EB8103DB6895
:1028A000DB680BB150469847013756E79C0708BFD5
:1028B0000A68072B98BF027003F101039CBF120A3C
:1028C000013069E7023304EB830201F5805152685D
:1028D00090690268D0F808C04068A2EB000E0022A0
:1028E000104697420AD104EB830463689B699A6897
:1028F0003A449A605A6817445F6050E712F0030F39
:1029000008BF0868964588BF8CF8000002F10102F4
:1029100084BF000A0CF1010CE3E700BFA42D0020E6
:10292000436D03EB4111D1F8003B43F40013C1F8B0
:10293000003B7047436D03EB4111D1F8003943F47C
:102940000013C1F800397047436D03EB4111D1F812
:10295000003B23F40013C1F8003B7047436D03EBC9
:102960004111D1F8003923F40013C1F80039704740
:1029700000F1604300F01F02400903F561430901C3
:102980008000C9B200F1604083F8001300F5614097
:1029900001239340C0F880310360704730B5039C39
:1029A0000172043304FB0325C361049B036300210C
:1029B000059B00604060C160426102618561046204
:1029C00042628162C162436330BD00000022416AFD
:1029D00041610161C2608262C2626FF00101FEF773
:1029E000EBBF000003694269934203D1C2680AB198
:1029F00000207047181D704703691960C2680132D2
:102A0000C260C269134482690361934224BF436A6E
:102A100003610021FEF7C4BF38B504460D46E368E4
:102A20003BB16269131D1268A3621344E362002084
:102A300038BD237A33B929462046FEF7A1FF002886
:102A4000EDDA38BD6FF00100FBE70000C368C26932
:102A5000013BC3604369134482694361934224BFCD
:102A6000436A436100238362036B03B118477047D5
:102A700070B52023044683F31188866A3EB9FFF7B8
:102A8000CBFF054618B186F31188284670BDA36AAE
:102A9000E26A13F8015BA362934202D32046FFF778
:102AA000D5FF002383F31188EFE700002DE9F84FED
:102AB00004460E4690469946202787F31188002544
:102AC000AA46D4F828B0BBF1000F09D149462046E8
:102AD000FFF7A2FF20B18BF311882846BDE8F88FDD
:102AE000A16AE36AA8EB050B5B1A9B4528BF9B46CE
:102AF000BBF1400F1BD9334601F1400251F8040BE2
:102B000043F8040B9142F9D1A36A40334036A362E3
:102B10004035A26AE36A9A4202D32046FFF796FF45
:102B20008AF311884545D8D287F31188C9E7304622
:102B30005A46FEF71DF9A36A5B445E44A3625D44F6
:102B4000E7E7000010B5029C0172043303FB042187
:102B5000C36100238362C362039B0363049B006021
:102B60004060C46042610261816104624262436309
:102B700010BD0000026AC260426A42610261002226
:102B80008262C2626FF00101FEF716BF43690269FB
:102B90009A4203D1C2680AB100207047184650F823
:102BA000043B0B6070470000C368C2690133C36017
:102BB0004369134482694361934224BF436A43617A
:102BC0000021FEF7EDBE000038B504460D46E3686F
:102BD0003BB123691A1DA262E2691344E36200203B
:102BE00038BD237A33B929462046FEF7C9FE0028AE
:102BF000EDDA38BD6FF00100FBE7000003691960F2
:102C0000C268013AC260C269134482690361934297
:102C100024BF436A036100238362036B03B1184737
:102C20007047000070B5202304460E4683F31188D8
:102C3000856A35B91146FFF7C7FF10B185F31188D2
:102C400070BDA36A1E70A36AE26A01339342A36255
:102C500004D3E16920460439FFF7D0FF002080F358
:102C6000118870BD2DE9F84F04460D4691469A46ED
:102C70004FF0200888F311880026B346A76A4FB9A1
:102C800051462046FFF7A0FF20B187F31188304658
:102C9000BDE8F88FA06AE76AA9EB06033F1A9F42D6
:102CA00028BF1F46402F1BD905F1400355F8042BC0
:102CB00040F8042B9D42F9D1A36A4033A362403609
:102CC000A26AE36A9A4204D3E16920460439FFF715
:102CD00095FF8BF311884E45D9D288F31188CDE743
:102CE00029463A46FEF744F8A36A3B443D44A362B2
:102CF0003E44E5E7026943699A4203D1C3681BB9C0
:102D0000184670470023FBE7836A002BF8D0043B8A
:102D10009B1AF5D01360C368013BC360C3691A44B2
:102D2000836902619A4224BF436A0361002383627C
:102D30000123E5E700F06CB94FF0804300225863AF
:102D40001A610222DA6070474FF080430022DA6095
:102D5000704700004FF0804358637047FEE7000063
:102D600010B5174CFEF712FDFEF734FE8022154910
:102D70002046FEF7B9FD012344F8180C0374124BEA
:102D8000124AD96821F4E0610904090C0A43104988
:102D9000DA60CA6842F08072CA600E490A6842F07E
:102DA00001020A601022DA77202283F82220002311
:102DB00083F3118862B60848BDE81040FEF7B6BD3F
:102DC00030260020FC35000800ED00E00003FA0585
:102DD000F0ED00E0001000E0043600082DE9F84FA7
:102DE0001F4C4FF00008656904F11407C1464FF00D
:102DF0008043266A5B6AAA689E1B96421DD34FF0E9
:102E0000200AAA68236AD5F80CB0134423622B6801
:102E1000BB425F60A6EB02066361C5F80C8001D17E
:102E2000FFF792FF89F311882869D8478AF3118840
:102E30006569AB689E42E4D2D9E76269BA420CD0B8
:102E4000916823628E1B9660A86802282CBF181810
:102E5000981CBDE8F84FFFF77DBFBDE8F88F00BFB5
:102E600008260020034B59685A68521A9042FBD832
:102E7000704700BF001000E04B6843608B688360C0
:102E8000CB68C3600B6943614B6903628B69436222
:102E90000B6803607047000008B5224B22481A698E
:102EA00040F2FF110A431A611A6922F4FF7222F0FC
:102EB00001021A611A691A6B0A431A631A6D0A43EE
:102EC0001A651A4A1B6D1146FFF7D6FF184802F122
:102ED0001C01FFF7D1FF174802F13801FFF7CCFFC3
:102EE000154802F15401FFF7C7FF144802F17001C1
:102EF000FFF7C2FF124802F18C01FFF7BDFF114836
:102F000002F1A801FFF7B8FF0F4802F1C401FFF773
:102F1000B3FF0E4802F1E001FFF7AEFFBDE8084045
:102F200000F0E0B8003802400000024024360008FB
:102F30000004024000080240000C02400010024061
:102F40000014024000180240001C02400020024011
:102F500008B500F037FAFFF703FFFFF767F8BDE8A1
:102F60000840FEF741BE000070470000064A536863
:102F700023F001035360EFF30983683383F3098877
:102F8000002383F31188704730EF00E010B5202351
:102F900083F31188104B5B6813F4006318D0F1EED3
:102FA000103AEFF309844FF0807344F84C3C0B4B1C
:102FB000DB6844F8083CA4F1680383F30988FEF752
:102FC00073FC18B1064B44F8503C10BD054BFAE7B2
:102FD00083F3118810BD00BF00ED00E030EF00E08A
:102FE00031030008340300084FF0804310B51A691C
:102FF000920708D500241C61202383F31188FFF772
:10300000EDFE84F31188BDE81040FFF7BFBF00005C
:10301000104B1A6C42F001021A641A6E42F001025F
:103020001A660D4A1B6E936843F0010393604FF0DC
:10303000804353229A624FF0FF32DA6200229A6193
:103040005A63DA605A6001225A6108211A601C2012
:10305000FFF78EBC00380240002004E01F4B1A69C5
:103060006FEAC2526FEAD2521A611A69C2F30802B9
:103070001A614FF0FF301A695A69586100215A6984
:1030800059615A691A6A62F080521A621A6A02F029
:1030900080521A621A6A5A6A58625A6A59625A6A9D
:1030A0001A6C42F080521A641A6E42F080521A660C
:1030B0001A6E0B4A106840F480701060186F00F4AC
:1030C0004070B0F5007F1EBF4FF48030186719675D
:1030D000536823F40073536000F054B90038024081
:1030E00000700040304B4FF080521A642F4A4FF46A
:1030F000404111601A6842F001021A601A68920792
:10310000FCD59A6822F003029A60274B19469A6808
:1031100012F00C02FBD1186800F0F90018609A60F8
:103120001A6842F480321A600B689B03FCD54B6F1F
:1031300043F001034B671C4B5A6F9007FCD51C4AA8
:103140005A601A6842F080721A60184A536859042B
:10315000FCD5154B1A689201FCD5164A9A60164B9D
:103160001A68164B9A42164B1BD1164A1168164A1A
:10317000914216D140F205121A600B4B9A6842F048
:1031800002029A609A6802F00C02082AFAD15A6C7C
:1031900042F480425A645A6E42F480425A665B6E30
:1031A000704740F20572E7E70038024000700040C7
:1031B0000854400700948838002004E0116400207F
:1031C000003C024000ED00E041C20F41084A08B552
:1031D000536911680B4003F00103536123B1054AA1
:1031E00013680BB150689847BDE80840FFF7CEBEA2
:1031F000003C014088250020084A08B55369116841
:103200000B4003F00203536123B1054A93680BB1ED
:10321000D0689847BDE80840FFF7B8BE003C0140C1
:1032200088250020084A08B5536911680B4003F04F
:103230000403536123B1054A13690BB150699847E0
:10324000BDE80840FFF7A2BE003C014088250020F1
:10325000084A08B5536911680B4003F0080353612D
:1032600023B1054A93690BB1D0699847BDE808407E
:10327000FFF78CBE003C014088250020084A08B5B5
:10328000536911680B4003F01003536123B1054AE1
:10329000136A0BB1506A9847BDE80840FFF776BE45
:1032A000003C014088250020174B10B55C691A6866
:1032B000144004F478725A61A30604D5134A936A41
:1032C0000BB1D06A9847600604D5104A136B0BB156
:1032D000506B9847210604D50C4A936B0BB1D06B09
:1032E0009847E20504D5094A136C0BB1506C984716
:1032F000A30504D5054A936C0BB1D06C9847BDE883
:103300001040FFF743BE00BF003C0140882500206D
:103310001A4B10B55C691A68144004F47C425A6177
:10332000620504D5164A136D0BB1506D98472305FD
:1033300004D5134A936D0BB1D06D9847E00404D5C2
:103340000F4A136E0BB1506E9847A10404D50C4A76
:10335000936E0BB1D06E9847620404D5084A136F80
:103360000BB1506F9847230404D5054A936F0BB1F6
:10337000D06F9847BDE81040FFF708BE003C014001
:1033800088250020062108B50846FFF7F1FA062136
:103390000720FFF7EDFA06210820FFF7E9FA0621DA
:1033A0000920FFF7E5FA06210A20FFF7E1FA0621D6
:1033B0001720FFF7DDFA06212820BDE80840FFF7B7
:1033C000D7BA000008B5FFF749FEFDF78DFDFDF700
:1033D0003BFFFDF70FFEFFF7C7FDBDE80840FFF715
:1033E000A9BC0000034611F8012B03F8012B002AA9
:1033F000F9D17047121012131211000053544D33BB
:1034000032463F3F3F00000000000000FC33000850
:103410003F00000013040000383400083F000000A3
:1034200019040000423400083F000000210400009D
:103430004C3400083F00000053544D3332463430C2
:10344000780053544D3332463432780053544D3360
:103450003246343436585800000000006D0F000822
:10346000590F0008950F0008810F00088D0F000804
:10347000790F0008650F0008510F0008F10F0008D0
:103480000000000001000000000000000200000039
:1034900000000000991100080112000840004000DF
:1034A000E02A0020F02A00200200000000000000B6
:1034B00003000000000000004512000800000000AA
:1034C00010000000002B00200000000001000000A0
:1034D00000000000A42D002001010200417264756B
:1034E00050696C6F740025424F415244252D424C67
:1034F000002553455249414C25000000891B000816
:10350000F11A0008051100086D1B000843000000B7
:103510001435000809024300020100C0320904000A
:103520000001020201000524001001052401000130
:10353000042402020524060001070582030800FF97
:1035400009040100020A0000000705010240000012
:1035500007058102400000001200000060350008ED
:10356000120110010200004009124157000201023D
:10357000030100000403090425424F415244250081
:103580004D6174656B46343035003031323334353B
:103590003637383941424344454600000040000078
:1035A000004000000040000000400000000001005A
:1035B0000000020000000200000002000000020003
:1035C00000000200000002000000020000000000F5
:1035D0008D1300086D160008191700084000400000
:1035E000042E0020042E002001000000142E0020D4
:1035F0008000000040010000030000006D61696E62
:10360000000000001C360008202E0020183000208A
:10361000010000005D2D00080000000069646C6579
:10362000000000000000801200000000AAAAAAAA60
:1036300000000000FFBF00000000000000A00A0022
:103640000000140000000000AAAAAAAA00001000AE
:10365000FFFD000000000000000000001500000059
:1036600000000000AAAAAAAA15000000FFFF00009F
:10367000000000000000000000000000000000004A
:10368000AAAAAAAA00000000FFFF00000000000094
:10369000000000000000000000000000AAAAAAAA82
:1036A00000000000FFFF000000000000000000001C
:1036B0000000000000000000AAAAAAAA0000000062
:1036C000FFFF0000000000000000000000000000FC
:1036D00000000000AAAAAAAA00000000FFFF000044
:1036E00000000000000000000000000000000000DA
:1036F0000A000000000000000300000000000000BD
:1037000000000000000000000000000000000000B9
:1037100000000000000000000000000000000000A9
:10372000FF00960000000008040000007435000847
:103730000000000000000000000000000000000089
:103740000000000000000000FFFFFFFFFFFFFFFF81
:10375000FFFFFFFFFFFFFFFFFFFFFFFFFFFFFFFF79
:10376000FFFFFFFFFFFFFFFFFFFFFFFFFFFFFFFF69
:10377000FFFFFFFFFFFFFFFFFFFFFFFFFFFFFFFF59
:10378000FFFFFFFFFFFFFFFFFFFFFFFFFFFFFFFF49
:020000040801F1
:100000000006002099120108C95E0A08255E0A0848
:10001000915E0A08255E0A085D5E0A089B120108C7
:100020009B1201089B1201089B120108D9B80C0809
:100030009B1201089B1201089B1201089B120108E8
:100040009B1201089B1201089B1201089B120108D8
:100050009B1201089B12010871C40C0899C40C087A
:10006000C1C40C08E9C40C0811C50C0881680C084F
:10007000A9680C08D5680C0801690C082D690C08E2
:1000800055690C0881690C0805680C089B12010869
:100090009B1201089B1201089B12010839C50C082C
:1000A00071C60C0885C60C0899C60C089DC60C08BC
:1000B000A1C60C08B5C60C08C9C60C080D6F0C0803
:1000C000B5700C089B1201089B1201089B120108D5
:1000D0009B1201080DC60C0821C60C0835C60C0879
:1000E0009DC50C089B1201089B120108D9C60C087B
:1000F000DDC60C08F1C60C08F5C60C08AD690C0885
:100100009B1201089B1201089B1201089B12010817
:1001100049C60C085DC60C089B1201089B12010819
:10012000D9690C08016A0C082D6A0C08596A0C0878
:10013000856A0C089B1201089B1201089B1201089A
:100140009B1201089B1201089B12010805C00C08B4
:10015000AD6A0C08D96A0C08056B0C089B120108E3
:100160009B1201089B1201089B1201089B120108B7
:100170009B1201089B1201089B1201089B120108A7
:100180009B1201089B1201089B1201089B12010897
:100190009B1201089B1201089B1201089B12010887
:1001A0009B1201089B1201089B1201089B12010877
:1001B0009B1201089B1201089B1201089B12010867
:1001C0009B1201089B1201089B1201089B12010857
:1001D0009B1201089B1201089B1201089B12010847
:1001E00081650108293B030811AF04084132060864
:1001F0006538060819B80608611C07082524070891
:100200005D270708BD87070801AD0708CD4208082C
:10021000259608087DA3080871500A0855550A0854
:10022000093A0B0885A60B08E5CC0B08D1D70B08BB
:100230005D070C08890D0C0800000000000000009C
:1002400081F0004102E000BF83F0004330B54FEA87
:1002500041044FEA430594EA050F08BF90EA020FF4
:100260001FBF54EA000C55EA020C7FEA645C7FEA87
:10027000655C00F0E2804FEA5454D4EB5555B8BFAA
:100280006D420CDD2C4480EA020281EA030382EA1B
:10029000000083EA010180EA020281EA0303362DAD
:1002A00088BF30BD11F0004F4FEA01314FF4801C80
:1002B0004CEA113102D0404261EB410113F0004F92
:1002C0004FEA03334CEA133302D0524263EB430349
:1002D00094EA050F00F0A780A4F10104D5F1200EE7
:1002E0000DDB02FA0EFC22FA05F2801841F1000142
:1002F00003FA0EF2801843FA05F359410EE0A5F116
:1003000020050EF1200E012A03FA0EFC28BF4CF046
:10031000020C43FA05F3C01851EBE37101F00045FC
:1003200007D54FF0000EDCF1000C7EEB00006EEB09
:100330000101B1F5801F1BD3B1F5001F0CD3490893
:100340005FEA30004FEA3C0C04F101044FEA4452EA
:1003500012F5800F80F09A80BCF1004F08BF5FEA71
:10036000500C50F1000041EB045141EA050130BD51
:100370005FEA4C0C404141EB0101013C28BFB1F563
:10038000801FE9D291F0000F04BF01460020B1FAAE
:1003900081F308BF2033A3F10B03B3F120020CDA81
:1003A0000C3208DD02F1140CC2F10C0201FA0CF05F
:1003B00021FA02F10CE002F11402D8BFC2F1200CC4
:1003C00001FA02F120FA0CFCDCBF41EA0C0190407A
:1003D000E41AA2BF01EB0451294330BD6FEA0404C3
:1003E0001F3C1CDA0C340EDC04F11404C4F12002AE
:1003F00020FA04F001FA02F340EA030021FA04F3C0
:1004000045EA030130BDC4F10C04C4F1200220FA16
:1004100002F001FA04F340EA0300294630BD21FA54
:1004200004F0294630BD94F0000F83F4801306BF1A
:1004300081F480110134013D4EE77FEA645C18BF0E
:100440007FEA655C29D094EA050F08BF90EA020FA5
:1004500005D054EA000C04BF1946104630BD91EA9D
:10046000030F1EBF0021002030BD5FEA545C05D1A0
:100470004000494128BF41F0004130BD14F58004DF
:100480003CBF01F5801130BD01F0004545F0FE4153
:1004900041F470014FF0000030BD7FEA645C1ABF88
:1004A000194610467FEA655C1CBF0B46024650EABF
:1004B000013406BF52EA033591EA030F41F40021EB
:1004C00030BD00BF90F0000F04BF0021704730B571
:1004D0004FF4806404F132044FF000054FF0000146
:1004E00050E700BF90F0000F04BF0021704730B507
:1004F0004FF4806404F1320410F0004548BF4042DC
:100500004FF000013EE700BF42004FEAE2014FEA30
:1005100031014FEA02701FBF12F07F4393F07F4F0B
:1005200081F06051704732F07F4208BF704793F00E
:100530007F4F04BF41F40021704730B54FF4607421
:1005400001F0004521F000411CE700BF50EA010224
:1005500008BF704730B54FF000050AE050EA0102CD
:1005600008BF704730B511F0004502D5404261EB3D
:1005700041014FF4806404F132045FEA915C3FF47E
:10058000D8AE4FF003025FEADC0C18BF03325FEA1B
:10059000DC0C18BF033202EBDC02C2F1200300FACC
:1005A00003FC20FA02F001FA03FE40EA0E0021FAF1
:1005B00002F11444BDE600BF70B54FF0FF0C4CF4DF
:1005C000E06C1CEA11541DBF1CEA135594EA0C0F91
:1005D00095EA0C0F00F0DEF82C4481EA030621EACC
:1005E0004C5123EA4C5350EA013518BF52EA033507
:1005F00041F4801143F4801338D0A0FB02CE4FF0B9
:100600000005E1FB02E506F00042E0FB03E54FF0E8
:100610000006E1FB03569CF0000F18BF4EF0010EE0
:10062000A4F1FF04B6F5007F64F5407404D25FEADC
:100630004E0E6D4146EB060642EAC62141EA55518F
:100640004FEAC52040EA5E504FEACE2EB4F1FD0CD1
:1006500088BFBCF5E06F1ED8BEF1004F08BF5FEA4F
:10066000500E50F1000041EB045170BD06F0004601
:1006700046EA010140EA020081EA0301B4EB5C04AE
:10068000C2BFD4EB0C0541EA045170BD41F48011A6
:100690004FF0000E013C00F3AB8014F1360FDEBFCB
:1006A000002001F0004170BDC4F10004203C35DAA7
:1006B0000C341BDC04F11404C4F1200500FA05F32A
:1006C00020FA04F001FA05F240EA020001F00042CB
:1006D00021F0004110EBD37021FA04F642EB060141
:1006E0005EEA430E08BF20EAD37070BDC4F10C046B
:1006F000C4F1200500FA04F320FA05F001FA04F22F
:1007000040EA020001F0004110EBD37041F100011A
:100710005EEA430E08BF20EAD37070BDC4F1200525
:1007200000FA05F24EEA020E20FA04F301FA05F28D
:1007300043EA020321FA04F001F0004121FA04F235
:1007400020EA020000EBD3705EEA430E08BF20EA05
:10075000D37070BD94F0000F0FD101F0004640003F
:1007600041EB010111F4801F08BF013CF7D041EAC1
:10077000060195F0000F18BF704703F000465200C5
:1007800043EB030313F4801F08BF013DF7D043EA96
:100790000603704794EA0C0F0CEA135518BF95EA4C
:1007A0000C0F0CD050EA410618BF52EA4306D1D1D3
:1007B00081EA030101F000414FF0000070BD50EAF2
:1007C000410606BF1046194652EA430619D094EA7C
:1007D0000C0F02D150EA013613D195EA0C0F05D166
:1007E00052EA03361CBF104619460AD181EA0301BA
:1007F00001F0004141F0FE4141F470014FF0000072
:1008000070BD41F0FE4141F4780170BD70B54FF00C
:10081000FF0C4CF4E06C1CEA11541DBF1CEA13558C
:1008200094EA0C0F95EA0C0F00F0A7F8A4EB05046E
:1008300081EA030E52EA03354FEA013100F0888065
:100840004FEA03334FF0805545EA131343EA12632E
:100850004FEA022245EA111545EA10654FEA0026E3
:100860000EF000419D4208BF964244F1FD0404F59C
:10087000407402D25B084FEA3202B61A65EB0305F8
:100880005B084FEA32024FF480104FF4002CB6EBB5
:10089000020E75EB030E22BFB61A754640EA0C0035
:1008A0005B084FEA3202B6EB020E75EB030E22BF75
:1008B000B61A754640EA5C005B084FEA3202B6EBB6
:1008C000020E75EB030E22BFB61A754640EA9C0075
:1008D0005B084FEA3202B6EB020E75EB030E22BF45
:1008E000B61A754640EADC0055EA060E18D04FEA03
:1008F000051545EA16754FEA06164FEAC30343EAA3
:1009000052734FEAC2025FEA1C1CC0D111F4801F6F
:100910000BD141EA00014FF000004FF0004CB6E768
:1009200011F4801F04BF01430020B4F1FD0C88BF07
:10093000BCF5E06F3FF6AFAEB5EB030C04BFB6EB12
:10094000020C5FEA500C50F1000041EB045170BD05
:100950000EF0004E4EEA113114EB5C04C2BFD4EB32
:100960000C0541EA045170BD41F480114FF0000EB6
:10097000013C90E645EA060E8DE60CEA135594EA32
:100980000C0F08BF95EA0C0F3FF43BAF94EA0C0F35
:100990000AD150EA01347FF434AF95EA0C0F7FF4AA
:1009A00025AF104619462CE795EA0C0F06D152EAFE
:1009B00003353FF4FDAE1046194622E750EA4106E2
:1009C00018BF52EA43067FF4C5AE50EA41047FF4F3
:1009D0000DAF52EA43057FF4EBAE12E74FF0FF3C58
:1009E00006E000BF4FF0010C02E000BF4FF0010C29
:1009F0004DF804CD4FEA410C7FEA6C5C4FEA430CA2
:100A000018BF7FEA6C5C1BD001B050EA410C0CBFF0
:100A100052EA430C91EA030F02BF90EA020F002052
:100A2000704710F1000F91EA030F58BF994208BFB9
:100A300090422CBFD8176FEAE37040F00100704776
:100A40004FEA410C7FEA6C5C02D150EA013C07D1CD
:100A50004FEA430C7FEA6C5CD6D152EA033CD3D018
:100A60005DF8040B704700BF8446104662468C4612
:100A70001946634600E000BF01B5FFF7B7FF002845
:100A800048BF10F1000F01BD4DF808EDFFF7F4FF6E
:100A90000CBF012000205DF808FB00BF4DF808EDF9
:100AA000FFF7EAFF34BF012000205DF808FB00BF1C
:100AB0004DF808EDFFF7E0FF94BF012000205DF83E
:100AC00008FB00BF4DF808EDFFF7CEFF94BF0120F3
:100AD00000205DF808FB00BF4DF808EDFFF7C4FFEC
:100AE00034BF012000205DF808FB00BF4FEA410C35
:100AF0007FEA6C5C02D150EA013C0AD14FEA430C18
:100B00007FEA6C5C02D152EA033C02D14FF0000054
:100B100070474FF0010070474FEA410212F5001292
:100B200015D211D56FF47873B3EB625212D94FEA34
:100B3000C12343F0004343EA505311F0004F23FA1E
:100B400002F018BF404270474FF00000704750EA73
:100B5000013005D111F0004008BF6FF00040704730
:100B60004FF00000704700BF4A0011D212F500128A
:100B700011D20DD56FF47873B3EB62520ED44FEAF5
:100B8000C12343F0004343EA505323FA02F0704775
:100B90004FF00000704750EA013002D14FF0FF30B3
:100BA00070474FF0000070474FEA4102B2F1E04356
:100BB00024BFB3F5001CDCF1FE5C0DD901F0004C44
:100BC0004FEAC0024CEA5070B2F1004F40EB830094
:100BD00008BF20F00100704711F0804F21D113F1C0
:100BE0003872BCBF01F00040704741F480114FEAF9
:100BF0005252C2F11802C2F1200C10FA0CF320FA82
:100C000002F018BF40F001004FEAC1234FEAD3239E
:100C100003FA0CFC40EA0C0023FA02F34FEA430308
:100C2000CCE77FEA625307D150EA01331EBF4FF091
:100C3000FE4040F44000704701F0004040F0FE40AC
:100C400040F40000704700BF80F0004002E000BFA9
:100C500081F0004142001FBF5FEA410392EA030FA7
:100C60007FEA226C7FEA236C6AD04FEA1262D2EBF1
:100C70001363C1BFD218414048404140B8BF5B42F6
:100C8000192B88BF704710F0004F40F4000020F08F
:100C90007F4018BF404211F0004F41F4000121F0A5
:100CA0007F4118BF494292EA030F3FD0A2F10102EF
:100CB00041FA03FC10EB0C00C3F1200301FA03F12D
:100CC00000F0004302D5494260EB4000B0F5000F50
:100CD00013D3B0F1807F06D340084FEA310102F10F
:100CE0000102FE2A51D2B1F1004F40EBC25008BFC1
:100CF00020F0010040EA03007047490040EB00008B
:100D0000013A28BFB0F5000FEDD2B0FA80FCACF18B
:100D1000080CB2EB0C0200FA0CF0AABF00EBC250B8
:100D200052421843BCBFD0401843704792F0000FA6
:100D300081F4000106BF80F400000132013BB5E7F9
:100D40004FEA41037FEA226C18BF7FEA236C21D06F
:100D500092EA030F04D092F0000F08BF08467047D4
:100D600090EA010F1CBF0020704712F07F4F04D1A2
:100D7000400028BF40F00040704712F100723CBFB5
:100D800000F50000704700F0004343F0FE4040F4DF
:100D9000000070477FEA226216BF08467FEA23639D
:100DA0000146420206BF5FEA412390EA010F40F488
:100DB000800070474FF0000304E000BF10F00043D4
:100DC00048BF40425FEA000C08BF704743F09643BB
:100DD00001464FF000001CE050EA010208BF7047D6
:100DE0004FF000030AE000BF50EA010208BF70475D
:100DF00011F0004302D5404261EB41015FEA010C72
:100E000002BF84460146002043F0B64308BFA3F169
:100E10008053A3F50003BCFA8CF2083AA3EBC2534B
:100E200010DB01FA02FC634400FA02FCC2F120026A
:100E3000BCF1004F20FA02F243EB020008BF20F0A1
:100E40000100704702F1200201FA02FCC2F1200207
:100E500050EA4C0021FA02F243EB020008BF20EAFC
:100E6000DC7070477BB972B90029BEBF00204FF01B
:100E7000004106E008BF00281CBF6FF000414FF0A2
:100E8000FF3000F007BAADF1080C6DE904CE00297F
:100E900009DB002B1ADB00F095F8DDF804E0DDE952
:100EA000022304B07047404261EB4101002B1BDB81
:100EB00000F088F8DDF804E0DDE9022304B04042E8
:100EC00061EB4101524263EB43037047524263EBD3
:100ED000430300F077F8DDF804E0DDE9022304B015
:100EE000404261EB41017047524263EB430300F023
:100EF00069F8DDF804E0DDE9022304B0524263EB57
:100F00004303704753B94AB9002908BF00281CBFE2
:100F10004FF0FF314FF0FF3000F0BCB9ADF1080CDD
:100F20006DE904CE00F04EF8DDF804E0DDE90223BF
:100F300004B07047430803F05533C01A830803F028
:100F4000333300F03330184400EB101000F00F3052
:100F500000EB002000EB0040000E704707EE900A07
:100F6000F5EEC07AF1EE10FA01D400F00BB8F1EE14
:100F7000677A08B517EE900A00F004F8404261EB7A
:100F8000410108BDD0B5FFF7BFFA0C4B0022064661
:100F90000F46FFF711FBFFF7E7FD0446FFF792FA54
:100FA000074B0022FFF708FB02460B463046394646
:100FB000FFF74AF9FFF7D8FD2146D0BD0000F03D0C
:100FC0000000F0412DE9F047089D04468E46002BB5
:100FD0004DD18A42944669D9B2FA82F252B101FAED
:100FE00002F3C2F1200120FA01F10CFA02FC41EAFD
:100FF000030E94404FEA1C48210CBEFBF8F61FFA82
:101000008CF708FB16E341EA034306FB07F199421C
:101010000AD91CEB030306F1FF3080F01F819942CF
:1010200040F21C81023E63445B1AA4B2B3FBF8F0A9
:1010300008FB103344EA034400FB07F7A7420AD930
:101040001CEB040400F1FF3380F00A81A74240F258
:1010500007816444023840EA0640E41B00261DB1C3
:10106000D4400023C5E900433146BDE8F0878B42F8
:1010700009D9002D00F0EF800026C5E900013046B7
:101080003146BDE8F087B3FA83F6002E4AD18B4291
:1010900002D3824200F2F980841A61EB030301203B
:1010A0009E46002DE0D0C5E9004EDDE702B9FFDE27
:1010B000B2FA82F2002A40F09280A1EB0C014FEAD2
:1010C0001C471FFA8CFE0126200CB1FBF7F307FB2F
:1010D000131140EA01410EFB03F0884208D91CEBD2
:1010E000010103F1FF3802D2884200F2CB8043466F
:1010F000091AA4B2B1FBF7F007FB101144EA01444E
:101100000EFB00FEA64508D91CEB040400F1FF31DC
:1011100002D2A64500F2BB800846A4EB0E0440EACA
:1011200003409CE7C6F12007B34022FA07FC4CEAD3
:10113000030C20FA07F401FA06F31C43F9404FEAC6
:101140001C4900FA06F3B1FBF9F8200C1FFA8CFEDB
:1011500009FB181140EA014108FB0EF0884202FA2F
:1011600006F20BD91CEB010108F1FF3A80F08880F0
:10117000884240F28580A8F102086144091AA4B2AD
:10118000B1FBF9F009FB101144EA014100FB0EFE2E
:101190008E4508D91CEB010100F1FF346CD28E455D
:1011A0006AD90238614440EA0840A0FB0294A1EBEE
:1011B0000E01A142C846A64656D353D05DB1B3EB4B
:1011C000080261EB0E0101FA07F722FA06F3F1407B
:1011D0001F43C5E9007100263146BDE8F087C2F122
:1011E0002003D8400CFA02FC21FA03F3914001439A
:1011F0004FEA1C471FFA8CFEB3FBF7F007FB1036D3
:101200000B0C43EA064300FB0EF69E4204FA02F47E
:1012100008D91CEB030300F1FF382FD29E422DD9D1
:10122000023863449B1B89B2B3FBF7F607FB163306
:1012300041EA034106FB0EF38B4208D91CEB010186
:1012400006F1FF3816D28B4214D9023E6144C91A06
:1012500046EA004638E72E46284605E70646E3E616
:101260001846F8E64B45A9D2B9EB020864EB0C0E20
:101270000138A3E74646EAE7204694E74046D1E72F
:10128000D0467BE7023B614432E7304609E76444DD
:10129000023842E7704700BF02E000F000F8FEE7C6
:1012A00072B6374880F30888364880F30988364894
:1012B0003649086040F20000CCF200004EF634716E
:1012C000CEF200010860BFF34F8FBFF36F8F40F283
:1012D0000000C0F2F0004EF68851CEF20001086026
:1012E000BFF34F8FBFF36F8F4FF00000E1EE100A96
:1012F0004EF63C71CEF200010860062080F314889F
:10130000BFF36F8FBAF046FBB9F072FB4FF0553068
:101310001F491B4A91423CBF41F8040BFAE71D49A3
:10132000184A91423CBF41F8040BFAE71A491B4A9C
:101330001B4B9A423EBF51F8040B42F8040BF8E7EE
:1013400000201849184A91423CBF41F8040BFAE7C3
:10135000BAF024FBB9F0A0FB144C154DAC4203DAF3
:1013600054F8041B8847F9E701F096FB114C124D25
:10137000AC4203DA54F8041B8847F9E7BAF00CBB17
:1013800000060020002200200000010808ED00E017
:101390000000002000060020A05F0F0800220020AF
:1013A0007C2B0020802B0020C0580120E001010888
:1013B0003802010838020108380201082DE9F04F0F
:1013C0002DED108AC1F80CD0C3689D46BDEC108A83
:1013D000BDE8F08F002383F311882846A047002042
:1013E000B9F078F8FEE7B8F0D5FE00DFFEE70000C0
:1013F00001F0FF01102A2BDB10F0070F08D010F8C6
:10140000013B013A8B422DD010F0070F42B3F6D1C9
:10141000F0B441EA012141EA014122F007047FF0E2
:1014200000070023F0E80256083C85EA010586EA39
:10143000010685FA47F5A3FA87F586FA47F6A5FA75
:1014400087F68EB9EED1F0BC01F0FF0102F0070281
:1014500032B110F8013B013A83EA010313B1F8D12C
:101460000020704701387047002D06BF354603380D
:10147000073815F0010F07D1013015F4807F02BF46
:10148000013015F4C03F0130F0BC0138704700BF97
:1014900010F8012B11F8013B012A28BF9A42F7D01E
:1014A000D01A7047034613F8012B002AFBD1181AF3
:1014B0000138704738B50022002304460D46FFF777
:1014C000EDFA28B920462946BDE8384000F00AB8B0
:1014D000204605F1004100F005F8404261EB410172
:1014E00038BD00BFD0B50C4B002206460F46FFF7B3
:1014F00063F8FFF739FB0446FEF7E4FF074B0022D1
:10150000FFF75AF802460B4630463946FEF79CFE76
:10151000FFF72AFB2146D0BD0000F03D0000F0415E
:10152000036800221B68184710B503685B6804460F
:10153000984708B194F84D0010BD00002DE9F04126
:10154000664B03F5C04490B094F9842106460F46DB
:10155000002A00F0C08094F8CC5135B9604A82F07E
:1015600039FE284610B0BDE8F081B3F9A4201AB9BD
:10157000B3F8A220A3F8A420B3F8A430632B05D8B5
:10158000584A3946304682F025FE002500212E2299
:1015900004A80391BEF03CF9D4F8E400036803AA60
:1015A0001B6832219847804630B94F4A03AB394611
:1015B000304682F00FFE4546B4F8C030A3F57A738A
:1015C0009BB241F65832934206D9484B3A46202105
:1015D000304682F01DFC002594F9F432002B69DDC1
:1015E00094F9AC32002B59DD414B3A46202130466C
:1015F00082F00EFC00253F49D4F8F000322303AA04
:101600008DF0E8FD804640B903AB00933A463A4B73
:101610002021304682F0FCFB45463849D4F8EC00E6
:10162000322303AA8AF008FE804640B903AB009338
:101630003A46314B2021304682F0EAFB45462021D4
:10164000304682F0DDFBB8B1D4ED507A9FED2C7AB4
:10165000F0EEE77AF4EEC77AF1EE10FA0CD594F9D1
:10166000F432002B02DD94F858332BB9254A394661
:10167000304682F0AFFD002594F9F432002B7FF75D
:1016800070AF94F9B131002B3FF46BAF1E4B3A466B
:101690002021304682F0BCFB002562E794F8588395
:1016A000B8F1000F06D1194B3A462021304682F09E
:1016B000AFFB454694F9AC32002B9CDD94F8DD82FB
:1016C000B8F1000F97D1124B3A462021304682F0F4
:1016D0009FFB45468FE7012543E700BF902B002085
:1016E000783C0D089A3C0D08C13C0D08CC3C0D0817
:1016F000DE3C0D084F3D0D08533D0D08653D0D08BE
:1017000000000034693D0D08833D0D08043D0D08BF
:101710002A3D0D0838B5044682F056FB114B93F86C
:101720009012114B1D68EB6A1A68002908BF014628
:101730001268184690475BF0EDFFEB6A93F89C1037
:101740005AF0D4FF94F837305BB194F0EFFBEB6ABA
:10175000D3F8A030C01AB0F5FA6F24BF002384F884
:10176000373038BD908B00208C2B002008B5FFF758
:10177000D1FF054B05481B68DB6A93F89C10BDE858
:10178000084011F0F7B900BF8C2B0020488C0020D6
:1017900070B50E46054667F031FA67F0F3F910B9F7
:1017A0000124204670BD0A4B93F90A32012BF7D170
:1017B00067F024FA437A002BF2D167F01FFA847A9B
:1017C000002CEDD1034A3146284682F003FDE8E7BC
:1017D000904B00209C3D0D08034BD3F874320BB99D
:1017E00082F0A8BA01207047904B00202DE9F04705
:1017F0002DED028BC47F90B006460F468CB990F950
:101800000430002B00F00581834B1D68A86A036833
:101810005B6B9847044650B9804A3946304682F09F
:10182000D9FC204610B0BDEC028BBDE8F087B36850
:101830004BB933685B6B3946304610B0BDEC028B58
:10184000BDE8F0471847E86AFFF76EFE0446002837
:10185000E7D13946304683F051FBDFF8F481054685
:101860003946304682F0DEFC98ED877AD8ED867AEC
:10187000B4EEE77A2840F1EE10FAC5B209D598F92E
:101880001432032B05D0664A3946304682F0A2FC5A
:101890002546D8ED6F7AB0EE088AF4EEC87AF1EEFC
:1018A00010FA0BD517EE900AFEF72EFE5D4ACDE931
:1018B00000013946304682F08DFC0025D8ED707A63
:1018C000F4EEC87AF1EE10FA0BD517EE900AFEF797
:1018D0001BFE554ACDE900013946304682F07AFCBC
:1018E0000025D8ED717AB8EE087AF4EEC77AF1EEF9
:1018F00010FA0BDD17EE900AFEF706FE4B4ACDE913
:1019000000013946304682F065FC0025B8F9A8315F
:10191000042B07DC052200923946454A304682F006
:1019200059FC0025D8F8300C67F0C4F980B198F95B
:101930000A326BB1D8F8303CB8F90C22B3F90E304A
:101940009A4205DA3B4A3946304682F043FC00258C
:1019500039463046FFF71CFFDFF8F8A081463946CC
:101960003046FFF7EBFD9AF8353F002B4AD109EAE4
:10197000050500EA050430484FF4806101F06EF877
:1019800078B1D8F8303CB3F90C30A3F2E24292B20D
:10199000B2F5FA7F05D9294A3946304682F01AFC59
:1019A0000024274890F888355BB100F5B06038F026
:1019B0002FFB054628B9234A3946304682F00AFCF7
:1019C0002C4600212E2204A80DF10C080391BDF035
:1019D0001FFFDAF8200F4246322109F06FFD05465D
:1019E00000287FF41EAFDAF8200F03689B68984741
:1019F000154ACDF8008003463946304682F0EAFBAE
:101A00002C460EE7114A3946304682F0E3FB0024AB
:101A1000B1E7012405E700BF8C2B0020AC3D0D0889
:101A2000C33D0D08E63D0D08063E0D08283E0D0895
:101A30004A3E0D08693E0D08902B0020A43E0D087B
:101A4000907B0020CC3E0D086C0C0E088F3E0D08DC
:101A5000904B0020906B002070B505460E46FFF7B6
:101A600097FE31460446284683F0FEF82040C0B277
:101A700070BD0000F0B591B005460E4682F072FCD4
:101A80000446D8B11021284682F0BAF9B0B100213D
:101A90002E2204A803AF0391BDF0BAFE1BF09CFFF9
:101AA00032233A4601211BF057FA044630B9054B60
:101AB000009732461021284682F0AAF9204611B03C
:101AC000F0BD00BFE03E0D0870B505460E46B1B949
:101AD00090F910408CB1164813F07EFFDFED157AB7
:101AE000B0EEC00AB4EEE70AF1EE10FA07D4124ADB
:101AF0000121284682F06EFB3446204670BDAB685B
:101B00009BB10E4B1B68D86AFFF70EFD044630B13F
:101B100065F0C8FD0A4A04215EF048FFEDE7314652
:101B20002846BDE8704082F0E9BE0124E5E700BF29
:101B3000902B002000000034EC3E0D088C2B002080
:101B4000FE3E0D0838B5044683F092FA0546A8B16A
:101B50000B4806F07FFB38B10A490B481BF054FBD9
:101B600010B1074800F04EFF2046FFF7FFFD0123AC
:101B7000064984F83730204683F090F9284638BD6E
:101B8000902B0020748B0020503E0020203F0D0839
:101B9000F8B505460E461746C2B1232901D00129E2
:101BA00014D8254808F04CFF044668B100242046AC
:101BB000F8BD95F91030022B08D065F073FD1F4A6F
:101BC00006215EF0F3FEF2E7002EF2D03A463146EF
:101BD000284683F003FB04460028E7D0184ED6F8C9
:101BE000202F06F548639A4203D006F5AC5038F032
:101BF00045FED6F8200F134F03689B6B984787F874
:101C0000580507F58057D7F80831012B07D166F042
:101C1000F5FF542167F0B4FF08B9C7F8080128465A
:101C2000FFF7A4FD4FF0FF330749C6F8583F284699
:101C300083F034F9BBE700BF902B0020303F0D0844
:101C4000906B0020907B0020483F0D082DE9F04F5D
:101C50002DED028BDFF8489191B00746884682F05F
:101C600055F999F9DF510446D5B9BD2109F556500A
:101C700038F09AFD38B1434B42464FF48041384624
:101C800082F0C6F82C464048BC2138F08DFD38B1B2
:101C90003E4B42464FF48041384682F0B9F800246A
:101CA0003B4E96F8CC31002B66D0A6F580531C2213
:101CB000002102A8B3F8B4A5DFED368ABDF0A8FD77
:101CC00004A821F005FBA6F5286B0125A6F5C04662
:101CD000554551D20BA821F0FBFA09AA29465846CE
:101CE00036F002FA002847D0BDF82610304607F03B
:101CF000C7FF80B3BDF80A30102B2CD104A90BA864
:101D000021F048FE09F64853B0EE408A93ED000AF0
:101D10002148B4EEE80AF1EE10FAB8BF99ED6B0A6B
:101D200020EE000A0FF032F8F6EE087A60EE277A1D
:101D3000B4EEE78AF1EE10FA0DD517EE900AFEF731
:101D4000E3FB164BCDE9000142464FF48041384693
:101D500082F05EF800240DF1240CBCE80F000DF1B8
:101D6000080EAEE80F009CE80700AEE8030001355E
:101D70008EF80020ADB2ABE7204611B0BDEC028B6F
:101D8000BDE8F08F5C3F0D0810810020883F0D08F2
:101D9000908B002000000034488C0020BB3F0D08D1
:101DA000904B002000207047014800F0ABBD00BF01
:101DB000902B002003685B68184700006AF05EB94A
:101DC00066F06ABE30F05EB95AF012BE08F08ABF03
:101DD00058F0FEBE0DF062BC15F05CB803F010BB0D
:101DE00057F092BA1FF08ABC69F0EEBC15F0B8B893
:101DF00013F070BE1EF0E0BF6BF0CEBE66F066BBA7
:101E000064F020BD08F01EB905F096B90CF014BFBF
:101E10000DF0A2BB14F07CBE15F050B913F08EBCCF
:101E200014F0B2BF01F0B6BB00F2545022F01ABB5E
:101E300008F096BC90F8C432B02202FB030390F87D
:101E4000082393F8A13012B1012B28BF01231846B3
:101E50007047000090F814310BB190F841311846EA
:101E600070470000034808602A21117008221A6098
:101E7000704700BFEC420D08F8B5044600F5C040BD
:101E8000703004F59656FFF745FC002130461BF0F4
:101E900015FD8021204615F081FB18B131F0E6FCDC
:101EA0002FF07EFD04F50055D5ED6F7A9FED317A68
:101EB00067EE877A05F64447FDEEE77A04F5C540FC
:101EC00017EE903AC5F8403CD5F8C4313B6070300D
:101ED00015F066FDF8B9D5F8403C07EE903A04F5E8
:101EE000805303F20C5292ED007AF8EEE77A03F594
:101EF000A16367EE877AFDEEE77A17EE902AC5F8C0
:101F0000402CD3ED007A97ED007AF0EEE77A67EE99
:101F1000877AC7ED007A04F5AF51183106F54570A0
:101F200035F060FB04F5A94594ED467AD5ED167AB7
:101F3000E7EE007AC5ED167AB0EE670A32F0BEF928
:101F400004F5C14085ED160A38300EF02FF804F57F
:101F5000C1400021443087F081F84FF40011204641
:101F600015F01CFB20B13046BDE8F84019F0D0BD9B
:101F7000F8BD00BF0000C842FFF77EBF70B500F596
:101F800080430546D3F8200F03689B6B984705F5FF
:101F9000C14438340646204610F0AEFD05F5A04396
:101FA000002893F8173518BF00262BB926B105F580
:101FB0003350183086F0B6FF204610F033FA18B9C7
:101FC0002046FFF747FF20B12046BDE8704010F0E3
:101FD000E1BF70BDFFF7D2BF38B54FF480110546A1
:101FE00015F0DCFA044620B90121284615F0D6FA8E
:101FF00004460221284615F0D1FA48B114B9284602
:1020000003F024F905F59650BDE8384019F07EBC80
:10201000002CF7D138BD0000FFF7DEBF38B54FF414
:102020008011044615F0BAFA01210546204615F044
:10203000B5FA18B115B9204603F008F91021204669
:1020400015F0ACFA60B1204603F0F2F94FF48001CC
:10205000204615F0A3FA18B931F008FC2FF092FDD4
:102060002021204615F09AFA28B1204603F056FAAE
:10207000204603F071FB4FF40051204615F08EFA14
:1020800010B1204603F050FB8021204615F086FA5F
:1020900028B131F0EBFBBDE838402FF0A5BC38BDCE
:1020A000FFF7BCBF10B5044622F0CCFA90F92130FE
:1020B0008BB190F8403373B194F978355BB1064B2E
:1020C0001B68DB6A93F89C302BB904F25450BDE8CE
:1020D000104021F0DFBF10BD8C2B0020FFF7E2BFC6
:1020E0002DE9F843434B1B68DB6A93F89C300446A8
:1020F000002B7CD000F5805797F8C935002B76D09F
:1021000008F09EFC002872D004F5F75507F58059B9
:10211000083599F83610284618F09CFF002866D03C
:1021200004F590763046FFF785FE02285FD994F8D3
:10213000E4334FF0B00808FB034393ED777AF1EEF8
:10214000007AB4EEE77AF1EE10FA50D499F836102E
:10215000284619F02FFA04F50053B3F9A82107EE29
:10216000902AB8EEE77AB4EEC07AF1EE10FA0CDD00
:1021700094F8E42308FB0242F8EE677A92ED777A4E
:10218000F4EEC77AF1EE10FA31DCD7F8B824D3F8C0
:10219000401C002AB8BF52428A4228DC07F2BC42E7
:1021A000D2ED007AD3ED706A9FED136AF8EEE77A0C
:1021B00066EE866AF4EEE67AF1EE10FA17DC03F6C4
:1021C000444292ED007A27EE067AF4EEC77AF1EEF9
:1021D00010FA0CD494F8E413B02202FB01612846F3
:1021E000B3F9AA21D431BDE8F84318F0B1BDBDE878
:1021F000F88300BF8C2B00200000C842FFF770BF9F
:102200002DE9F04190F8E4332D4D00EB03132F68D6
:10221000D3F8948100F5907604463046FFF70AFE25
:10222000474514D0022814D904F58047C5F800802A
:1022300097F8503F012B15D817D104F5A045D5F8D4
:10224000EC3FE3B9D5F8F03FCBB905230BE002280A
:1022500010D804F5804393F8502F5AB1052283F823
:10226000502F07E0013B87F8503F04F5B7501C3072
:102270001CF066FD2046BDE8F0410CF0C7BE114BD6
:102280001B68D86A03685B68984780460028ECD1D1
:1022900094F8E413B02303FB0161AC31204606F04F
:1022A00049F8D5F8D03F0FCB05F6D47605F6F4758E
:1022B00086E80F0085E80F0087F8508FD5E700BF4C
:1022C000802B00208C2B0020FFF79ABF70B500F503
:1022D000C043044693F8CC3100F58056BBB100F5FD
:1022E000C540703015F062FE18B1012386F8C9357B
:1022F00070BD04F5C1453835284610F093F808B193
:102300000023F3E72846FFF7A5FD0028F8D104F5E0
:10231000A04393F81725002AF2D1D3F85C35042B9B
:10232000E3D104F5BE40143090F038F886F8C905C2
:10233000DEE7000010B500F5804400F59943D4F8BD
:10234000201F994200F5A04308D000F59C420832B6
:1023500091421CBF4FF0FF32C3F8D02403F59862BE
:102360000749116003F2C443064A1A60FFF7AEFF43
:10237000D4F8200F0368BDE810401B69184700BF60
:102380000000C8420000C8C2FFF7D4BFF7B500F58F
:10239000A0470446D7F85C358B420D4624D00B1F6E
:1023A00000F5BE46594206F11406594130460191E6
:1023B0008FF0E4FE019930468FF0E0FE072D0BD13F
:1023C00004F54F50D7F8E0246423052192FBF3F382
:1023D0002830064A5EF0EAFA2046C7F85C5503B09A
:1023E000BDE8F04003F006B903B0F0BD4C400D0865
:1023F00070B500F580460446D6F8200F03689B6B45
:102400009847B0B104F5A04595F858358BB9D6F882
:10241000202F04F599439A424CD104F5C146383631
:1024200030460FF013FA60B995F810357BB90121E9
:1024300008E004F5C145383528460FF0F3FF0028C1
:102440003ED002212046BDE87040FFF79FBFB5F89F
:10245000BE35152B27D195F8181F11F0010120D199
:10246000D5F85C35072B1CD095F98E3F0BB90421AC
:10247000E8E7204613F0B0FADFED127AB4EEE70A8F
:10248000F1EE10FAF3DB04F5BE4014308FF0C6FE17
:102490000028ECD004F54F500B4A062128305EF09E
:1024A00085FA0721CEE73046FFF7D4FC0028C8D1D3
:1024B0000321C7E704F59C4308339A42F8D170BD65
:1024C0002846F1E70000B44270400D0838B5314CA1
:1024D000D4F8202F04F548639A422DED028B05466F
:1024E000B0EE408A03D00020BDEC028B38BD2A48F4
:1024F0000FF0ACF940B1BDEC028B05F5C1403830AE
:10250000BDE8384010F0C6BA04F58055D5F85C3502
:10251000042B35D194F8513F33B12049A1F6642002
:1025200038F024FC0028DFD11D4C94F8CC315BB18D
:1025300004F1B8000FF08AF90028D4D104F1B800F2
:102540000FF044F90028CED19FED167AF0EEC87A4C
:10255000F4EEC77AF1EE10FA09D49FED130A28EED3
:10256000008ABDEEC88A18EE103AC5F8E0340F486C
:102570008FF054FE0028B6D0002385F81335B3E75A
:10258000B5F8BE15A4F5804007F07AFB0028C1D14C
:10259000A9E700BF906B0020488C0020748B0020BE
:1025A000908B0020000000340000C842A48A002064
:1025B00010B52DED028B00F5A0430446D3F85C3531
:1025C000042B0BD105F036F82046B0EE408A05F01A
:1025D00055F938EE400ABDEC028B10BD00F5C04441
:1025E00094ED080AF7E700002DE9F0412DED028B8C
:1025F00000F586658AB0044628461DF059FD002383
:1026000007A904F596500793089309931AF0E2FF7F
:10261000002800F08D809DED090ADFED5D7A04F55C
:10262000A04505F59E6393ED007A20EE270ADFEDC5
:10263000597AA7EE270A04F58047204683ED000A61
:10264000FFF7D6FED7F8200F03689B6B9847064626
:1026500004F5C140383010F04FFA95F817350028CE
:1026600018BF0026002B5ED1002E5CD095F858359F
:10267000002B58D1D5F85C35042B70D09FED468ADD
:10268000204605F01DF904F5C04204F59943C2F84F
:102690001C04D7F8201F2C3399421CD192F86830C3
:1026A000CBB904F50053B3F90C3C002B04DC3B49D7
:1026B000D1F8EC1BC9060ED5D5F8D06FD5F8D81FC8
:1026C00076680A33891B642673438142ACBF5B186A
:1026D0001B18C2F81C34D5F85C35D2F81C14D7F896
:1026E000542F059120460492039316F05DFCB7F930
:1026F000627F06462046FFF75BFFCDE9006704F5E1
:102700000050D0ED911A059905F5AF6504F53350E9
:10271000F0EE400ADDE9033295ED001AB0EE480A0A
:10272000183086F0A3F80AB0BDEC028BBDE8F0814A
:1027300004F59070FFF77EFB02280AD994F8E43381
:10274000B02202FB034393F8102212B193ED7F0AEB
:1027500063E728461DF046FBB1EE400A5DE704F54D
:10276000BF4604F5BF48643608F1740804F5BF415C
:1027700042465431304621F079F800283FF47EAFCC
:102780004146304621F006F9B0EE408A78E700BFB6
:10279000CDCC4C3ECDCC4C3F00000000904B0020F7
:1027A000FFF722BFF8B500F5804200F59A43D2F852
:1027B000202F20339A4204460E4623D000F5C1470D
:1027C000383738460FF02EFE0546A8B138460EF0D1
:1027D000A5FA70B104F5C044D4F8F40003689B680E
:1027E0009847DFED097A20EE270A86ED000A284691
:1027F000F8BD9FED060AF8E704F5A9440125A36F8B
:102800003360F4E70025F2E70AD7233C000000001C
:10281000F8B500F5804200F59A43D2F8202F203316
:102820009A4204460E4630D000F5C1473837384644
:102830000FF0F8FD0546A8B138460EF06FFA70B1FA
:1028400004F5C044D4F8F4000368DB68984707EE49
:10285000900AF8EEE77AC6ED007A2846F8BDDFED7B
:102860000C7AF8E704F540540125D4F8040603680F
:102870001B69984707EE900A9FED067AF8EEE77A13
:1028800067EE877AC6ED007AE7E70025E5E700BF47
:10289000000000000AD7233CF8B500F5804200F59F
:1028A0009A43D2F8202F20339A4204460E4624D071
:1028B00000F5C147383738460FF0B4FD054688B1FA
:1028C00038460EF02BFA50B104F5C044D4F8F43079
:1028D00018698BF0E9FB86ED000A2846F8BD9FEDEC
:1028E000080AF8E704F540540125D4F80406036803
:1028F0005B69984786ED000AEFE70025EDE700BF2A
:102900000000000030B505460FC985B06C4684E86C
:102910000F0040F279322146284605F09DFB0C4B12
:1029200003F6E442D3F8203F93420ED19DF8001005
:1029300011F0040102D1204620F094FD0548214603
:1029400005F044FC012005B030BD0020FBE700BFCE
:10295000906B0020902B002010B5044606480FF025
:1029600095FB40B904F58044D4F8200F0368BDE816
:1029700010409B6C184710BD488C002010B50446D1
:1029800006480EF0D1FF40B904F58044D4F8200F7A
:102990000368BDE81040DB6C184710BD488C002070
:1029A00070B5044600F5C14038300E4615460EF0AD
:1029B00017FB50B104F5C044D4F86C339B682B600E
:1029C000D4F86C335B68336070BD04F5805303F555
:1029D000996203F2C44312682A601B68336004F5ED
:1029E0000054D4F8EC3B9B05EED4D4ED916AD5EDC0
:1029F000007A9FED037AE6EEC77AC5ED007AE3E749
:102A000035FA8E3C38B50C4D044629460B481AF071
:102A10000DFD04F5804305F13C0183F8510F04F5E9
:102A2000965004F5C0441AF099FBD4ED087AF1EE03
:102A3000677AC4ED087A38BD748B0020503E0020C0
:102A400010B5044600F590702AF07EF92046BDE8E6
:102A50001040FFF7D7BF0000FFF7F2BF00F50050AE
:102A6000D0F8EC3B194214BF012000207047000051
:102A700010B500F580430446D3F8200F03689B6D22
:102A80009847014604F59C406030BDE8104091F045
:102A900033BE0000FFF7ECBF38B5054B1C68236858
:102AA0000A461D68034B01462046A847002038BD52
:102AB0008C2B0020902B002070B52DED028B04464E
:102AC000036804F500559B6D9847D5F8EC3B1B0651
:102AD00017D5B5F9A831B5F9AA11CA1A0B4402EBFA
:102AE000D27203EBD37352105B1000EE902A00EE0B
:102AF000103AF8EEE00AB8EEC00A04F596501AF063
:102B0000B3F85F4BB5F8DA211A7004F5C04568F0E8
:102B1000F1F8703567F080FD00212846FEF766FE6B
:102B2000584E0123B0712846F37181F04DF928B950
:102B3000284682F0C7F9B0FA80F0400930710421CC
:102B4000204614F02BFD20B104F5AC40783058F04D
:102B5000F1F8284681F038F904F5C045C8B994F871
:102B6000E43304EB031341F28832D3F89461EB6E43
:102B7000F31A93420DD904F59070FFF75BF9022820
:102B800007D9EE66204605F065FB04F5BE4300223A
:102B90005A61B4F9A4301BB9B4F8A230A4F8A43037
:102BA000B4F8A430DFED388A07EE903AF8EEE77A11
:102BB000B7EE008A88EE270AD4ED2B7AF0EEE77A9A
:102BC000F4EEE87AF1EE10FA09D5B4F9A23007EE86
:102BD000903AF8EEE77A88EE277A84ED2B7AD4EDF6
:102BE0002B0A31F06DFA70BB58F082FF40F27D1273
:102BF0004FF4801158F034FF56F03CFC56F0A4F826
:102C000095F8CC31B0EE408A23B1D5F8EC000368DA
:102C10001B6F984704F53E50B0EE480A143079F027
:102C2000CDF804F54350B0EE480A303079F0C6F8DC
:102C3000B0EE480ABDEC028B04F548502430BDE8E4
:102C4000704079F0BBB8D4ED2B7A94ED460AF0EEE3
:102C5000E77AF4EEE87AF1EE10FA09D5B4F9A23089
:102C600007EE903AF8EEE77A88EE277A84ED2B7A31
:102C7000D4ED2B0A31F024FA0028B5D0BCE700BF10
:102C8000942300205D90002000000034FFF714BF63
:102C900070B500F5A046044696F98C3F002B28DD60
:102CA00007F0CEFE28BB04F5C0457035284682F0FB
:102CB00009F9F0B1284681F087F8D0B193F036F9E0
:102CC000D6F80035C01A96F98C3F4FF47A72534308
:102CD00098420ED301221C212846FEF759FF40B12D
:102CE00004F54F50034ABDE87040062128305DF0DE
:102CF0005DBE70BD90400D0800B52DED028B9FEDBF
:102D00000B8AD0ED4E7A67EE887A83B0C0ED4E7AAA
:102D10003830019079F0B0F8019820EE080A03B03D
:102D2000BDEC028B5DF804EB79F0BEB952B87E3F82
:102D300000B52DED028B9FED0B8AD0ED4F7A67EE3B
:102D4000887A83B0C0ED4F7A3C30019079F094F8E6
:102D5000019820EE080A03B0BDEC028B5DF804EB8D
:102D600079F0A2B952B87E3F30B52DED048B83B017
:102D7000044601A900F596501AF0FEFB002800F069
:102D8000B98004F5A94595ED1A7ADDED017AB4EE26
:102D9000E77AF1EE10FA05F1680507D504F5C040B1
:102DA000703081F01BF808B1019B2B6004F50055D1
:102DB00095ED7F7AB5F9A831DFED606A052BB8BFD4
:102DC000052307EE903AB5F9AA31F8EEE78A07EE47
:102DD000903AF8EEE77AB6EE009A77EEA77A1820E6
:102DE000C7EE270ADFED567A68EEA77AF4EE490AB5
:102DF00087EE271AF0EE007AF1EE10FAB4EE671AB9
:102E0000C8BFF0EE490AF1EE10FA48BFB0EE671AFB
:102E1000DDED017AF4EEE67AF1EE10FACCBF87EE42
:102E2000270AB0EE410A31F05DFA04F5C1403830AE
:102E3000B0EE408A0FF0F6FA38B904F5C04393F8C3
:102E4000CC21D2B393F8F931BBB304F5C040703054
:102E500080F0C4FF88B328EE892A9DED011AB4EEF4
:102E6000C21AF1EE10FA28D5D5ED7F0ADFED351A3A
:102E70009FED350AC0EE820A31F066F904F53D5047
:102E80001C30B4EE408AF0EE408AF1EE10FA48BFF2
:102E9000F0EE488AFFF730FF04F54250343004F575
:102EA0004054FFF745FFD4EDD97A9FED287A67EEBD
:102EB000877AB0EE688AC4EDD97A254819F00AFB02
:102EC00090B924484021FFF7C9FD68B1224BD3F8DF
:102ED0005C35012B08D1F7EE007AB4EEE78AF1EE0B
:102EE00010FA58BFB0EE678AB0EE480A03B0BDECE6
:102EF000048B30BD04F5C040703080F06FFFB7EE3A
:102F0000008A0028D9D0462067F09CF9B4EEC80AA0
:102F1000DFED127AF1EE10FAD8BFB0EE480A87EE74
:102F2000800ABAF0C5FB2F209FED0D1ADFED0D0AC8
:102F300031F0D8F9B0EE408ABFE700BF17B7D138FB
:102F40003333333F000000006F12833A52B87E3FA4
:102F5000503E0020902B0020907B00200000344247
:102F60008FC2D53F9A99193FF8B5044665F046FEE1
:102F70000368DB689847054610B900252846F8BD68
:102F800004F58046204607F0D9FBD6F8202F04F53B
:102F90009B4330339A42074605D104F5C04393F86A
:102FA0008C32022BE9D804F5C14038300FF060FCB8
:102FB0000028E2D1D6F8200F03689B6B984758B9D8
:102FC00096F8343F002BD9D004F5005494F91452EC
:102FD000023D18BF0125D1E7084BD3F8200F036845
:102FE0005B6B98470028EBD004F5005494F95132FC
:102FF000002BC2D0032BC0D03D46BFE7906B002012
:1030000070B52DED028B044600F5804600F5C140F9
:1030100006F5776382B0383093ED008A0FF03CFB01
:1030200004F53D551C35002846D104F5C046D6F8B8
:10303000EC0003689B689847D6F87C335B0225D583
:10304000D6F8EC3093ED437AD3ED097A67EE877AC0
:103050009FED327AF4EEC77AF1EE10FA16DB04F542
:10306000005404F5766393ED007A67EE877AF7EE05
:10307000006A86EEA77A04F65C74B4EE667AF1EE26
:1030800010FAC8BFB0EE667A84ED497ADFED247A93
:1030900090ED250AF0EE480A20EE270A284682F035
:1030A000B5FD28468DED010AFFF726FE9DED010ACC
:1030B00002B0BDEC028B70BDD6F8202F04F597430B
:1030C00010339A4228D104F50053D3F8283CB3F9C1
:1030D0000860003E18BF012604F5A04204F58054A4
:1030E000D2F87035D4F8B8441C1B92F86C353BB15B
:1030F0000C484FF40061FFF7B1FC80F00100C3B24F
:103100003246B0EE480A2146284602B0BDEC028B9A
:10311000BDE8704082F07EBD0026DDE7000000348F
:10312000E02E6542902B002010B5044606F0CEFE3E
:1031300098B104F5A042D2F8703503F58C415031B6
:10314000C2F8701504F58051D1F8B8140029BEBF3B
:10315000A3F58C43503BC2F870352046FFF750FF73
:10316000BDE81040042067F059B800002DE9F04791
:1031700000F5C1442DED048B00F580493834054637
:1031800009F577632046D3ED008A0FF085FA05F53F
:1031900042563436002844D105F5C044D4F8EC003A
:1031A0000368DB689847D4F87C335B0221D5D4F8F8
:1031B000EC3093ED447AD3ED0B7A67EE877A9FED8E
:1031C000537AF4EEC77AF1EE10FA12DB05F54055AA
:1031D00095ED2E7A67EE877AF7EE006A86EEA77A8B
:1031E000B4EE667AF1EE10FAC8BFB0EE667A85EDFD
:1031F000777A90ED250ADFED467AF0EE680A20EE48
:10320000270A304682F05CF93046B0EE408AFFF77C
:103210008FFDBDEEC80ABDEC048BB8EEC00ABDE858
:10322000F087204605F500580DF0A6FD9FED399A70
:1032300098ED918A28EE098A05F5A047BDEEC88A67
:10324000D7F8743518EE102A1A4408EE102A824670
:10325000462066F0F7FFB8EEC88AD8ED7B7AD9F839
:10326000200FA0EE278A05F5974310339842FDEE14
:10327000C87A17EE904A45D1D8F82C3CB3F90880AB
:10328000B8F1000818BF4FF00108BAF1000F1ED1C5
:1032900003685B699847D0B9D9F8200F03689B6B26
:1032A0009847A0B905F5C043D3F81434022B0ED1CA
:1032B000284612F0DBF950B107F66C73D3ED007AB3
:1032C00067EE897AFDEEE77A17EE903A1CB205F5C3
:1032D0008055D5F8BC34E41A97F86C353BB10E48EC
:1032E0004FF40061FFF7BAFB80F00100C3B2B0EE0B
:1032F000680ABDEC048B424621463046BDE8F047E3
:1033000082F0C4B94FF00008BFE700BF00000034EE
:10331000E02E65420000C842902B002010B5044604
:1033200015F08AFF68B100B200EB4000C0EB00135B
:1033300000EE103AB8EEC00ABDE81040132066F067
:103340006DBF2046FFF712FFF6E7000010B51048EA
:10335000FFF70AFED0B10F480FF0C4FBB0B10E4C1E
:10336000042066F06FFFD4F8280C65F0B7FE042047
:1033700066F054FF132066F065FFD4F82C0C65F05E
:10338000ADFEBDE81040132066F048BF10BD00BF81
:10339000902B0020488C0020904B0020F8B52DED9C
:1033A000028B0446FFF7E0FD002800F0AB8004F537
:1033B000804704F59742D7F8203F4832934200F007
:1033C000A18004F598420432934200F09B8004F5FA
:1033D00098426432934200F0958004F5984220327E
:1033E000934200F08F8004F598423C32934200F003
:1033F000898004F59A423C32934200F0838004F5C0
:103400009A42583293427DD004F59A4274329342E4
:1034100078D004F59B421432934273D004F59B425A
:10342000503293426ED004F5C14038300FF05AFB51
:10343000002867D0D7F8202F04F597432C339A4201
:1034400060D004F50055F6EE008AD5F8280C65F03A
:1034500005FDB4EEE80AF1EE10FA40DDB0EE087AB0
:10346000FFEE007AE0EE077AB0EE670AD5F8402C5E
:1034700004F5A04607EE902AD6F87035B8EEE77A44
:1034800007EE903AF8EEE77A5142E7EE007AFDEE69
:10349000E77A17EE900AC6F8700530F0C3FFC6F859
:1034A0007005D7F8202F04F5994348339A4222D06B
:1034B000D5F82C0C65F0D2FCB4EEE80AF1EE10FA67
:1034C000B0EE408A21DCFEEE007AB4EEE70AF1EEBF
:1034D00010FA22D5B0EE087AF7EE007A19E0FEEE87
:1034E000007AB4EEE70AF1EE10FABFD5B0EE087A32
:1034F000F7EE007AB6E725484FF48051FFF7AEFAB1
:103500000028D5D0BDEC028BF8BDB0EE087AFFEEF6
:10351000007AE8EE077AB0EE678A204606F0D6FC1D
:1035200008B1B1EE488AD6F87435D5ED706A9FEDD2
:10353000186A05F6444595ED007AB5EEC08A07EEA7
:10354000903AF1EE10FACCBF28EE268A27EE488A90
:10355000F8EEE77A66EE866AE8EE067A27EE067AF5
:10356000FDEEE77AFDEEE66A17EE903ABDEEC77A19
:1035700016EE902A17EE101A17EE900AC6F8743558
:1035800030F050FFC6F87405BCE700BF902B002058
:103590000000C842F8B5044604F5C04792F0C6FCE6
:1035A00097F8CC31064653B1D7F8F401036804F517
:1035B000AA4204F5AA411B6A70327431984704F597
:1035C0008045D5F8303FF31AB3F5FA6F03D9D5F833
:1035D000200F07F08DFF2C4BC5F8306FD3F8200F6C
:1035E0000268136898470021204612F0F5F9DFEDD4
:1035F000277AB0EEC00AB4EEE70AF1EE10FA42D52F
:10360000D7ED087AB1EE047AF0EEE77AF4EEC77AF5
:10361000F1EE10FA37D504F586601CF0E3FBF6EE08
:10362000007AB0EEC00AB4EEE70AF1EE10FA2AD53D
:1036300004F5B65595ED017AF0EE087AB4EEE77A26
:10364000F1EE10FA05F104051DD504F53D501C30CE
:1036500082F050FB04F54250343082F0C7F804F594
:1036600048500C3082F0F4FF95ED007AF7EE007AC6
:10367000B4EEE77AF1EE10FA05D504F54E50BDE848
:10368000F84082F03BBDF8BD906B00200000003494
:1036900000F5005090F99F31012BC3BF00F6D840D0
:1036A00090ED290ADFED047A9FED040AC8BF20EEF1
:1036B000270A462066F0B2BD0000C84200000000A4
:1036C0002DE9F8432DED028B00F5804909F577636C
:1036D000D3ED008A054611F0CDFD8046D9F8200FC4
:1036E00003681B6A984705F548560C3698B14F4C4D
:1036F000D4F83C35002B0EDD92F018FCD4F83C35A4
:10370000C01A40F6B733984205D8B4F93045304670
:1037100082F0AAFF7AE005F5C04305F5005793F85B
:10372000093443B1B7F93032002B04DD05F54053BD
:1037300093F9223203BBD9F8203F05F597451035A0
:10374000AB426DD00021B0EE680A304682F024FD15
:103750000546042066F076FD2BB207EE903A97ED11
:10376000797AF8EEE77AE0EE077AFDEEE77A17EE7F
:10377000904A444424B2CAE72846012111F06CFF64
:103780009FED2B7AB7F93032C0EE077A05F5A045E8
:1037900005F27C5508EE103A55F80C3C9FED250AD1
:1037A000B8EEC88A28EE278A07EE903AF8EEE77A54
:1037B00067EE807A9FED200A27EE800AB9F09CFD23
:1037C000B7F9A831DFED1D7A95ED007A20EE270AD2
:1037D00007EE903AF8EEE77A0021B4EEE77AF1EEE0
:1037E00010FA58BFF0EE477A80EE277A3046DFEDC8
:1037F000147AB0EE480AA7EE270AF0EE680A82F0C3
:1038000027FEBDEEC00A10EE103A1CB2BDEC028BD2
:1038100020460C49BDE8F84341F2941230F012BE44
:10382000B8F1000118BF01218DE700BF907B002097
:1038300000A08C450AD7233C35FA8E3C0AE81C418F
:10384000E02E65426CEEFFFF38B500F540530546AB
:10385000D3F804060368DB689847014605F54E5027
:1038600082F02EFC04B22846FFF77EFB70B107EE13
:10387000904A05F50055B8EEE70AD5F8340C65F026
:103880002DFCBDEEC00A10EE103A1CB220460349D2
:10389000BDE8384041F2941230F0D4BD6CEEFFFF29
:1038A00038B590F8E433B02202FB030393ED777A46
:1038B000F7EE007AB4EEE77AF1EE10FA054600F57D
:1038C000A0441DD5002112F087F8DFED417AB0EE5B
:1038D000C00AB4EEE70AF1EE10FA11D5D4F85C355F
:1038E000012B0DD0072B0BD0002384F8D43404F522
:1038F0009B64002323602846BDE8384011F0BABC21
:1039000092F014FBD4F8DC34C4F8DC04C31AB3F529
:103910007A7F84BF002384F8D434284611F0AAFCAF
:10392000D4F85C35012B07EE100A2CD0072B2AD0D7
:10393000B8EEC77ADFED276AC7EE267A05F50052A2
:10394000B2F9F42100EE102AB8EEC00A27EE800A80
:10395000DFED1F7AB0EEC07AB4EEE77AF1EE10FA3E
:1039600013D4002384F8D43494F8D43405F54E509D
:10397000DBB982F08DFABDE83840174900B241F258
:10398000941230F05FBD9FED150A94F8D424002AFC
:10399000EAD10122934284F8D424E5D0072B1EBF3C
:1039A00004F59B6300221A60DEE704F59B6494ED46
:1039B000007ADFED0B7A67EEC77A9FED0A7A67EE41
:1039C000877AFDEEE77A17EE901A82F079FBD2E75C
:1039D0000000003400A08C456CEEFFFF00000000EA
:1039E000E02E65420000C84270B52DED028B00F557
:1039F000BE46143682B0044630468EF03FFB054684
:103A0000D8B904F50053D3F8282CB2F9082072B9BC
:103A100004F5C042D2ED087A93ED7C7AF0EEE77AB5
:103A2000F4EEC77AF1EE10FA4CBF012500253046BE
:103A30008EF038FB002808BF002530468EF01EFBB4
:103A400050BB04F5A043D3F8D03401331ED01DBBC6
:103A50009FED1C8A2046FFF733FE07EE900AB8EE72
:103A6000E70A8DED010AFDB9152066F0D7FB9DED43
:103A7000010A1A2066F0D2FB04F5C240403002B0C1
:103A8000BDEC028BBDE8704003F028BB002DDFD0F9
:103A90002046FFF705FF02E02046FFF7D5FE07EEC0
:103AA000900AB8EEE78AD5E71A2066F063FE9DED2E
:103AB000010A08B9B0EE480A152066F0AFFBB0EE77
:103AC000480AD6E70000000010B500F5005303F6E1
:103AD0004442D3ED706ADFED127A92ED007A9FEDE9
:103AE000116A03F6D84366EEA76A27EE277AD3ED6C
:103AF0002A7A67EE867AFDEEE66ABDEEC77AFDEEBB
:103B0000E77A044616EE902A17EE101A17EE900A7E
:103B100030F088FC04F5A044C4F8740510BD00BF63
:103B20000000C842A00CB34510B5044613F03AFD9E
:103B3000031E2ADB04F5005191F99F219A4224DDEE
:103B400004F5A040D0F85C45022C1ED0D1ED7E7A61
:103B5000DFED0E6AD31A66EEE76A07EE102A07EE6B
:103B6000903AB8EEC77AF8EEE77AD0F8743587EE77
:103B7000876A07EE903AF8EEE77AE6EE867AFDEE8F
:103B8000E77A17EE903AC0F8743510BD0000C842CD
:103B900070B52DED028B00F5A0459FED550AD5F8C7
:103BA00070359FED547A07EE903AF8EEE77A0446C6
:103BB00067EE807A9FED500AF0EEE76AF4EE476A0E
:103BC000F1EE10FAC8BFF0EE477A27EE800AB9F09E
:103BD00003FA30F0A9FAB7EE008AC8EE007A05F5CC
:103BE000AF6304F50056C3ED007A04F5C04393F8C3
:103BF000CC219AB1D3F8F401036804F531515B6A22
:103C0000984758B1D6F8402CD5F87005514230F09D
:103C100009FCC5F87005BDEC028B70BD96F9D0317A
:103C2000002BF8D0204606F051F90028F3D104F516
:103C3000C540703013F0B4FE0028ECD1B6F9A831BD
:103C4000012BB8BF012307EE903A05F27C52F8EE43
:103C5000E77AD2ED006A86EEA77AB4EEC87AF1EE82
:103C600010FA13D840F6C4122449D5F8700530F084
:103C7000D9FBC5F87005D6F8402C40F6C4139A421B
:103C8000D4BFC6F8402CC6F8403CC4E705F5AF6386
:103C9000D3ED007AF4EEC77AF1EE10FABBDD88EED0
:103CA000070A20EE000AB9F051FBDFED157AD5F8CE
:103CB000700520EE270ADFED137A20EE270A40F682
:103CC000C413FDEEC07A17EE904A9C42B8BF1C4662
:103CD0002246614230F0A6FBC5F87005D6F8403C9C
:103CE000A342D4BFC6F8403CC6F8404C93E700BF9F
:103CF0000AD7233C0000AA4235FA8E3C3CF6FFFF6F
:103D0000E02E65420000C84210B500F5405304465D
:103D1000D3F8040603681B68984704F50053D3F8EA
:103D2000402C514230F07EFB04F5A043C3F87005EF
:103D30002046BDE81040FFF72BBF00007047000091
:103D4000012070470820704701207047014B93F80D
:103D5000DC017047904B0020034B93F9E4090038D5
:103D600018BF0120704700BF904B0020014B93F912
:103D7000DE017047904B002013B5064BD3F8200F9F
:103D80004B690468009308310EC9646CA04702B007
:103D900010BD00BF906B002070470000704700000E
:103DA00038B5264DD5F8200F03685B689847192869
:103DB0003CD8DFE800F00D39370D0D373737373B8A
:103DC0003939393939393B37373737393B0D393993
:103DD00040241B4B93F8E12312B193F8E0330BB965
:103DE00044F01004174BD5F8202F9A42A3F11C037E
:103DF00003D09A4218BF44F01004134991F95102BC
:103E0000B0B19A4216D0032803D101F532518A424B
:103E100001D144F040040D487FF0D6FF50B144F08A
:103E2000800407E01024D4E71824D2E70124D0E767
:103E30009A42F0D144F0010038BD00BF906B0020E1
:103E4000905B0020B0780020904B0020008C002078
:103E500008B5044806F0F4FD00280CBF012002203C
:103E600008BD00BF902B0020F0B52DED028B8BB06C
:103E7000054619F0B1FD4FF48071D0F8047290ED51
:103E8000828AD0F80C6204461948FEF7E7FD30B983
:103E9000184BDFED197A93ED917AA7EE678A1748F0
:103EA0000DF09EF830B1164BD3F86C335F6893ED8C
:103EB000028ADE682D7C92F039F8D4F81823D4F801
:103EC0001C33D4F814130892099327221C23CDE93C
:103ED00000320390079103AA1E21284604978DED16
:103EE000058A06965DF080FD0BB0BDEC028BF0BD3F
:103EF000902B0020904B002035FA8E3C488C0020FF
:103F0000908B002038B5C5780B46352D044628BF68
:103F10003525352200211846BBF07AFC2A4604F1EB
:103F20000C01BDE83840BBF029BC000008B50248D0
:103F300013F038FB00B208BD902B002037B50D46BA
:103F4000134840F2EF2204F087F82C7814F00404B0
:103F50000AD0696803220F481FF0C0F90C4803B06B
:103F6000BDE8304003F0D8B901AA214628461FF029
:103F700089FA0028F2D0DDED017A9FED077A67EE2D
:103F8000877A2246FDEEE77A17EE901AE3E700BF44
:103F9000902B0020848B00200000C84210B5054CF7
:103FA000012384F8E3335FF0A1F9002384F8E333BD
:103FB00010BD00BF905B002062F0F2BA2DE9F04125
:103FC0002DED028B4FF0000882B0CDE900281E4F86
:103FD0009FED1E8A0C461546B0EE480AB1F9022044
:103FE000D7F8281C4FF47A73064662F0B3FD01231C
:103FF000CDE90053B4F90020D7F82C1CB0EE480AE4
:1040000030464FF47A7362F0A5FDB4F90420D7F876
:10401000301C9FED0F0A43463046CDE9005862F050
:1040200099FDCDE90058B4F90620D7F8341CB0EE5C
:10403000480A4FF47A73304662F08CFD02B0BDEC52
:10404000028BBDE8F08100BF904B00200000FA44D5
:1040500000007A4410B5074B93F9782640F24D34AE
:1040600040F24D13002A08BF1C465EF037FF204384
:1040700010BD00BF907B002010B504461FF062FD0C
:10408000204610BD10B50B4C002384F813355FF0AB
:1040900027FE54F8E02CA4F560739A4208D194F8F6
:1040A00084352BB904F5B060BDE8104036F0B8BDDA
:1040B00010BD00BF907B002013B5124C94F8361051
:1040C000A4F58C7016F0C6FF78B194F83610A4F5FC
:1040D0008C7017F02DFA40B194F83610A4F58C705E
:1040E00002B0BDE8104017F065BA19F075FC01A9DF
:1040F00019F042FA18B19DED010A02B010BD9FED12
:10410000020AFAE7904B002000000000044B93F8ED
:10411000CC0120B1D3F8F40103681B6B184770473A
:10412000908B002008B5084BD3F8D02B002A03DC75
:10413000BDE808405EF016BF03F52F605BF0A4FFFA
:1041400090ED000A08BD00BF904B002008B5124852
:10415000D0F8202F00F604539A4216D0B0F9383F19
:10416000ABB900F5805393F89D2482B990F8352FB0
:104170006AB993F8493563B9A0F5804006F060FC50
:1041800000280CBF0320042008BD0220FCE7052006
:10419000FAE70620F8E700BF906B002010B5224B2D
:1041A00003F55262D3F8203F934290B0044639D0D1
:1041B00000231E4802931FF07BF8014618B91B48E4
:1041C00002AA1FF0C1F8247C91F0B0FE184BDDED7F
:1041D000027AD3F8FC2F9FED177A03F58053F8EE9F
:1041E000E77A1B68059300230793089309930A93C2
:1041F0000B930C930D930E934FF6F853ADF83C30A0
:104200000023CDE9030267EE877A96228DF83E30CF
:104210003323CDE90032572103AA2046CDED067A9B
:104220005DF0E2FB10B010BD906B0020848B00208D
:10423000907B00200AD7233CF0B58DB0044691F066
:1042400075FE184AD2F8F031C31A642B28D8D2F878
:10425000EC300290D3F88C10D3F89020D3F884601F
:10426000D3F88850D3F8DC70D3F894E0D3F898C032
:10427000D3F89C30099300238DF82C300692252327
:104280001622CDE900320591207CCDF81CE002AA6F
:104290005321CDF820C00A97039604955DF0A4FB46
:1042A0000DB0F0BD908B002010B55FF061F80446B2
:1042B00078B9094850F8E02C80F81345A0F56073F0
:1042C0009A4206D190F884351BB900F5B06036F0FB
:1042D000A7FC204610BD00BF907B00202DE9F047D1
:1042E0002DED088B8B4CD4F8202F04F552639A42A5
:1042F00090B0054600F0E7808748DFED888ADFED63
:10430000889A9FED889A0CF06BFE002867D082484F
:104310000CF004FD002862D004F500589FED820ADD
:10432000D8F8EC006C3033F0E1F808F1C400B0EEDE
:1043300060AAB0EE418ACDED070A8DED081AF0EEC5
:1043400040AA8DED060A84F0DDFED8F8F030014673
:10435000D3F85C23D3F85833059204A8049332F0C1
:10436000C5FE09A88DED090AB0EE680ACDED0A0A6E
:1043700032F0CCFE28EE288A02A8BDEEC88A95F855
:104380001090CDED030A18EE103A8DED020A1EB220
:1043900032F030FFDFED657A20EE270A02A8BDEE8D
:1043A000C00A6AEEA8AA10EE103A1FB232F06CFFF3
:1043B000B4EEE90AF1EE10FA58BFB0EE690ABCEEAD
:1043C000C00AD4F8202F10EE103A9DB204F63C53E8
:1043D0009A422AEE28AA7BD1DFED558A7EE0DFF8EB
:1043E00054A195F81090DAF804760AF5005838468A
:1043F000D8F8703507EE903AD8F87435B8EEE7BAC9
:1044000007EE903A3B689B68F8EEE7AA984707EEFC
:10441000900AF8EEE77A384667EEA87A08F59F68C2
:10442000FDEEE77A04F65C7417EE903A1EB23B6834
:104430001B69984707EE900AF8EEE77A98ED00AA14
:1044400067EEA87AB4EEE9AAFDEEE77AF1EE10FA8B
:1044500017EE903ADFED327AAAF5405058BFB0EE31
:1044600067AA1DB203F03EF83B68D4ED007A5B69A1
:1044700008EE100A384627EE899A9847B8EEC88A9F
:10448000BCEECAAA2BEE28BA6AEEA8AA1AEE103A17
:1044900068EE288A8DED09BACDED0AAACDED0B8A1A
:1044A0008DED0C9A8DED0D0AADF83860ADF83A50EF
:1044B000ADF83C30B7221A23CDE900323E2109AADB
:1044C00048465DF091FA10B0BDEC088BBDE8F0876E
:1044D000D8F8F030D3ED0F7A67EEA88AD8F8F43028
:1044E00004F65C74D4ED007A186927EE899A89F095
:1044F000DBFDCDED09AA8DED0AAACDED0B8A8DED80
:104500000C9A8DED0D0AADF83860ADF83A70ADF843
:104510003C50CFE7906B0020488C00200AD7233C0A
:1045200000FF7F470000C8429F0CB345E02E654264
:1045300000000000905B002001480CF001BC00BFAF
:10454000488C002008B5034BD3F8200F03685B6844
:10455000984708BD906B002030B587B0054619F02C
:104560003BFA04462D7C91F0D9FCD4F88422D4F88F
:1045700088320492059300211023CD22CDE9003228
:104580000290039102AA42F60C3128465DF02CFA03
:1045900007B030BD30B52DED028B89B0054619F05E
:1045A0001BFA00F55A7393E8070002AC84E8070091
:1045B000DDED020A9DED030A2D7CF1EE600AB1EEFD
:1045C000400AB8F02BFF2046B0EE408A33F012FCD0
:1045D000DFED0B7A049B079328EE278A0C23012238
:1045E000CDE90032A82105AA28468DED058A8DED7A
:1045F000060A5DF0F9F909B0BDEC028B30BD00BFD1
:10460000E02E6542282938B5054623D007D824294D
:104610002BD0272911D01B2908D1012413E04329CD
:1046200037D008D84029F8D0422928D02846BDE8FC
:10463000384062F0C1BD5329EEE712215CF0D2FB95
:10464000044610B90024204638BD297C134855F093
:10465000B1FAF8E716215CF0C5FB04460028F1D05A
:10466000297C0E4855F080FBEDE70C215CF0BAFB8D
:1046700004460028E6D02846FFF78CFFE3E7102128
:104680005CF0B0FB04460028DCD02846FFF764FF4E
:10469000D9E7017C02488DF0EFFCBEE708820020DC
:1046A000A48A0020F0B52DED028B05468DB016468C
:1046B000B0EE408A0C46002930D0007C5DF02AF92B
:1046C0000746287C5EF02AF800F121039F4207D2BA
:1046D000287C0DB0BDEC028BBDE8F0405CF070BBF7
:1046E00063690893636A2269CDF82530236AA0695B
:1046F000E1680792CDF829306222212327680590CE
:10470000CDE900320691287C0397192303AAC22120
:104710008DED048A8DF824605DF066F90DB0BDEC76
:10472000028BF0BDF8B54B4CD4F8202F04F5526342
:104730009A42054600F08C80A4F50056B6F8823205
:10474000DF0713D544480DF06DFE002879D004F53D
:104750000054D4F8EC0003689B68984700F194017A
:1047600091ED010A01222846FFF79CFFB6F882323C
:104770009C0712D538480DF055FE002864D0374B01
:10478000D3F8EC000368DB68984700F1940191EDE1
:10479000010A02222846FFF785FFB6F88232580741
:1047A00012D52D480DF03EFE00284FD02B4BD3F8EC
:1047B000EC0003681B69984700F1940191ED010A30
:1047C00003222846FFF76EFFB6F88232190708D594
:1047D0002349052291EDED0A284601F56C71FFF79A
:1047E00061FFB6F88232DA0616D51E4FD7F85C356F
:1047F000042B11D119F0F0F8044607F614708DF06F
:104800006BFC94EDC70ADFED187A014620EE270A0B
:1048100006222846FFF746FFB6F882329B0617D5D8
:104820000D480DF0FFFD98B10C4BD3F8F010284661
:1048300091EDAB0ABDE8F840042201F52A71FFF7BB
:1048400031BFA4F67C718BE70849A0E70849B5E7BA
:10485000F8BD00BF906B0020488C0020908B00209A
:10486000905B0020907B0020E02E6542705D002070
:10487000E45E002070B504460E4628F0A3FA90F8D6
:10488000C412B02303FB0101AC31204603F052FDFA
:104890000546C0B13EB119F09FF890F87C3243F064
:1048A000020380F87C3204F58043D3F8200F04F52E
:1048B00099432C33984204D004F59B443034A042F1
:1048C00001D106F039FD284670BD000073B51646CB
:1048D0000191044619F080F8019918F095FC0546FD
:1048E000C0B13EB119F078F890F87C3243F0020381
:1048F00080F87C3204F58043D3F8200F04F5994307
:104900002C33984204D004F59B443034A04201D1AA
:1049100006F012FD284602B070BD000030B5054615
:1049200085B00C46D1E9040130F0D6FD40B16846AF
:104930001EF0CEFC6A462146284662F07BF808B994
:10494000022067E0344840F24F32694603F084FBAE
:10495000D4ED037AF4EE677AF1EE10FA22D69FEDE9
:104960002F7AF0EEE77AF4EEC77AF1EE10FA54BF40
:10497000012200229DF80030294962F34103684674
:104980008DF800301EF00EFE0028D9D1254869466A
:104990006EF01AF940B958F0BDFE0522162158F004
:1049A00071FCCDE70022E5E7D4ED017AFDEEE77A70
:1049B00017EE903ADB0706D41B4B03F6E442D3F81C
:1049C000203F934225D119491348022212F0F8FBE7
:1049D0009DF8001011F0040102D168461EF042FD5E
:1049E0000D48694603F0F2FB94ED020AB4EE400A6A
:1049F000F1EE10FA0BD6B5EEC00AF1EE10FA06DDB4
:104A00009DF800100948C1F3400107F085FE002021
:104A100000E0042005B030BD902B002000000034E1
:104A2000748B0020304C0020906B002074780020A4
:104A300010B52DED028BD1ED017A91ED008AFCEEDF
:104A4000E77A8AB0CDED037A9DF80C1005AA0446EA
:104A500061F0DAFFC8B1DFED0E7A059B009368EED6
:104A6000277A0022FDEEE77A114617EE903A06A863
:104A70001EF04EFC23682046D3F8C43006A99847A0
:104A800000200AB0BDEC028B10BD0220F9E700BF88
:104A90000000C84237B5124DD5F8200F03681B6AD5
:104AA0000C46984740B9D5F8202F05F548639A423F
:104AB00002D0042003B030BDD4ED007AD4ED020A58
:104AC00094ED010A0748FCEEE77ACDED017A9DF8F6
:104AD000041004F0DDF80028EBD00020EAE700BF66
:104AE000906B0020902B0020134610B524220C461A
:104AF00018460021BAF08CFEA27F8277E27FC2774F
:104B0000072280F82020A28B8283D4ED067AF1EE72
:104B1000677AC0ED067A10BD10B48C8B162C03D1C9
:104B20005DF8044BFFF7E0BF5DF8044B61F0AAB9F4
:104B300008B591F82030072B0DD1094890F8CC31F9
:104B40003BB191ED060AB830B1EE400A0DF030FAF3
:104B500018B9042008BD0220FCE70020FAE700BFD6
:104B6000908B002008B5D1ED007A9FED087A0848B7
:104B7000F0EEE77AF4EEC77AF1EE10FA54BF0121B5
:104B8000002105F09DF9002008BD00BF00000034A1
:104B9000902B00201FB5D1ED017AFCEEE77A0B4691
:104BA000CDED027AD1ED007A1A7C017C0192FCEE07
:104BB000E77A0B48CDED037AD3ED027AFCEEE77A83
:104BC00017EE902A92B2009293ED030A9DF80C2002
:104BD0009DF8083009F0D8FE05B05DF804FB00BF71
:104BE000488C002007B5D1ED007A0848FCEEE77A42
:104BF000CDED017A9DF804100BF0AAFC00280CBF43
:104C00000420002003B05DF804FB00BF488C0020A6
:104C100070B58B8BC02B05460C4633D8B12B0DD805
:104C2000142B00F0AA80162B53D0112B00F0A1807A
:104C300021462846BDE8704063F056B9B23B0E2BC2
:104C4000F6D801A151F823F0C14C0108314C0108FC
:104C5000314C0108314C0108314C0108314C01083C
:104C6000314C0108314C0108B74C0108314C0108A6
:104C7000EB4C0108274D0108314C0108DB4C0108C1
:104C8000AD4C0108B3F5967F58D007D8D12B1CD076
:104C9000D42BCDD1BDE87040FFF764BF40F6B836E5
:104CA000B342C5D1BDE87040FFF79CBF2146BDE8C7
:104CB0007040FFF733BE2146BDE87040FFF7B8BE35
:104CC0002146BDE87040FFF7E5BEBDE87040FFF744
:104CD00061BFBDE87040FFF72BBF94ED000A294883
:104CE000FDF7F4FBE8B100201CE0274C94F8513F9D
:104CF000BBB1264904F5AC5036F090F888B104F504
:104D00008053012283F8B92504F548610222A4F5F5
:104D1000804012F055FA0028E5D11D4B002283F89F
:104D2000B925042070BD184C94F8513F002BF8D0E1
:104D3000164904F5AC5035F0F5FFDFE7D1ED007A08
:104D40009FED147AF0EEE77AF4EEC77AF1EE10FAFE
:104D500016D5D1ED017AF0EEE77AF4EEC77AF1EEEE
:104D600010FA0DD50C490222A1F5994012F028FA4B
:104D7000B9E70A4902220348F8E709490222FAE79B
:104D80000220CFE7902B0020906B0020748B002036
:104D9000907B00200000003410780020587800201C
:104DA0003C78002070B5434B03F6E442D3F8203F33
:104DB00093428EB00C467BD1CD78272D28BF272576
:104DC0002722002104A8BAF023FD2A4604F10C0191
:104DD00004A8BAF0D3FC059B9DF836400093069BCF
:104DE0000193E443079B0293E4B2089B03938DF87D
:104DF000364091F09BF814F0810F04F087050646C9
:104E000001D1802D13D1684631F0DAFEDFED2A7A28
:104E10002A4B20EE270ADFED2A7AC3F8346520EE0C
:104E2000270ABDEEC00A10EE102AC3F8282514F098
:104E3000820F01D1802D13D1684631F0DBFEDFED0A
:104E40001E7A1E4B20EE270ADFED1D7AC3F8386567
:104E500020EE270ABDEEC00A10EE102AC3F82C255A
:104E600014F0840F01D1802D13D1684631F0D2FEA9
:104E7000DFED117A114B20EE270ADFED117AC3F82E
:104E80003C6520EE270ABDEEC00A10EE102AC3F8DA
:104E9000302563060CD5DDED0C7A9FED097A074BC2
:104EA00067EE877A03F5A862C2ED007AC3F844651D
:104EB0000EB070BD906B0020E02E6542907B00200C
:104EC0000000C84230B5214C91B0084602A9FFF756
:104ED00019F8D4F8202F04F6E4439A4233D19DF810
:104EE0003C30072B2FD104F58054DDED056AD4F852
:104EF000F83F9FED177A07EE903AF8EEE77AE6EE84
:104F0000C77AFDEEE77A17EE903AC4F8F83F62F000
:104F1000C9FBD4F8D02FD4F8F83F52689FED0D7A32
:104F20009B1A07EE903AF8EEE77A054667EE877A25
:104F300017EE900AFBF7E8FA074ACDE900010621CF
:104F400028465BF033FD11B030BD00BF906B0020F0
:104F50000000C8420AD7233C3C460D0810B51D4B43
:104F600003F6E442D3F8203F9342044696B0084645
:104F70000FD108A9FEF7C6FF9DF8541003AA2046DA
:104F800061F042FD38B962F08DFB134A04215BF0F9
:104F90000DFD16B010BDBDF8503023F004039BB2D8
:104FA000002BF6D0DDED0B7A9FED0C7A039B00937E
:104FB00067EE877A0022FDEEE77A114617EE903A07
:104FC00004A81EF0A5F9236804A9D3F8C43020462C
:104FD0009847DEE7906B002050460D080000C8425D
:104FE00030B48D7A4B7A43EA0523CD7A43EA054300
:104FF000562B04460A461BD008D8522B12D0542BED
:1050000013D02046114630BC61F006BE03F1807318
:10501000863B23F07F43012BF3D8017C064830BC4C
:1050200054F06ABF30BCFFF7BDBE30BCFFF74ABFCB
:1050300030BCFFF793BF00BF0882002000207047FC
:10504000C82070470120704700207047002070473B
:1050500090F890308B4286BF00EB8100D0F894002E
:105060000020704790F890308B4286BF00EB8100A3
:10507000D0F894000020704703207047014B93F84C
:10508000DA017047904B002070B504464C4810F090
:105090009DFC18B1236A43F400032362484810F0D2
:1050A00095FC88B1462065F0CDF8DFED467AB4EE88
:1050B000E70AF1EE10FA07D8636A43F4000363626B
:1050C000A36A43F40003A362236A43F4F843236210
:1050D0003D4BD3F8200F03685B68984701381828C8
:1050E00015D8DFE800F03B430D4543434343143BF1
:1050F0003B3B3B3B3B14434343433B14453B3B005F
:10510000324A92F8E0338BB392F8E1238AB3304B02
:1051100093F8103F012B3DD0022B44D02D4B1D683E
:10512000DDB12D4E284696F81A1C4EF0E5FDA0B1D3
:10513000236A43F48073236296F980321BB1636A59
:1051400043F48073636296F81A1C28464EF00CFEF6
:1051500018B1A36A43F48073A36270BDD4E9092334
:1051600042F4E04243F4E0436262A362012300E0C0
:105170000023616A41F480626262A26A42F4806044
:10518000A062002BC3D041F4406142F440626162EE
:10519000A262BCE7236A43F480032362636A43F498
:1051A00080036362BAE7236A43F480032362636A7D
:1051B00043F480036362A36A43F48003A362ADE710
:1051C000902B0020000000B4906B0020905B00202A
:1051D000907B002004910020904B002013B54FF4E9
:1051E0004470CDE900211EF0A5FC044628B1DDE99C
:1051F000002162F075FA024B2360204602B010BD18
:105200004C480D0800207047002070470020704770
:105210000020704700F508503C3070470048704748
:10522000886E0D0800F58040D0F8200F03685B6899
:105230001847000000F5804300F59940D3F8203F5F
:105240001B1A584258417047A22070472DE9F0417F
:1052500000F5A04303F2745353F8042CDFED666AA3
:1052600007EE902AB8EEE77AD3ED007AF8EEE77A07
:1052700000F5C14890B027EE267A67EEA67A08F1CD
:1052800038080446002340468DED017ACDED027AC0
:1052900003930BF0A5FE04F5C046002800F0A6809D
:1052A000D6F8EC3084330FCB0CAF87E80F0008AD95
:1052B00004AF87E80F0085E80F0001A9384603AB6B
:1052C00002AA31F0C1FC9FED4D0AD6F86C7301A81B
:1052D00032F00CF9294638468DED080ACDED090A61
:1052E0008DED0A1A16F072FC90F020FED6F8F0311F
:1052F000C01A632804F57C652DD8D6F8EC00036845
:105300009B689847042100F19402284657F0CEF894
:10531000D6F8EC000368DB689847052100F1940299
:10532000284657F0C3F8D6F8EC0003681B69984785
:10533000062100F19402284657F0B8F8D6F8F0207C
:10534000284602F52A72072157F0B0F804F5C54047
:10535000703013F08BFB40460DF064F890B1D6F836
:10536000F00088F07DFB68B1D6F8F0206E21903215
:10537000284657F09BF8D6F8F0206F21BC3228461B
:1053800057F094F804F5425204326921284657F048
:105390008DF804F5475220326A21284657F086F8E6
:1053A00004F5405393F9222232B9D3ED867AF5EE13
:1053B000C07AF1EE10FA06DD04F54D5214326B217D
:1053C000284657F073F804F54E54204680F09AFEB4
:1053D00028B104F130026D21284657F067F818F023
:1053E000FBFA18F00DF810B0BDE8F08101A904F542
:1053F000965016F0B3FA77E70AD7233CE02E6542C1
:1054000010B54FF48011044612F0C8F810B12046D0
:10541000FFF71CFF4FF48001204612F0BFF828B1BF
:105420002EF024FABDE810402CF0ACBB10BD0000FB
:1054300030B591B0002300F59655029302A90023E0
:1054400004460DF1070228468DF8073018F09AF847
:1054500003A9284617F08EF808B92E4B0393302283
:10546000002104A8BAF0D4F9A3238DF810309523B5
:105470008DF8113090F062FD04F5A042CDF81300D4
:10548000D2F87035ADF81B3004F58053D2F874258E
:10549000CDF817104620D3F8B814D3F8BC34ADF8C3
:1054A0001D10ADF81F20ADF8213064F0CBFE10EEDA
:1054B000103A1520CDF8233064F0C4FE10EE103AF7
:1054C000CDF8273004F533539FED137AD3ED2F7ABF
:1054D00067EE877A284617EE903ACDF82B30029B7C
:1054E000CDF82F309DF807308DF83330039B0D93A6
:1054F00018F04EFA04F580433022D3F8643F8DED66
:105500000E0A04A904F57C600F9357F00BF911B053
:1055100030BD00BF2292CA7F0000C84270B58EB075
:105520003522044600216846BAF072F9A3238DF8AB
:10553000003095238DF80130012304F5A0468DF845
:10554000023090F0FBFC04F5405506F59F63CDF862
:1055500003001B68D5F80406CDF80710CDF80B3012
:1055600003681B699847ADF80F00D5F80406036877
:105570009B689847ADF811001D4801F0B3FFADF8E6
:105580001300D5F8040603685B69984710EE103ADB
:10559000D5F80406CDF8153003689B69984710EEDE
:1055A000103ACDF8193004F5804303F65C713522CA
:1055B0000968CDF81D10D6F8FC1FCDF8211004F5B0
:1055C000C041D3F8543F0868CDF82500D1F81C1429
:1055D000D6F8F80FCDF82900CDF82D1004F57C6031
:1055E0006946CDF8313057F09DF80EB070BD00BF60
:1055F000902B002030B587B0162204460021684663
:10560000BAF006F9A3238DF8003095238DF8013008
:1056100002238DF8023090F091FC04F5A045CDF8FE
:1056200003002046CDF8071005F00AFA05F5AC6333
:105630008DF80B001B680393124B1B68D86A90F817
:105640009C308DF810300368DB69984795F8493530
:105650008DF812308DF811002EF008F92DF056FA61
:10566000D5F85C358DF813008DF81430162295F8B6
:105670004A358DF81530694604F57C6057F052F8CC
:1056800007B030BD8C2B002010B58AB0272204460D
:1056900000216846BAF0BCF8A3238DF800309523AA
:1056A0008DF8013009238DF8023090F047FCCDF8D9
:1056B00003000420CDF8071064F0C4FD10EE103A8A
:1056C0001320CDF80B3064F0BDFD10EE103A4620EB
:1056D000CDF80F3064F0B6FD10EE103A1520CDF87D
:1056E000133064F0AFFD10EE103A0320CDF8173000
:1056F00064F0B8FD10EE103A1A20CDF81B3064F0BB
:10570000A1FD10EE103ACDF81F3004F59E43703322
:1057100027221B68CDF82330694604F57C6057F0DA
:1057200001F80AB010BD000013B5044600F57C6016
:10573000019056F029FB019856F0C0FB04F5805308
:10574000019893F9D4300BB156F060FC204602B0BA
:10575000BDE81040FFF798BF7047000030B500F576
:10576000C04389B093F8CC21044600F57C6552B162
:10577000D3F8E4001E2269468AF0A2FA0F496A466D
:10578000284657F06BF904F58043D3F8200F0368DF
:105790005B68984704F50053014693F85C2128465E
:1057A00057F080F904F5965018F090FB04F59070CE
:1057B00009B0BDE8304026F06FBB00BF58490D0866
:1057C0009FED020A00224CF079BD00BF0AD7233CAE
:1057D000134B70B5044640F8043B63F08FF8114E4C
:1057E000114B63605425601963F03EFA6651303501
:1057F000B5F5557FF7D104F5557065F019F90B4AE9
:1058000004F5EC6002F63C318DF0C2FA012320462B
:10581000074984F891394CF061FF204670BD00BF04
:10582000D0370020A4990D08B8990D082C4D002000
:105830008C890D082DE9F04100F507519AB00D2231
:105840001831044655F08CFB0022C04827214CF04B
:10585000ADFC0421002065F075F81321012065F0EE
:1058600071F84621022065F06DF81521032065F0DE
:1058700069F864F037FE04F5C04393F9843123B12D
:105880009FEDB30AB3484DF0C9FA4DF02DF9B24A75
:10589000B24E138843F0040313804FF000080AAFA0
:1058A000002110223846B9F0B3FF01238DF83030C3
:1058B0003388ADF8283005A973680B9338464CF04F
:1058C0007DFBC8B19DF91430002B15DD63F096F90E
:1058D0009DF81410036801391B68C9B2984758B184
:1058E000051D28464CF0B4FA30B9B368ADF818304D
:1058F00006A928464DF0ACFD08F10608B8F1240FC2
:1059000006F10C06CCD1964800220DF10B014CF0AB
:1059100087F806AD064620B34CF09AFA08BB914BC7
:105920000FCB85E80F0004A928464CF047FB002860
:1059300040F03B814FF004088B4B0FCB87E80F0002
:1059400005A938464CF03AFB28B105A84CF080FA7E
:1059500008B148F0010803A930468DF80C804DF0DD
:1059600025FD824B0FCB85E80F0003A928464CF09C
:1059700025FB002846D00998002204A94CF050F8D5
:10598000064600283ED04CF063FA0546002839D17F
:105990009DF80C30013BDBB2032B96BF744A0346E3
:1059A000D35C8DF82830304639464DF0FFFC714805
:1059B000002205A94CF034F806466DF047FB78B19B
:1059C0006DF042FB90F8302090F8281090F84830A5
:1059D000114490F840200A44D34214BF0125002509
:1059E00086B130469DF90C804CF032FA50B91DB1A9
:1059F000B8F1000518BF0125394630468DF828500A
:105A00004DF0D4FC04F509500022B7EE000A012144
:105A100034304CF053FC04F508500022B7EE000A75
:105A2000022110304CF04AFC012304F5F751009399
:105A3000514A002308318E204CF0BCFB94F974C904
:105A4000BCF1000F1AD14D4E0FCE3D460FC50FCE03
:105A50000FC50FCE0FC596E80F0085E80F00624610
:105A6000042138464CF0A2FB9FED450A45484DF015
:105A7000D5F94548B7EE000A4DF0D0F9012504F5F7
:105A80000251424A00950023203140F205104CF0AB
:105A900091FB04F5095002210430FFF791FE04F553
:105AA000065003212C30FFF78BFE04F5065003212E
:105AB0003430FFF785FE032104F50950FFF780FE1F
:105AC00004F5095002210830FFF77AFE022104F59F
:105AD0000750FFF775FE04F5075002210430FFF769
:105AE0006FFE04F5065002213C30FFF769FE04F515
:105AF000BE4014308CF054FC254A1368D90705D4F5
:105B00002449156004F5015308330B6004F50A506D
:105B100020490122083001254CF09EFB1E4A0095C9
:105B2000002304F57C61FD204CF044FB1B4B1A68FC
:105B3000D20705D41A4A1D6004F58F540834146046
:105B4000174801214CF0A4FB2CE000BFD4860D08BF
:105B500000009643D8720E08E890002044890D0892
:105B600098860D083C3A0D084C3A0D085C3A0D0831
:105B7000D0860D08A3860D08C8CA0D086C3A0D081A
:105B800000000000B0860D08BF860D084CCB0E0843
:105B9000842B0020002200200C590E08882B0020A6
:105BA0000C2200201AB0BDE8F08104A84CF050F996
:105BB00000283FF4BFAE4FF00C08BDE67047000070
:105BC0000020704700207047002070470020704779
:105BD0000020704770470000002070470020704789
:105BE00084B001A880E80E0004B0002070470000D7
:105BF0000020704700207047704700001020704759
:105C000000487047A0950D0800487047B0950D08F2
:105C10000020704770470000012070470120704746
:105C200000207047002343608360C36003614361C9
:105C3000002303767047000010B50446FFF7F2FF1B
:105C40000023637610BD0000027E531CDBB2042BE0
:105C5000037600EB820288BF002382ED010A88BF31
:105C60000376704710B50446FFF7EEFFD4ED017AD6
:105C70009FED107A94ED020A637E77EE877A042B0B
:105C800077EE807A94ED030A94BF0133052377EE13
:105C9000807A94ED040A637677EE807A637E94EDE1
:105CA000050A77EE807A00EE103AB8EEC00A87EE69
:105CB000800A10BD0000000010B504461DF042FF30
:105CC000204610BD04F0DABB03F0F2B903F0BEBF0A
:105CD00003F0FAB901F006BF01F062BA01F0EABBC5
:105CE00001F02ABCFCF7D4BFFCF782BB70B51F4B98
:105CF000036000F540530446D3F898051C4AC3F8E6
:105D0000E82308B11DF022FF1A4B236004F58053ED
:105D100093F8842E42B9D3F8805E2DB128462AF03C
:105D2000B9FF28461DF00EFF04F58E500C307DF0B3
:105D300091FB04F58650143065F07AFF04F6C445F3
:105D400004F66446B54204D0183D28462AF0F8FB14
:105D5000F8E7094BC4F8983804F6941059F070FE2F
:105D600004F5106059F06CFE204670BD207D0D08D2
:105D7000EC730E08F0510E08D4180E0838B5474BD6
:105D8000044640F8043B66F099FA04F110001BF059
:105D900039F904F1680053F045F804F5907025F0E6
:105DA0005DFC04F5866019F0F3FF04F254501DF019
:105DB000CFFE04F698002CF009F804F5446066F074
:105DC0005BF804F551604DF0BDFE04F57C6056F0C3
:105DD000DDFB04F58650143065F012FF04F58850A1
:105DE00010301CF029FC04F58E500C307DF01EFBA9
:105DF00004F58F50083053F0D7FB04F591501C3058
:105E000067F03AFC04F5805304F5935200251046E0
:105E100083F86052224B10301A6049F0B1FC2946D9
:105E200004F5965016F088F804F5C850103076F056
:105E3000F9F904F5E85014307AF03EFB04F5F1501E
:105E40000C307CF04DFC04F5F45010307DF082F8FD
:105E500004F5F750083014F091FF04F501500830B4
:105E600076F03EFE04F5025020306CF0C5FB04F5E0
:105E7000005304F5055083F85C510A4D34307DF031
:105E8000A9FE2B6813B1084890F022F82046074974
:105E90004CF024FC2C60204638BD00BFF0510E08A9
:105EA000DC9900203C910020B8950D0818510E088F
:105EB0002DE9F04F2DED028B04469FB0FFF75EFFFA
:105EC000E24B236004F50A500830FFF781FC04F52B
:105ED0003050203004F500577FF0A0F904F5085346
:105EE0002233C7F8483C04F53150062387F84C3C70
:105EF000343065F097FA04F5BE431433C7F8F03C2C
:105F00000E934FF40063C7F8F43C5A2387F8743DAE
:105F100004F5065807F6D84308F11C08CC4AC7F820
:105F2000EC8C04F5965BC7F8E8BCC3F86021C94A5D
:105F3000C3F86421B7EE008AC74AC3F8682104F5A4
:105F40003A50C3F8CC2183ED578A34305AF098F890
:105F500004F5335A04F53B505AF092F80026BF4B33
:105F6000C7F8D03E0AF1180A87F8E86E0AF5FC7007
:105F7000FFF758FEBA4BBB49C7F8D03E87F8E96E29
:105F800050464CF0ABFBB84BC7F8F03E07F56F63DB
:105F90000022C7F8F4BEC7F8F8AE04F53B555A63C3
:105FA000DA6304F53D50012387F8343F303508307B
:105FB0001DF08EF987F8586FAC4928464CF08EFBDF
:105FC00004F53D5041461C307FF0DEFC04F54250A4
:105FD000414634307FF03CF904F54850414604F521
:105FE00040570C3080F09AF82C22314607F56C703F
:105FF000B9F00EFC04F54F569D4904F54E504CF097
:106000006DFB28369B4BC7F8E83306F108008EF08D
:10601000BDFE04F5505904F5515309F11409383304
:1060200048460F935EF020FE0F9B09F114094B4583
:10603000F6D10723C7F89C350023A7F8A0354FF405
:10604000CB701DF07DFDC7F8980504F5565024303F
:106050008EF09CFE04F5575028308EF097FE864B4C
:106060001A6802B91E60854BC7F8E83304F558502A
:106070004FF48051C7F8045608301BF0C5F804F5FA
:106080005A5008304DF09AFA04F55A501C306EF010
:1060900059FB04F5964004F58045743005F020F96D
:1060A000774BC5F8743B04F59740103005F018F9AC
:1060B000744BC5F8903B04F597402C3005F010F96F
:1060C000714BC5F8AC3B04F59740483005F008F932
:1060D0006E4BC5F8C83B05F53F63002204F59840B8
:1060E000DA609A605A6083ED008A043005F0F8F8AF
:1060F000674BC5F8043C04F59840203005F0F0F8F3
:10610000644BC5F8203C04F598403C3005F0E8F8B5
:10611000614BC5F83C3C04F59840643005F0E0F86C
:106120005E4BC5F8643C04F5994005F0D9F85C4B2A
:10613000C5F8803C04F599402C3005F0D1F8594B56
:10614000C5F8AC3C04F59940483005F0C9F8564B09
:10615000C5F8C83C04F59940643004F59A4605F04A
:10616000BFF80436514BC5F8E43C304605F0B8F8AA
:106170004F4BC5F8043D04F59A40203005F0B0F8C7
:106180004C4BC5F8203D04F59A403C3005F0A8F88A
:10619000494BC5F83C3D04F59A40583005F0A0F84D
:1061A000464BC5F8583D04F59A40743005F098F810
:1061B000434BC5F8743D04F59B40143005F090F84E
:1061C000404BC5F8943D04F59B40303005F088F80D
:1061D0003D4BC5F8B03D04F59B40503005F080F8CC
:1061E0003A4BC5F8D03D04F59B406C3005F078F88B
:1061F000374BC5F8EC3D04F59C40083008F014F925
:1062000004F59C40443005F06BF8324BC5F8443E31
:10621000314BC5F8603E04F59C404FF4C053A5F8DF
:10622000B43E2E4960304CF059FAFE2385F82C3FDD
:10623000052385F8503F4FF0FF33C5F8583F284BF2
:10624000C5F8206FC5F8246F11934BE0207D0D0831
:10625000000080BF0000B4420000B4C2F0950D08F9
:1062600000960D0878050F08D8020F0880020F0865
:10627000D8000F08EC730E085894002020490D0830
:1062800058A10D0854A80D0874AB0D08549F0D08B3
:1062900068A20D08F0A20D08D0A10D08D8A00D0825
:1062A00054A00D08E4A70D08E0A30D0870A30D0885
:1062B00038960D0860A40D086CA70D0860A50D08A0
:1062C00050A60D08D0A50D08E8A60D08E0A40D08FD
:1062D000E49E0D08F0AA0D0828960D0838260F0830
:1062E000C55C010805F57765894B85ED008A04F5E5
:1062F0009E4004F5A0454FF4007100932246854B63
:10630000109474301AF0DEF94FF0FF33C5F8D03432
:1063100005F59C63804ADA6003230026C5F85C35E6
:1063200005F5AF63C5F82865C5F82C65C5F8306577
:10633000C5F83465C5F83865C5F83C6583ED008A55
:10634000764BC5F8A03504F5AB49754BC5F8A835B3
:106350004846744BC5F8B035C5F89C45C5F8A4450A
:10636000C5F8AC4544301CF0B3FF484660301CF023
:10637000AFFF48467C301CF0ABFF6B4BC5F81036C6
:106380004FF0FF33A5F8143609F198001CF0A0FF78
:106390004FF0FF32654B6649C5F874264846C3F88E
:1063A00000904CF09BF94FF6FF73A5F8BC3504F54F
:1063B000AC404FF0FF33A5F8D835783054F0C4F92D
:1063C0005C4BD7F804261294CDE913345A4BCDE92F
:1063D00015345A4BCDE91734594BCDE91934594B83
:1063E000CDE91B34584B1D931EA911E903000CABDA
:1063F00083E80300DDE91A010AAB83E80300DDE965
:10640000180108AB83E80300DDE9160106AB83E859
:106410000300DDE9140104AB83E80300DDE91201A8
:1064200002AB83E803004946CDE9002853465A46AB
:106430000E988BF0BFFD0BF51B7304F5BF40C5F83C
:10644000D03F54301CF044FF04F5BF4064301CF0D2
:106450003FFF04F5BF4004F5C04774301CF038FF1F
:1064600007F170081C223146381DB9F0D1F94046B9
:106470007DF06AFC354B36493B6740464CF02EF9BF
:10648000344A3549116004F5C14328334FF0140CE8
:10649000B0B20CFB00120136127C002AF8D12F4A50
:1064A00010802F4A166816B12E488FF011FD04F5A2
:1064B000C1402C3013607DF031FC2B4BC7F8AC3061
:1064C00004F5C1405946383009F07CFA274BC7F82B
:1064D000B033642387F8B433254BC7F8E83304F5A9
:1064E000C740244BC7F8EC33234930304CF0F6F862
:1064F000224BC7F8B03320460123C7F8106487F851
:10650000186485F810351FB0BDEC028BBDE8F08F24
:1065100034460D08C55C01080000B442C95C01089E
:10652000CD5C0108D15C01080000FFFF3090002025
:106530000C270E08D55C0108D95C0108DD5C010858
:10654000E15C0108E55C0108E95C010804400D0814
:10655000DC3F0D08F89000203C8B0D08F4900020E3
:10656000B4900020CC950D0844400D0810960D08FD
:106570001CC70D0874C70D08E47A0E08F4C80D088E
:1065800010B58EF0E3FF064C064B18602046FFF76F
:106590008FFC2046044A0549BDE81040B6F0F6BB22
:1065A000902B00208C2B0020B0F00020ED5C010827
:1065B0000069C0F3401070470F299DBF302303FBD3
:1065C0000100503000207047014B93F921027047C1
:1065D000904B0020014BD3F8340C7047904B0020B7
:1065E00008B503689B68984730B9044B93F83A0F95
:1065F000B0FA80F0400908BD0020FCE7906B002055
:1066000008B504480EF052FF10B9034B93F8340F4D
:1066100008BD00BF902B0020906B0020022A10B50F
:106620000C4605D1BDE810400948352210F0A0BE47
:10663000084BD3F8200F03685B689847A04205D148
:1066400062F0DCFABDE8104062F062BA10BD00BF33
:10665000902B0020906B0020012910B50C4610D023
:10666000022904D061B961F01DF8084A02E061F026
:1066700019F8074A06215AF099F9064BC3F8504118
:1066800010BD61F00FF8044AF4E700BF50970D0801
:1066900028970D08908B00203F970D08012910B511
:1066A0000C4614D0022907D0D1B90E4BC3F81014F0
:1066B00060F0F8FF0C4A05E00A4BC3F8101460F0D4
:1066C000F1FF0A4ABDE8104006215AF06FB960F0A8
:1066D000E9FF074A06215AF069F9024BC3F8104452
:1066E00010BD00BF908B00208F970D0864970D0898
:1066F00078970D08012903D0022914BF0021022137
:10670000014BC3F8D41B7047904B0020012902D0E5
:10671000022900D011B9024BC3F81414704700BF0E
:10672000908B00206C2942DC3F2914DC382952DC94
:1067300026292DDC042964D010294CD17047A1F101
:10674000AA030B2B47D8DFE803F05C46465C4646BD
:106750005C464646465CA1F140032C2B3BD8DFE863
:1067600003F0443A3A3A3A3A3A3A503A3A3A3A50D4
:106770003A3A3A3A413A413A414141503A41503A23
:106780003A50503A503A3A3A3A3A3A3A3A50500035
:10679000A1F12703112B1ED8DFE803F0331D1D1DC7
:1067A000331D1D1D1D1D1D1D33331D1D3333A0291C
:1067B0000DDC95290FDDA1F196030A2B0BD8DFE83C
:1067C00003F0200A0A0A20200A200A0A1100B5292B
:1067D00003DCA929B3DC63F021B8A1F1D003022BBB
:1067E000F9D87047002362F0EBBF064B012283F813
:1067F0000C24A3F58043D3F8300C10B1642162F06F
:1068000043BA7047908B00206C2938B50346154673
:1068100000F3A0803F290FDC382907DC26296DDC36
:10682000042900F01A81102900F000812A46184638
:10683000BDE8384062F0BABDA1F140022C2AF5D87B
:1068400001A050F822F000BF056A01082D68010878
:106850002D6801082D6801082D6801082D680108C0
:106860002D6801082D680108356A01082D680108A6
:106870002D6801082D6801082D6801085F6A01086C
:106880002D6801082D6801082D6801082D68010890
:10689000A76A01082D680108FB6A01082D68010834
:1068A000B16A0108F16A01089D6A0108336B0108A9
:1068B0002D6801081B6B0108656A01082D68010835
:1068C0002D680108F36901083D6B01082D68010876
:1068D000436A01082D6801082D6801082D68010828
:1068E0002D6801082D6801082D6801082D68010830
:1068F0002D680108C56B01086B6A0108A1F1270228
:10690000112A93D801A050F822F000BFF3690108C2
:106910002D6801082D6801082D680108F769010834
:106920002D6801082D6801082D6801082D680108EF
:106930002D6801082D6801082D680108556A0108B5
:106940003D6A01082D6801082D6801084F6A010899
:10695000496A0108A02921DC95297FF767AFA1F1D9
:1069600096020A2A3FF662AF01A050F822F000BF5B
:10697000476B01082D6801082D6801082D68010882
:106980004D6B01089F6B01082D680108AD6B010874
:106990002D6801082D6801086D6B0108B52923DCFD
:1069A000A9297FF743AFA1F1AA020B2A3FF63EAF18
:1069B00001A050F822F000BF716A01082D6801089B
:1069C0002D6801088D6B01082D6801082D680108EC
:1069D000776A01082D6801082D6801082D680108F3
:1069E0002D680108E56B0108A1F1D002022A3FF6EB
:1069F0001DAF01248FE0A91E834B4D424D4183F80A
:106A00002D5FF6E7AA1E5542804C554184F80B5481
:106A100060F048FE7E4A94F80B147E4B002908BFB4
:106A200013467D4A062159F0C1FFE2E70A21FFF72C
:106A3000F5FDDEE72A4601211846F8E72A4604213B
:106A4000FAE72A460321F7E72A460C21F4E72A460B
:106A50000F21F1E72A460021EEE70B21E7E72A465E
:106A60000D21E9E72A460521E6E72A461521E3E755
:106A70002A461121E0E7AB1E5A425A41634B93F874
:106A8000B0119142B5D083F8B02160F00BFE634A9B
:106A9000634B022D08BF1346624AC3E729461846D6
:106AA000FFF728FEA5E729461846FFF7D5FDA0E722
:106AB000564CD5B1022D0DD1012384F80834A4F52C
:106AC0000053D3F8200F03685B6A984710B156480B
:106AD00000F09AFF60F0E6FD504A94F80814504B1D
:106AE000002908BF1346514A9CE784F80854E6E79A
:106AF00029461846FFF7D2FD7BE7012445B1022D58
:106B000009D1424BC3F80841002283F8F82102E082
:106B10003E4BC3F80851204638BD01242DB1022D4B
:106B2000F9D1434B83F83440F5E7414B83F83450B7
:106B3000F1E729461846FFF7E9FD5AE762F05EF8EB
:106B400061F0E6FF55E72A46072175E71846294612
:106B500062F05CFB37487DF037F9044600283FF4CB
:106B600048AF2A4B0122C3F80821CDE7274BD3F8C1
:106B7000C831002B3FF43DAF012425B1022DCAD10D
:106B800083F82C40C7E783F82C50C4E7022D7FF42C
:106B900030AF9FED290A2448FBF798FC29E7022D26
:106BA0007FF427AF20480EF08FFB22E701242DB1A0
:106BB000022DB0D1154B83F80A44ACE7134B83F890
:106BC0000A54A8E7022D19D10F4DD5F8200F0368FC
:106BD000DB6B9847044650B10121A5F5804003F0D6
:106BE0006FF998E7154829468DF062FA01E760F0E1
:106BF00059FD134A042159F0D9FEFAE60A4800214A
:106C000003F05EF9F5E600BF906B0020908B00204A
:106C1000A4970D08B37F0D08AC970D08C3690D0844
:106C2000C0A80D08BC970D08902B0020C8970D0830
:106C3000904B0020008C002000000000F079002024
:106C4000DB970D0810B599B104681168416004B96B
:106C50000160126801681B68521A9A4202D800212A
:106C6000084610BD017A012381F001010372F7E7A4
:106C7000037A3BB144682CB11368029A12681B1B5B
:106C80009342ECD90023C0E90033EFE70023C0E9C9
:106C90000533C0E908338385037780F828307047CF
:106CA000F0B52DED028B044687B09F48B0EE408AC8
:106CB0000E467DF093F840B1236933B1206B00F5A7
:106CC0000E7010F04FFE054638B12046FFF7DEFF8C
:106CD000002007B0BDEC028BF0BD236B93F93C2282
:106CE000002A1EDD93F8A032DBB1904BD3F81424B8
:106CF000002AEAD12369D4ED007A991E4842F5EEC4
:106D0000C07A4841F1EE10FA84F82C0027D8C4E983
:106D10000822C4E9052284F82D2084F8282022774F
:106D2000D7E7834FD7F8200F03689B6B984728B1AC
:106D300007F5805797F85835002BD6D07D480021AD
:106D40000EF04AFEDFED7C7AB4EEE70AF1EE10FABF
:106D5000CBDA784803F074FE0028C6D1B5E76EB1EF
:106D6000F4EEC87AF1EE10FA3CDD236BD3F8C432AE
:106D7000DB0403D5714815F0ADFB064684F82D60A1
:106D80008FF0D4F8D4ED027A9FED6D7A039067EE20
:106D9000877AFCEEE77A17EE903A5B000593B4F938
:106DA0000630CDED047A002B1EDC0023C4E9083345
:106DB00084F8283094F90430002B41DC0023C4E926
:106DC0000533237794F82C00002882D194F82D0005
:106DD00000287FF47EAF94F8280000287FF479AF74
:106DE000207F76E71646C9E70421524800F0B8FC38
:106DF000B4F9063007EE903AF8EEE77A05ABF4EE18
:106E0000C07AF1EE10FA0093CCBF0121002104AB4F
:106E100003AA04F12000B0EE408AFFF713FF002818
:106E2000C8D060F03FFC064618EE100AF9F76CFB7C
:106E3000444ACDE900010421304659F0B7FDB9E7D5
:106E4000414E9FED427AD6F8B824DFED416A06F54F
:106E50008051D1ED6F7A82EAE270B0EE476AA0EB22
:106E6000E270A7EEA66A07EE900AF8EEE77AF4EE73
:106E7000C67AF1EE10FA53D8D6F8BC0491ED706AD8
:106E800007EE900AA6EE267AF8EEE77AF4EEC77AD5
:106E9000F1EE10FA44D591ED716A9FED2E7AA6EECF
:106EA000267AF4EEC77AF1EE10FACCBF012700275C
:106EB000642113FB01F1284BD3F87005121A002A44
:106EC000B8BF52428A422DDAD6F8BC24D3F87435C2
:106ED000D31A002BB8BF5B428B42ACBF0023012307
:106EE00004F114000FB983F0010505AB009303AA68
:106EF00004AB2946FFF7A6FE00283FF463AF60F01D
:106F0000D1FBD6F8B814D6F8BC24642392FBF3F274
:106F100091FBF3F300920421104A59F047FD51E729
:106F20000027C5E70023DBE7008C0020908B0020C2
:106F3000906B0020902B002000000034503E002079
:106F400000007A44D4990D08903B00200000FA43D9
:106F50000000C8420000FAC3907B0020E5990D08AC
:106F600073B58289036BD20704466CD493F93C2233
:106F7000002A03DD93F8A022002A64D1524DD5F8EF
:106F8000201F05F55D6291425DD0A5F54055B3F92E
:106F90000860D5F8B83407EE903AD5F8BC34B8EEAE
:106FA000E77A07EE903AF8EEE77A6846CDED017A97
:106FB0008DED007A30F068F9730007EE903AF8EE44
:106FC000E77AB0EEC00AF4EEC07AF1EE10FA42D4DD
:106FD000236B93F8F1223AB307EE906AF8EEE77A62
:106FE000F4EEC07AF1EE10FA1EDB002183F8F11204
:106FF000236B586B85F030FC236B9FED347ADA6B92
:10700000D2ED067A05F2C46267EE877A92ED007AD5
:10701000F4EEC77AF1EE10FA06D5986B87F07CFE95
:10702000236B986B87F012FCA389226B13F0020389
:1070300002D192F8F11299B9002382F8F232236B4F
:1070400093F8F10205E0002083F8F102236B83F846
:10705000F20202B070BD236B012283F8F122B7E780
:1070600005F2DC51D1ED007A9FED197AF0EEE76A76
:10707000F4EEC76AF1EE10FADFDD05F2D451D1ED7E
:10708000006A9FED146AB0EEE67AB4EEC67AF1EECD
:1070900010FAD2DD05F5BB6191ED007AB0EEC77A4A
:1070A000B4EEC67AF1EE10FAC7DD67EEA67AF5EE19
:1070B000C07AF1EE10FAC0D5D5F8BC3406498B423F
:1070C000ACBF00230123B8E7906B00200AD7233C14
:1070D000C2B8323E920A063F6CEEFFFF08B5036B62
:1070E00093F8F2223AB1DA6A92F8A020022A03D089
:1070F000002283F8F22208BD0B4B9FED0C0AD3ED62
:10710000007AF5EEC07ADFED0A7AF1EE10FAD8BF18
:10711000B0EE670A152063F081F8BDE808409FEDE6
:10712000050A132063F07AB86C41002000A08CC5DA
:1071300000A08C450000000000F58040D0F8200F32
:1071400003681B6C1847000000F5005393ED907A1C
:1071500000F5A040B5EEC07AF1EE10FA5DBFD0F8B0
:10716000D03FDFED086AD3ED017AD0F8E80F5FBFBA
:10717000F8EEE77AE7EE267AFDEEE77A17EE900A68
:10718000704700BF0000C84200F5005090F8800230
:1071900028B141F00101084214BF012000207047CE
:1071A00010B54B68516800F5C0448B42D8BF0A4601
:1071B0006068CCBF1A4619462DF034F9606010BDE6
:1071C00010B5044650486BF073FB10F0080117BF70
:1071D0004E4BDFED4F7A93ED2B7AD3ED2D7A1FBF17
:1071E00077EE877A9FED4B7A012167EE877A10F070
:1071F000010317BF454B9FED467AD3ED2D6A93ED02
:107200002A7A1CBF37EE667ADFED426A04F5005237
:1072100018BF27EE267AD2ED926AF5EEC06A18BF43
:107220000123F1EE10FA33DD384A9FED3A6AD2EDD0
:10723000926A66EE866A0121F4EE676AF1EE10FA50
:1072400058BFF0EE667A04F5C042107B28B373B1E4
:10725000D2ED046AF8EEE66AF4EEC76AF1EE10FACF
:1072600058BFF0EE476AFDEEE66AC2ED046A99B1D6
:1072700092ED047AB8EEC77AB4EEE77AF1EE10FA3E
:10728000D8BFB0EE677ABDEEC77A82ED047A03E02C
:107290000029D8D1002BD6D110BDC3B104F5A0432D
:1072A000D3F8D03FD3ED016AF8EEE66A76EE876A4E
:1072B00092ED017AB8EEC77AF4EEC76AF1EE10FAF1
:1072C000D8BFB0EE667ABDEEC77A82ED017A0029AA
:1072D000E2D004F5A044D4F8D03F93ED017AB8EEA3
:1072E000C77A77EE277A92ED017AB8EEC77AF4EE94
:1072F000C77AF1EE10FA58BFB0EE677ABDEEC77AE2
:1073000082ED017AC8E700BF304C0020904B00208E
:10731000000000000000C84200F5C0400023836068
:107320007047000073B51646044600236A4630468F
:1073300000931CF0BBF848B1DDED007A9FED257A93
:1073400067EE877AFDEEE77A17EE900A04F5C045FE
:10735000A86033785B0717D52B7BABB104F5AC4045
:10736000012201A9783053F075FB68B1D5ED047A9C
:10737000DDED016A9FED177AF8EEE77AE6EEC77A5F
:10738000FDEEE77AC5ED027A04F5A043D3F85C354B
:10739000042B1DD004F50054B4F97A22002A15DD1F
:1073A000AB689FED0D7A83EAE371A1EBE37107EE21
:1073B000901AF8EEE77A67EE877A07EE102AB8EEB1
:1073C000C77AF4EEC77AF1EE10FA01D50023AB606C
:1073D00002B070BD0000C8420AD7233C37B50B7815
:1073E0005A0704460D461DD500F5AC40012201A9FF
:1073F000783053F02FFBA8B1D5ED017A2B78DFED73
:107400001C6AF8EEE77ADB0767EEA67A1BD59DEDDE
:10741000017AB4EEE77AF1EE10FACCBF0120002039
:1074200003B030BD2B78D5ED017A13F0010FF8EEE3
:10743000E77A04F5A04411D104F6E87393ED007ADD
:10744000B8EEC77AE5E704F5A044D4F8D03F93ED51
:10745000017AB8EEC77AE7EE667AD8E7D4F8D03F7B
:1074600093ED017AB8EEC77A77EE877AE4E700BF4A
:107470000AD7233C00F5005300F58042B3F92A32C5
:10748000D2F8202F00EE103A00F599439A42B8EE58
:10749000C00A0ED100F5A040D0F85C35042B02D014
:1074A00090F811352BB100F61470D0ED007A30EE63
:1074B000270A7047014608B501F5A041FFF7DAFF3A
:1074C00001F6E873D3ED007A9FED057AF8EEE77ADE
:1074D000E0EE477AFDEEE77A17EE900A08BD00BFAE
:1074E0000000C84237B500F5C04504462B7BDBB130
:1074F00000F5AC40012201A9783053F0ABFA98B105
:10750000D5ED047AD5ED056A9FED0A7AF8EEE77AB3
:10751000E6EE877ADDED016AE6EEC77AFDEEE77A00
:1075200017EE900A03B030BD2046FFF7C3FF6B682B
:10753000181AF7E70000C842014608B5FFF79AFF9E
:1075400001F5C041D1ED087A37EEC00ADFED047ACB
:1075500020EE270AFDEEC07A17EE900A08BD00BFA4
:107560000000C8422DE9F04100F5BF4800F5BF45D5
:1075700008F1640874350446294640461CF00AFAAE
:1075800004F5A04704F5BF4607F59F6354362A4625
:10759000314683ED000A40461CF032F907F2FC4701
:1075A000DFED220A87ED000AB7EE001A76202CF0F4
:1075B00099FE04F5335383ED770A2046FAF718FF56
:1075C00004F58043D3F8200F03685B6898470B28C5
:1075D0000CD007D80A2810D004F5C0440023A360BB
:1075E000BDE8F0810E38C0B20128F5D82946204602
:1075F000FFF7F4FE0028EFD011E029462046FFF700
:10760000EDFE30B90A484FF48041FBF727FA002815
:10761000E2D12046FFF790FFB0F5FA6FE6DD2A468B
:1076200031462046BDE8F041FFF77CBE0000000077
:10763000902B002010B52DED028B00F5A043DFED5F
:10764000208AD3F8F82F93F8F43F07EE902AB8EE8B
:10765000E78ADA0728EE288A82B0044609D400F5C2
:10766000805202F5A662D2ED007AF8EEE77AA7EE34
:10767000E88A5B070FD504F5AC40012201A97830F8
:1076800053F0E8F938B19DED010A30EE480A02B036
:10769000BDEC028B10BD204604F58054FFF70AFFB5
:1076A00004F5A66393ED000A07EE900AB8EEC00A4F
:1076B000F8EEE77A28EEC00AA7EEA80AE5E700BFD1
:1076C0000AD7233C73B504461646FFF75DFD78B92B
:1076D00066BB04F5C145383528460AF0D7FCB8B377
:1076E00028460AF073F898BB2046FFF7A3FF09E08D
:1076F00004F5005595F8503CDB0705D505F66C45BB
:1077000095ED000A02B070BD04F5C14038300AF0B2
:10771000E3FC0028DCD095F81A1C04F551604CF00D
:10772000E1FA0228D4D19FED0D0AEBE704F5A0435E
:1077300093F8103F022BCCD104F5AC40012201A9F3
:10774000783053F087F90028C3D09DED010AD9E7BE
:1077500004F5C04494ED080AD4E700BF000000001F
:1077600000F5C0431A7BFFF7ADBF000038B52DED23
:10777000028B00F5804200F59843D2F8202F203389
:107780009A4204464CD100F58053D3F8C05400F51A
:107790000053B3F97832002B65DD04F5B65292ED53
:1077A000017AF7EE007AB4EEE77AF1EE10FA5AD4E5
:1077B00004F53452D2ED007AF6EE006A67EEA67A4E
:1077C00087EE871AB5EEC01AF1EE10FA4BD907EE24
:1077D000905A9FED278AB8EEE70A07EE903A04F533
:1077E000AC4004F5C044F8EEE70A20EE080A783011
:1077F00053F03CFAA3689FED1F1ADFED1F0A002B20
:10780000BCBF07EE903AF8EEE77A4FF42970B8BFA4
:10781000A7EE880ABDEC028BBDE838402CF062BDB3
:1078200007F0E2FDF8B904F54053D3F80406036805
:107830001B69984704F50053DFED0F0AB3F978325E
:1078400001EE103A04F5A94393ED1E0AB8EEC11AF1
:10785000054640F27F202CF045FDBDEEC00A10EE3B
:10786000103A1BB297E7BDEC028B9FED030A38BDBF
:107870000AD7233C00007A440000000010B50446FB
:107880008EF054FB04F50053D3F8642C801A41F2B7
:10789000883290420FD802212046FFF775FC50B184
:1078A00004F5A044D4F85C25042A04D103F6584317
:1078B00093ED000A10BD9FED010AFBE700000000F8
:1078C00030B52DED028B00F5C045DFED278A2B7B0F
:1078D00083B004465BB3D5ED047A9FED240AF8EE3D
:1078E000E77A00F5AC4027EE800A012201A9783042
:1078F00053F0E8F8D8B12046FFF738FFDDED017A04
:1079000085ED050A37EE800A20468DED010AFFF766
:10791000B5FFDDED017A30EE270A20EE280ABDEE34
:10792000C00A10EE100A03B0BDEC028B30BD04F5A6
:10793000A0432046D3F8D02F6B6852689B1A08EEFC
:10794000103AFFF797FDB8EEC88A2046A0EE288AC5
:10795000FFF794FFBDEEC88AB8EEC88AA0EE288A69
:10796000BDEEC80ADDE700BF0000C8420AD7233CCD
:1079700010B500F580430446D3F8200F03685B6A16
:10798000984718B104F5C04494F8080410BD0000ED
:1079900038B500F5C0440D4663680B446360237B33
:1079A0002BB1FFF7E5FF10B921692944216138BDEA
:1079B00030B500F50050D0F87422D3070FD4094B2E
:1079C0000B201D785C688D4204D1224214BF012037
:1079D000002030BD013803F10803F2D1F9E701209E
:1079E000F7E700BF3C9A0D0810B500F58043044648
:1079F000D3F8200F03685B68984701462046BDE82E
:107A00001040FFF7D5BF000037B500F5A04300F5E3
:107A1000C045D3F8E83F6B600023AB600446FFF736
:107A2000E3FFC8B104F5AC40012201A9783053F05E
:107A300011F888B12046FFF79BFF68B9DDED017AA8
:107A40009FED077A67EE877A0123FDEEE77A2B73C5
:107A5000C5ED047A03B030BD00232B73FAE700BFF5
:107A60000000C84238B504460D46FFF7BDFF30B1EF
:107A7000032128461BF0F6FC80F00103D8B204F580
:107A8000C044607338BD000073B500F5C0454A6856
:107A90006A600B780E46D907044606D500F5A04368
:107AA000D3F8D03F5B6813446B606B7B2BB104F55C
:107AB000BF4174312046FFF7D5FF33785B070DD502
:107AC00004F5AC40012201A9783052F0C3FF28B17F
:107AD00001232B7373682B6102B070BD00232B73DD
:107AE000FAE70000F0B52DED028B044683B004F5F3
:107AF000C0450E468DED010AFFF7C6FFDFED320AE5
:107B00009DED010A40F24310B7EE001A2CF0EAFB9B
:107B1000AB685B4207EE903AF8EEE77A204667EEF4
:107B2000807A04F50057FDEEE77AB0EE408A17EE52
:107B3000901AFFF72DFFD7ED9F7AF5EEC07AF1EEA0
:107B400010FA3DDDAB68002B3ADD2046FFF7CAFC9A
:107B500007EE900ADFED1D6AB8EEE77AD7ED9F7A5F
:107B600067EEA67AB4EEE77AF1EE10FA28D5314640
:107B70002046FFF789FF04F5BF41324664312046B5
:107B8000FFF7D0FBAB685B4207EE903AF8EEE77A7E
:107B9000204667EE887AFDEEE77A17EE901AFFF737
:107BA000F7FEB5EEC08AF1EE10FA09DDD5ED027AE6
:107BB000B8EEE77AC7EE087AFDEEE77AC5ED027A0D
:107BC00003B0BDEC028BF0BD000000000000C8C295
:107BD000F0B500F5A04487B094F8F43F03F0050336
:107BE000052B07460BD053F083FF4FF4AE724FF4D2
:107BF000801153F035FF0025284607B0F0BD1E4820
:107C00006A4603211BF03EFC0028F4D01B4801AA61
:107C100003211BF037FC05460028ECD0184BDFEDA4
:107C2000190A93ED000A40F26D10B7EE001A2CF01D
:107C300059FB04F6F4730FCBB0EE401A02AEDFED41
:107C4000111ADDED010A9DED000AB7EE002A86E863
:107C50000F002CF079FADFED0C7A20EE270A30467F
:107C6000FDEEC07A032217EE901A1BF037FB314667
:107C70003846FFF709FFBFE7648B0020848B0020A4
:107C80008C800020000000000000C842F7B50E46BE
:107C900002210446FFF778FA70B304F5A045D5F841
:107CA0005C35042B28D12046FFF79EFE20B304F557
:107CB000AC47783704F5BF4101236A466431384642
:107CC00052F0B2FDC0B104F5BF41012301AA7431E5
:107CD000384652F0A9FD78B19DED017ADDED007ACC
:107CE00077EEC77A96ED007A37EE277A05F21C55C3
:107CF00086ED007AC5ED007A03B0F0BDF0B52DED4C
:107D0000048B00F5005489B000F5516694F81A1CF4
:107D10000391054630464BF0E5FF03990746304690
:107D20004BF0F2FF042F0399B0EE408A20D10023DC
:107D300005A88DED050A069307932FF025FD05A9EB
:107D400005F5AF502DF0EEFBDFEDAB7A8DED050ABA
:107D5000B4EEE71AF1EE10FACDED060A8DED071A32
:107D600006DB05F5805393F83C7517F001070CD13D
:107D700094F8503C002262F3000384F8682C84F8E5
:107D8000503C09B0BDEC048BF0BD94F8503C9A0710
:107D90005FBF43F0020384F8503C04F6544383ED84
:107DA000008A05F5315104F66C4383ED001A2C313D
:107DB0002846FFF76BFF94F8683C092B00F2888097
:107DC00004F54763D3ED000A9FED8C9AB0EE480AA4
:107DD0002CF076F900BB04F6544394F81A1CD3ED4A
:107DE000008A30464BF0AEFF07EE900A9FED847A92
:107DF000F8EEE77A78EEC88A67EE877AF0EEE88ADE
:107E000067EE897AF4EEE78AF1EE10FAC2BF94F8D1
:107E1000683C013384F8683C04F5476394F81A1C05
:107E2000D3ED008A30464BF08DFF07EE900AF8EE56
:107E3000E77A9FED747A67EE897A78EEC88A67EE02
:107E4000877AF0EEE88AF4EEE78AF1EE10FA02DDC6
:107E5000002384F8683C04F5476383ED008A94F8B6
:107E6000503CDA078DD52846FFF7E4FB04F66C4357
:107E700093ED008A05F5C04330EE488A1B7B002B4A
:107E800070D005F5AC40012205A9783052F0E2FD32
:107E900000286DD18EF04AF8D4F8642C41F2883174
:107EA000821A8A42034604F6584204F65C4168D9B5
:107EB00082ED008A284681ED008A0221FFF764F9ED
:107EC00018B105F5BE452A6AEA61C4F8643C58E772
:107ED00094F8503C43F0010384F8503C05F5A0436E
:107EE00005F59B42D3F85C6505F58043301FD3F858
:107EF000203F464202F114024641934211D005F55B
:107F00009B42303293420CD005F59942934209D1FD
:107F10003D4B05F5C140B3F8BE15383009F072FC91
:107F200000B13E4694F8503C590794D4002E92D0AC
:107F300002212846FFF728F900288CD043F00403DB
:107F400084F8503C04F66C4305F54F561868F8F772
:107F5000DBFA2836CDE900012C4A0621304658F0DC
:107F600025FD78E72846FFF73FFD002889D191E7F6
:107F700004F66C4393ED000A9DED058A38EE408AC5
:107F800088E79FED200A92ED007ADFED217A28EE56
:107F9000008AA7EE278A82ED008AC4F8640CD1ED2E
:107FA000007A38EE678AF3EE0E7AB0EEC88AB4EE45
:107FB000E78AF1EE10FA7FF7E4AE94F8503C5B07E5
:107FC0000ED504F66C4405F54F562068F8F79CFA78
:107FD0002836CDE900010F4A0621304658F0E6FC6C
:107FE00005F5315024220021103009B0BDEC048B7E
:107FF000BDE8F040B7F00CBC000000340AD7233CC9
:10800000CDCC4C3DCDCC4C3E907B0020FC990D0856
:10801000CDCC4C3F199A0D0838B52DED028B0D468D
:108020000446FFF707FB002320462B70B0EE408A82
:10803000FFF724FC0221204638EE400AFFF7A4F89F
:1080400028B104F5005494F8500C00F00100BDEC88
:10805000028B287038BD000070B50B7803F0050363
:10806000042B05460C46164615D105F5A04553F0E0
:108070003FFDB2B24FF4801153F0F2FCD5F8D02F8F
:10808000636852689B1A13F5FA7FC8BF6360237850
:1080900043F00103237070BDF8B500F5805300F57F
:1080A000A047D3F83065D7F82055B542044619D01B
:1080B0000E4A1268D26A92F89C209AB100F5BF412C
:1080C000751B25227431FFF7C7FF07EE905AB8EEF3
:1080D000E70ADFED077A04F5335020EE270A18305F
:1080E00080F052FDC7F82065F8BD00BF8C2B002042
:1080F0000AD7233CF8B500F5A044054694F813C50B
:108100000F4604F6D476BCF1000F53D004F6F47396
:108110000FCB86E80F00012384F8143597E80F0091
:1081200004F6F47686E80F00D4F8FC3F05F5BF4668
:10813000743693B905F5C0431A6872B9D4F8EC2FB8
:10814000C4F8FC2FD4F8F02F1A60D4F8F82F22B915
:10815000D4F8E81F30461BF0C1F8314628222846E3
:10816000FFF77AFF94F8F41F11F0040102D13046B2
:108170001BF078F905F5BF4105F5BF403246543193
:1081800064301BF073FB38B104F6D47604F6E47463
:1081900094E80F0086E80F00284606F0FDFC28460C
:1081A000FFF7E0F9284607F0E5F82846BDE8F84073
:1081B000FEF7C2BF04F6E4730FCB86E80F0001237D
:1081C00084F8133584F814C5A8E70000F8B500F565
:1081D00000530446B3F9D231002B0E4636DB0B7840
:1081E00013F0020F14BF4FF0FF33012304F5A04535
:1081F00005F6D47785F8AC3F05F6E4730FCB87E836
:108200000F0096E80F0005F6F47787E80F0004F5F5
:10821000BF41572274312046FFF71EFF2046FFF76B
:10822000F3FB2046FFF79EF9204607F0A3F800264F
:10823000204604F5C04485F81465C5F8B06F85F88C
:10824000196506F0A9FC84F8FA61F8BD4FF0FF3318
:10825000CCE700002DE9F043354B1B6885B005469F
:10826000D86AF9F761F900285FD105F5005393F951
:10827000E83B5A1C52D0002B05F5866611DD95F8B7
:108280004124242107EE903A01FB026292ED0B7A21
:10829000F8EEE77AB0EEC77AB4EEE77AF1EE10FACC
:1082A0003CDC05F5805305F5965793F83C3513F003
:1082B000010429D0C3F340089B0732D495F8E41396
:1082C00095F828444FF0B00909FB015191F8C131EC
:1082D0004CBB022B18D968461AF0FAFF694638469B
:1082E00015F0A4F8044678B195F8E43309FB03537C
:1082F0004246D3F8D01168461AF0F0FF15F06CFB37
:10830000694614F081FF0446304617F015FE3846E2
:1083100014F098FE2846FAF775FB204605B0BDE834
:10832000F0830024F0E74446EEE70020F6E700BFC4
:108330008C2B002038B50C4B1B680546D86A0C46C0
:10834000F9F7F2F810B10024204638BD15F044FBCF
:10835000214614F059FF04460028F4D005F5AB403F
:1083600030F02CF8F0E700BF8C2B0020F0B500F5C2
:10837000A045002385F8133585F8143505F6E47318
:10838000044600EE101A0FCB87B005F6D47686E8C7
:108390000F0002AE04F5BF42B8EEC00A30461749DE
:1083A00064324BF013FA96E80F0005F6F47787E88D
:1083B0000F0004F5BF4140F257127431204601917D
:1083C000FFF74AFE01992046FFF74CFB0199204632
:1083D000FFF75AFB04F500532046B3F9D231002BC6
:1083E000B4BF4FF0FF33012385F8AC3FFFF7BAF875
:1083F000204607B0BDE8F04006F0BCBF1862002080
:1084000010B5034904464BF0E1F9204610BD00BF0A
:1084100018620020F8B500F5A04404F6E4730546A0
:108420000E460FCB04F6D47787E80F0006F108015B
:108430002846FFF75FFEB388D4F8F82F03EB8303D9
:1084400003EB83039B001BB2002BD8BF4FF4C87310
:10845000A4F80E35D4F8D03F5968521AC4F8E02475
:108460009A680A32C4F8FC2FDB6805F5C0420A336B
:1084700013600023C4F8F43484F8103584F82435EC
:10848000C4F8E43404F59B6300221A604FF0FF3314
:10849000C4F8D03495F8412405F58663242101FB06
:1084A000023304F5A164DB6A2360F8BD70B50E46A3
:1084B00008310446FFF71EFEB38804F5A04543B318
:1084C000642213FB02F3C5F8E034B5F90E35002B36
:1084D000D8BF4FF47A7304F53150D8BFA5F80E35E4
:1084E000242200211030B7F093F904F5C04304F5BD
:1084F000BE4093ED080A3146143089F051FED5F89C
:108500005C35072B0CD120460421BDE87040F9F7FB
:108510003DBFD5F8E034002BD7DC40F6B833D2E7C6
:1085200070BD000030B5083104460FC985B06D46F6
:1085300085E80F0004F5BF41643128461BF032F88E
:1085400020462946FFF7D6FD04F580440123C4F8F0
:10855000483F05B030BD00000B7A00F5A04013F095
:10856000020F14BF4FF0FF33012380F8AC3F704778
:108570007FB501F1080305460E460FCB6C4684E833
:108580000F0005F5BF41643120461BF00BF8214672
:108590002846FFF7AFFD31462846FFF7DDFF04B060
:1085A00070BD00007FB501F1080304460E460FCBF5
:1085B0006D4685E80F0004F5BF41643128461AF086
:1085C000F1FF29462046FFF795FD20463146FFF78B
:1085D000C3FF337907EE903A337E9B0748BF9FED88
:1085E0000C7AF8EE677A04F5A04448BF67EE877A04
:1085F0009FED087A67EE877AFCEEE77A17EE903AFD
:10860000C4F8A43F0123C4F8C43F04B070BD00BF48
:108610000000803B00A00C477FB501F10803044631
:108620000E460FCB6D4685E80F0004F5BF4164315F
:1086300028461AF0B7FF29462046FFF75BFD204683
:108640003146FFF789FFB38804F5A0444FF47A72EE
:108650005343C4F8BC3F0123C4F8C43F04B070BD09
:108660002DE9F34100F5BF450446743500F5BF40E0
:108670000E46543029461AF055FF04F5A047C0B9FC
:108680004FF0FF33C7F8D03406F1080840461AF01F
:108690004FFE032802463AD1F16828461AF01EFE22
:1086A000B388C7F8C43F204602B0BDE8F041FEF7EA
:1086B00033BE24F087FBF9F7BDFB012812D94FF038
:1086C000FF33C7F8D03424F07DFB90F8C432DFEDDF
:1086D000150AB02202FB030090ED300A28461BF079
:1086E000FFF9D1E704F58058D8F8C0042BF0CEFD8F
:1086F00004F5A653C7F8D004D3ED007A9FED0A0A1B
:10870000DFED080AF8EEE77A27EE800AE6E701AA2D
:10871000002140461AF018FE0028C1D0019900221D
:10872000BBE700BF00007A440AD7233C7FB501F1C4
:10873000080304460E460FCB6D4685E80F0004F58E
:10874000BF41643128461AF02DFF29462046FFF725
:10875000D1FC20463146FFF7FFFE04F5A04400237C
:10876000C4F8C43F04B070BD37B504460D468DF063
:10877000DDFB2062D5ED027AF5EEC07AF1EE10FA5B
:1087800015DD9FED127A67EE877AFCEEE77AC4ED8D
:10879000077A5EF087FFE2694FF47A73B2FBF3F376
:1087A0000B4A062103B0BDE8304058F0FFB869F02D
:1087B000CDFE0023009395F90D2095F90E3095F923
:1087C0000C1069F05FFEE061E3E700BF00007A444F
:1087D000949A0D082DE9F0432DED028B85B00446E7
:1087E00015F0FAF814F0E0F904F5805304F5A0450B
:1087F00093F8B8370BB9002877D0D5F8D0340133C7
:1088000073D1D5F8F434002B4BD08DF08FFBD5F815
:10881000F434C01AB0F5FA6F67D394F8E423DFEDAF
:108820005F7A9FED5F8A4FF0B00808FB024292ED3D
:10883000780A20EE270A2BF041FD05F59B69D9ED5A
:10884000007A30EE670A2BF039FDDFED567A20EE24
:10885000080A04F54F5720EE270A2BF0D7FCFDEE4F
:10886000C07A283717EE906AC5F8D064D9ED007A3F
:1088700067EE887A17EE900AF7F746FECDE9020117
:1088800094F8E43308FB0343D3F8DC01F7F73CFE2C
:10889000454ACDE9000133460621384658F086F8AE
:1088A00023E004F59070F9F7C5FA02281DD994F871
:1088B000E433B02202FB034393ED777AF1EE047ABE
:1088C000B4EEE77AF1EE10FA0FDD384B1B68D86A88
:1088D0000368DB699847012803D08DF027FBC5F8B2
:1088E000F404D5F8F434002B8FD104F54053D5F8B7
:1088F000D014D3F804064A1C036845D01B6B984774
:108900002B4810F0FFFC18B104F5AB4031F0B6FF76
:108910002046FEF711FED5F8E0348342064636DAEB
:1089200007EE906A9FED237AF8EEE77A04F54F544C
:1089300067EE877A283417EE900AF7F7E5FD1E4AAE
:10894000CDE900012046062158F030F801244FF00F
:10895000FF33C5F8D03485F8104505F6E4730FCB26
:1089600005F6D47605F6F47786E80F0087E80F0061
:10897000124869F067FF002385F81335204605B0DB
:10898000BDEC028BBDE8F0835B6B9847B8E7084805
:1089900010F098FC0028C3D1F1E700BF35FA8E3CF7
:1089A000E02E65420000C842A49A0D088C2B0020DE
:1089B000902B00200AD7233CC89A0D08304C002089
:1089C0002DE9F04100F5BF4700F5BF455437743538
:1089D0000446294638461AF0A5FD04F5A04604F5DC
:1089E000405830B3D6F8D0144B1C22D0D8F8040627
:1089F00003681B6B9847D6F8C43F012B47D0D6F8C5
:108A0000C43F022B06D12046FEF754FDD6F8F83FAE
:108A1000984243DD2046FEF74DFDD6F8F83FC01AD8
:108A20000028B8BF4042B0F5FA7FCCBF002001203B
:108A300035E004F5BF40294664301AF0ABFFDFEDA6
:108A4000197AB4EEE70AF1EE10FA16D5384629463F
:108A50001AF070FE9FED147ADFED140AF6EE007A3C
:108A6000E0EE077A28469FED120AFDEEE77AF8EE6F
:108A7000E77A27EE800A1BF033F8D8F804069FED5A
:108A80000D0A03682A469B6A39469847B3E7204691
:108A9000FEF710FDD6F8F83F9842B0DB0120BDE8A4
:108AA000F08100BF00004843A00CB345000096438E
:108AB0000AD7233C0000000073B5394CD1ED026A9F
:108AC000D4F8E83F9FED377A07EE903AF8EEE77A70
:108AD0000546D7EE876A0E46F5EEC06AF1EE10FA4B
:108AE00008DD5EF0DFFD304A062157F05FFF012010
:108AF00002B070BDD1ED037AF5EEC07A04F59E6444
:108B0000F1EE10FA94ED006A12DDF4EEC67AF1EEA1
:108B100010FA0DD55EF0C6FD05462068F7F7F4FCA7
:108B2000224ACDE900010621284657F03FFFDEE743
:108B3000DFED1F7A337CB4EEE76AF1EE10FA54BF32
:108B4000B0EE677AB0EE467A0BB90020D0E7B5EE0A
:108B5000C06AF1EE10FA0CDC86EE876A03EB830341
:108B600007EE903AF8EEE77AF4EEC67AF1EE10FAF4
:108B7000EBD595F82440002CE7D18DF0D7F9AB6AFE
:108B8000C01A337C4FF47A7253439842DDD90123E3
:108B900085F824308DF0CAF9A8622046A8E700BF06
:108BA000907B00200AD7233CE49A0D08F59A0D0823
:108BB0000AD723BC38B505467CF02AFB7BF00EF9BA
:108BC000044640B98DF0B2F92B6AC01AEB6998429D
:108BD00084BFEC610124204638BD000038B504464E
:108BE0000D468DF0A3F904F5A0439FED077AC3F875
:108BF000C80FD5ED027A67EE877AFDEEE77A17EEB9
:108C0000902AC3F8C42F38BD00007A4410B504463A
:108C10008DF08CF904F5A043D3F8C82F801AD3F84F
:108C2000C42F90424FF0000084BFC3F8C40F01204E
:108C300010BD000000F5A04303F59F61D3F8C42FD9
:108C400091ED007A22EAE27207EE902AF8EEE77AD6
:108C50000020B4EEE77AF1EE10FA44BFC3F8C40F77
:108C60000120704710B500F5005300F5A040B3F99E
:108C7000D231002BB4BF4FF0FF33012380F8AC3F5B
:108C800000F6F47400F6E4700FC884E80F0010BD1D
:108C900038B504462DED028BF0EE408AB0EE608AC6
:108CA00009B301295ED0B5EEC08AF1EE10FA69DD94
:108CB000DFED357AB4EEE78AF1EE10FA62D8FCEE19
:108CC000C87A04F54F5017EE903A304A0621283002
:108CD00057F06CFEFDEEC87A04F5005417EE903A9A
:108CE00084F89F313CE0F8EE000A2BF0E9F940B13E
:108CF00004F580444FF0FF33C4F8583FBDEC028BBD
:108D000038BD04F50053B3F9A82107EE902AF8EE18
:108D1000E77AF4EEE87AF1EE10FAC4D8B3F9AA31A2
:108D200007EE903AF8EEE77AF4EEE87AF1EE10FA10
:108D3000B9DBDFED157A68EEA77A04F58043FDEE26
:108D4000E77A04F54F5017EE902AFCEEE87AC3F864
:108D5000582F062117EE903A0D4A283057F026FE7C
:108D60000120CBE7FCEEC07A00F54F5017EE903AA9
:108D7000084A0621283004F5005457F017FEC4EDC8
:108D80006D8AEDE70020B9E70000C8423B9B0D0863
:108D9000149B0D08289B0D08D1F80D3000EE903A79
:108DA000D1F80930097A00EE103AFFF771BF0000E0
:108DB00070B58B88012B04460D4611D100F59076D5
:108DC0003046F9F737F802280AD994F8E413B023AB
:108DD00003FB01612046AC31BDE87040FFF7AABA41
:108DE00014F0FAFD05F10801BDE8704014F00CBA6A
:108DF000F0B500F5A0470024AA4B87F8194589B0C3
:108E0000054608460E465C732FF0EAF898B3012336
:108E100087F8103505F54053D3F804060368DB6B7B
:108E2000984787F81745C7F8B04F03A81AF050FACB
:108E3000B7F8BC154FF6FF73994208BF21460131C0
:108E400001AA89B205F5AB4031F09AF8F0B1BDF84E
:108E50000630A3F115025342534187F8113550B142
:108E600005F5C140BDF80610383008F0CBFC10B154
:108E7000002387F8113573885E2B4DD8522B07D805
:108E8000103B9AB20F2A21D90024D4E00346E4E72C
:108E9000533B0B2BF8D801A252F823F03190010874
:108EA0003D9001084D900108898E0108898E0108C6
:108EB000898E0108898E0108898E0108898E010832
:108EC000898E0108999001084D9001080F2BDBD87D
:108ED00001A252F823F000BFB58F0108EF8F0108FF
:108EE000F98F01080390010817900108C18F01084C
:108EF000878F0108898E0108898E0108898E0108F3
:108F0000898E0108898E0108898E0108898E0108E1
:108F1000279001080D900108BD2B1AD8BB2B47D80C
:108F2000B22B00F0A7800DD8702B00F09E80722B22
:108F3000AAD1D6ED027AFDEEE77A17EE903AC7F89D
:108F4000C43F35E0B32B9FD131462846FFF730FFB1
:108F50002EE0D42B00F0938040F6B832934200F01C
:108F60009680D22B90D1B388012B21D803F0010336
:108F700087F8123505F54F50B3884B4A0621283043
:108F800057F014FD14E0002305F5C14487F8493576
:108F900038347188204607F0DBFE314628B1204680
:108FA00009B0BDE8F04008F0D5B82846FFF732FA1E
:108FB000012440E006F108012846FFF79BF8F7E797
:108FC00005F5C14438341521204608F01BFC48B192
:108FD000002387F849353146204609B0BDE8F04006
:108FE00007F0BCBF31462846FFF760FAE0E731469C
:108FF0002846FFF7BDFADBE731462846FFF7D2FAED
:10900000D6E731462846FFF707FBD1E73146284629
:10901000FFF78CFBCCE705F5994129222C31284636
:109020000EF0CEF8C4E731462846FFF719FBBFE73C
:10903000012487F81745204609B0F0BD002305F547
:10904000C14087F8493531463830A9E705F5C147B1
:109050003837384608F0BAFB3146044618B128467E
:10906000FFF760FAE7E73846B7E731462846FFF7EB
:10907000B5FD9DE731462846FFF78EFE98E7B1889B
:10908000003918BF0121284600F01AFF90E7317A15
:10909000064807F05DFA8BE7314605F59940FFF782
:1090A00063FB85E7908B00204C9B0D08488C0020CB
:1090B00000F5804200F59943D2F8202F9A4201D161
:1090C000FFF796BE0120704710B500F5804200F50D
:1090D0009943D2F8202F9A4204460DD1194608220E
:1090E0002C310EF06DF804F54F50044ABDE81040E5
:1090F0000621283057F05ABC10BD00BF5C9B0D08FC
:109100002DE9F04F2DED048B00F5C04393ED4E8A11
:10911000DFEDD77AB0EEC87AB4EEE77AF1EE10FA66
:1091200048BF00F50053DFEDD37A42BFB3F9D23127
:1091300008EE103AB8EEC88A00F5A048B4EEE78A07
:10914000F1EE10FA94BF4FF0FF37012700F580458C
:1091500088F8AC7FD5F8483F9BB004460E46F0EE49
:10916000C88A052B16D8DFE813F006002C0069002A
:109170008800C5005F0100F540543A46D4F8040663
:109180000368B0EE680ADB6A08319847BA4806F00F
:109190002BF908B9002048E1B84C54F8303CB4F938
:1091A00078115B68642201FB0231A4F5C040FFF72F
:1091B000DDF8A4F5C04005F0EFFC0123C5F8483FF9
:1091C000E8E700F540533A46D3F804060368B0EEEA
:1091D000680ADB6A08319847D8F8A83F002BB8BF67
:1091E0005B42012BD6DD98F8AD3F1BB998F8AE3F36
:1091F000002BCFD004F5B153D3ED020A93ED030A4F
:10920000F1EE600AB1EE400AB4F008F9DFED9C7AA5
:1092100020EE270A05F64C7383ED000A10EE100AC3
:10922000F7F772F904F54F542834CDE90001954A57
:109230000621204657F0BAFB0223BFE700F5BF49DD
:1092400001F1080A09F16409494650461AF0A2FBE7
:1092500030EE680AF1EE047AB0EEC00AB4EEE70A26
:10926000F1EE10FA00F3E680D8F8A83F0133022BA4
:1092700040F2EA800323C5F8483F04F5405306F165
:109280000808D3F8040603683A46DB6AB0EE480AD9
:1092900041469847DFED7C6A9FED7C7A05F64C737A
:1092A000D3ED007A012F18BFB0EE667A04F5A6530D
:1092B00077EE877A93ED030A9FED757AA7EEC70ADA
:1092C0002AF0FCFFDFED737AB0EEC00AB4EEE70AD5
:1092D000F1EE10FA7FF55EAF04F54F50062128300D
:1092E0006D4A57F063FB0423C5F8483F41462046CA
:1092F000FEF700FF06F1080595E80F000AAF0DF133
:10930000380887E80F0088E80F0004F5804303F66B
:109310004C7A9FED629A9AED000ADFED610A0393A1
:10932000384630EE090A1AF0DBFBDFED5D0A9AEDF4
:10933000000A9FED5C8A40461AF0D2FB04F54053C8
:109340004246D3F80406036839469B6AB0EE480AE1
:10935000984795E80F0004F5C1490DF1480B09F154
:1093600038098BE80F00DAED009A484607F016FD41
:1093700079EE899A04F5BF48F0EE400A5846B0EEFF
:10938000690A08F164081AF0ABFB5A4639464046B0
:109390001AF06CFA834695E80F009AED000A16AFB2
:1093A00087E80F00F0EE680A30EE090A38461AF036
:1093B00097FB394640462A461AF022FA07A904F5D7
:1093C0009650F0EE408A8DED078A8DED088A8DED7E
:1093D000098A14F0FFF8002866D0294640461AF0A2
:1093E000E5F905A907A8CDED060A8DED050A2DF0D2
:1093F0005FFFDFED237A20EE270A2AF0F3FEB0EEBE
:10940000C00ABBF1000F3FF4C5AEF3EE0E7AB4EE26
:10941000E70AF1EE10FA23D5039A0523C2F8483F74
:109420003146484607F09AFD01201BB0BDEC048B85
:10943000BDE8F08F494650461AF0ACFAB4EEE80A9F
:10944000F1EE10FA7FF510AF04F540543A46D4F827
:1094500004060368B0EE680ADB6A5146984799E64D
:10946000F6EE007AF4EEE78AF1EE10FAD4DC91E63B
:1094700000000034000000B4902B0020908B0020EE
:10948000E02E6542849B0D080000B4420000874333
:1094900035FA8E3CC2B8B23DA69B0D08000034439D
:1094A00000007A4400000000BBF1000F3FF472AEF0
:1094B000B2E700BF2DE9F041054600F5C1408EB08E
:1094C0003830884608F0C2F9044650BB09AF05F5AC
:1094D000A046384619F0FCFEB6F8BC354FF6FF72D0
:1094E000934208BF0023013307AA99B205F5AB40A8
:1094F00030F046FDC8B1B8F1000F01D0C6F8A84F52
:1095000097E80F0001AC84E80F0005F5C04506F6AA
:10951000F4762B68009396E80E00054803F0C6F930
:10952000044620460EB0BDE8F0810124F9E700BFF3
:109530005878002070B5064606F5A045002106F0D3
:1095400051F8D5F8B04F7CB9304605F04DFF10B951
:109550000024204670BDD5F8A83F012BF8DD8CF023
:10956000E5FCC5F8B00FF4E7D5F8C41F61B18CF085
:10957000DDFCD5F8B03FC01AD5F8BC3F9842E7D91A
:109580000023C5F8C43F01213046FFF793FF04468E
:109590000028DDD006F54F50044A0621283057F048
:1095A00005FA002385F81935D3E700BFC89B0D08DD
:1095B00070B50A468B88190A137E0546DB0748BF3B
:1095C00001EB810105F5A04448BF4900002606F0E3
:1095D00009F884F81965284605F006FF10B900243B
:1095E000204670BDD4F8C41F51B1D4F8A83FD4F8B8
:1095F000A42F9342F3DD012BF1DDC4F8C46F0121E8
:109600002846FFF757FF04460028E8D005F54F50DD
:10961000024A0621283057F0C9F9E1E7E09B0D081E
:1096200038B5054605F5A044898805F0DBFFD4F878
:10963000C43F83BBD4F8A83F002BB8BF5B42012BCB
:1096400002DC0024204638BD94F8AD2F94F8AE3FDC
:1096500072B9002BF5D005F54F50D4F8E82F6423EC
:10966000062192FBF3F328300C4A57F09FF901E0F2
:10967000002BF0D10121C4F8C41F2846FFF71AFFC0
:1096800004460028DDD005F54F50054A0621283054
:1096900057F08CF9D6E70021EFE700BFF89B0D08E3
:1096A000169C0D0810B504460B4808F0BBFE48B1E7
:1096B0000A4BDFED0B7AD3F8F43093ED090A20EE74
:1096C000270A10BD04F50054B4F9003200EE103A38
:1096D000B8EEC00AF5E700BF488C0020908B002050
:1096E0000AD7233C38B52DED028B00F5005300F569
:1096F000A045B3F904120029ACBF01234FF0FF339A
:109700000029B8BF494285F8AC3F044689B205F04C
:1097100069FF05F59F65204695ED008AFFF7C2FFBA
:10972000B5EEC00AF1EE10FAD8BF9FED0E0ABCEEFE
:10973000C00AB8EE400AB4EEC08AF1EE10FA0AD8B8
:1097400004F54F502830084A062157F02FF9012020
:10975000BDEC028B38BD204605F046FE0028EFD157
:10976000F6E700BF00000000309C0D082DE9F0472F
:1097700000F5A0472DED028B4FF0FF33C7F8D03432
:1097800007F6F4738C4605460FCBBCF804609CF8D2
:10979000049088B004AC360A84E80F0020D005F5A8
:1097A000BF4808F15408214640461AF0F3F8214614
:1097B0004046B0EE408A19F0BDFFDFED587AB4EEB6
:1097C000E78AF1EE10FA0BDBF3B200EE903ADFED30
:1097D000547AF8EE600A20EE270A20461AF080F943
:1097E00005F5405A97F81425DAF804069FED4D0A5E
:1097F000036805F5BF489B6A08F1640832B305F5B4
:10980000BF4122465431984705F50053B3F902325F
:10981000002B1EDD07EE903A07F59F62F8EEE77A1F
:1098200092ED007AB4EEE77AF1EE10FA11DD05F56B
:10983000BF412246543140461AF018F8F8B90026C4
:10984000304608B0BDEC028BBDE8F08722464146A9
:10985000D9E7B9F1000F1DD1002E3DD1DAF8046629
:1098600033682846D3F82090FFF71CFF07F2EC433B
:10987000D3ED000A3046C847B0EE408A0EE0002E15
:10988000DDD107F6D47407F6E47797E80F0084E893
:109890000F00D5E707EE909AB8EE678A214640465A
:1098A0001AF078F8B4EEC08AF1EE10FA17DBB7F8C8
:1098B000BC350393214640461AF06CF8BCEEC00A52
:1098C00005F54F50039B184A8DED000A06212830FC
:1098D00057F06CF80126B3E79FED128ADEE705F535
:1098E000BF4122465431404619F0C0FF06460028C9
:1098F000A5D0B7F8BC350393214640461AF04AF884
:10990000BCEEC00A05F54F50039B084A8DED000AD6
:109910000621283057F04AF892E700BF00000034D3
:10992000E02E654200000000489C0D08669C0D0872
:109930002DE9F0474B881F2B8AB004460D466BD8A3
:109940000F2B41D804F54F50BE4A0421283057F060
:109950002DF89BE0A3F1BC02182AF3D801A151F81D
:1099600022F000BF8D9A01088D9A010845990108DF
:10997000459901084599010845990108459901084B
:109980008D9A0108459901088D9A010845990108A9
:1099900045990108459901088D9A010845990108E2
:1099A00045990108459901088D9A01088D9A010889
:1099B0008D9A010845990108459901088D9A010879
:1099C000459901088D9A0108A3F110020F2AB9D810
:1099D00001A151F822F000BFC99A0108AF9B01080C
:1099E000B99B0108C59B0108DB9B0108D59A0108BA
:1099F0009F9A010845990108459901084599010870
:109A000045990108459901084599010845990108BA
:109A1000E59B0108CF9B01085E2B21D8522B91D9E1
:109A2000A3F153020B2A8DD801A151F822F000BFF7
:109A3000EF9B0108FF9B0108099C0108459901085B
:109A4000459901084599010845990108459901087A
:109A50004599010845990108339C0108099C0108B2
:109A6000722B00F0E18007D8702B7FF46BAF0AB047
:109A7000BDE8F047FFF7CAB8D42B09D8BB2B3FF697
:109A800069AFA3F1B202012A3FF65CAF012052E0B8
:109A9000DF2BFBD040F6B8329342F7D052E700F507
:109AA000C14638361621304607F052F930B1294602
:109AB00030460AB0BDE8F04707F03EBC20460AB089
:109AC000BDE8F047FEF786BE29460AB0BDE8F0477C
:109AD000FFF74CBE00F5C14538351521284607F083
:109AE00091FE28B128460AB0BDE8F0470BF08EB9C8
:109AF00004F5A04504F5BE46D5F85C3504F5BF472E
:109B000004F5BF4804F5BF49072B06F1140607F119
:109B1000540708F1740809F164090FD104F5AA4447
:109B200058340194D5F8E034009342464B46394608
:109B3000304688F0F9FB0AB0BDE8F0870DF1270147
:109B40008DF827004048FEF767FA05F21C53D3ED65
:109B5000007AD5F800A505F59E63D3ED000A05F25D
:109B6000FC4330EE670A93ED001A8DED070A04F509
:109B7000C0407030CDED060A8DED051A7AF024F95B
:109B80000546204600F05CFF9DF827309DED051A44
:109B9000DDED060A9DED070ACDE90203CDE900A53A
:109BA0004B4642463946304688F014FBC3E7A98845
:109BB00005F018FD0020BEE729460AB0BDE8F047D1
:109BC000FFF7F6BC0AB0BDE8F047FFF7B3BC294683
:109BD0000AB0BDE8F047FFF723BD0AB0BDE8F04783
:109BE000FFF780BD0AB0BDE8F047FEF7E9BE2946A1
:109BF00004F599400AB0BDE8F047FEF75DBF04F5F3
:109C0000C1402946383054E704F5C146383630465D
:109C100007F0DCFD08B9304665E729462046FFF726
:109C20006FFA0028F7D186E70AB0BDE8F047FFF7E2
:109C300001B8294604F599400AB0BDE8F047FEF79F
:109C4000B9BF00BF849C0D08902B002070B500F5B3
:109C5000804200F59943D2F8202F9A4205460E46DD
:109C600002D00024204670BDFFF762FE04460028A3
:109C7000F7D005F54F50318828305AF0D7FFF1E77B
:109C800021F04003152B04D0A1F15E035842584146
:109C9000704701207047000000F5804200F59943AD
:109CA000D2F8202F9A4207D100F5A040B0F8BE3577
:109CB0005B1A58425841704700207047192962D8F2
:109CC000DFE801F00D1115191D2125282C61303315
:109CD000365539393C3F4246494D6151595D00F591
:109CE0009A402030704700F596407430704700F578
:109CF00097401030704700F597402C30704700F5C2
:109D000097404830704700F598400430704700F5A0
:109D10009840E6E700F598403C30704700F59840E1
:109D20006430704700F59940704700F59940E4E7CA
:109D300000F59940E5E700F59940F1E700F59A4014
:109D4000E3E700F59A40E7E700F59A40583070479E
:109D500000F59A40C9E700F59B401430704700F5C4
:109D60009B403030704700F59B405030704700F505
:109D70009C400830704700F59C404430704700F527
:109D80009B406C30704700207047000000290DDBBD
:109D9000074890F84C2CCBB29A4207D3D0F8483CF5
:109DA0000122595CA0F500500DF0E2BA704700BFE7
:109DB000904B00202DE9F34100F5005300F54F557D
:109DC00093F8183C03F0010603F0020803F00407BF
:109DD0005B07044605F1280535D01F4A06212846B1
:109DE00056F0E4FD26B104F53D501C307CF01EF821
:109DF000B8F1000F04D004F5425034307BF092FDEE
:109E000027B104F548500C307CF03AFC04F5C0440E
:109E1000012384F80934114A114B1249B8F1000F9B
:109E200008BF1A46002F08BF1946CDE900210E4A87
:109E30000621002E18BF134628460C4A56F0B6FDE0
:109E400002B0BDE8F0810A4A0621284602B0BDE80A
:109E5000F04156F0ABBD00BFB19C0D08A69C0D08AB
:109E600038880E08AD9C0D08A09C0D08C29C0D08FA
:109E7000D49C0D0810B5044600F53D501C307CF014
:109E800001F804F5425034307BF078FD04F5485079
:109E90000C307CF02FFC04F5C04393F809245AB130
:109EA000002283F8092404F54F50044ABDE810400D
:109EB0000621283056F07ABD10BD00BFF49C0D0875
:109EC00009B1FFF777BFFFF7D5BF000000F580436A
:109ED0000949D3F8202F8A420CD093F82D3F3BB983
:109EE00000F599418A4203D100F5A04090F812355F
:109EF000184670470023FBE7B078002010B50446F1
:109F00008CF014F8054BD3F8403FC01A642804D8ED
:109F10002046BDE810405EF0EBBD10BD906B002008
:109F200010B500F53054D4ED027AF5EEC07AF1EEBA
:109F300010FA8AB04FF0000304F1080444D90793E3
:109F40000893099306AB019307AB009303AA05ABF3
:109F500004A900F5965013F0DDF930B3DDED080AE1
:109F60009DED070AB3F0BEF8DDED090AB3F0BAF8CB
:109F7000D4ED007A9DED047A77EEA76AB4EEE70A95
:109F8000F1EE10FAF4EEC76AACBF01200020F1EE4A
:109F900010FA0CD802309DED037AF4EEC77AF1EE98
:109FA00010FA0CD8003818BF01200AB010BDF4EE2A
:109FB000C77AF1EE10FA9CBF0130C0B2EBE701287E
:109FC00094BF00200120F0E70020EEE738B5124BE7
:109FD0001A7A0446FAB901251D7253F09BFB2A46F2
:109FE00004F5C1451121383553F04CF9284607F0E6
:109FF00071FC80B1284607F029FC062238B104F52F
:10A000009B411431BDE8384004480DF0D9B804F53F
:10A010009A415831F6E738BDB08F0020902B0020D0
:10A0200010B5074B1A7A4AB100241C7253F072FB28
:10A0300022461121BDE8104053F024B910BD00BFE5
:10A04000B08F00202DE9FF41054605F5965868467A
:10A0500019F03EF96946404613F0B0FA0646E8B1F9
:10A06000374879F0B1FE50B105F53053D3ED027A9F
:10A07000F5EEC07AF1EE10FA94BF0126002605F540
:10A08000C140383007F026FC2E4C2F4F00B146B1AE
:10A09000002328462380FB73FFF7C2FF04B0BDE80E
:10A0A000F0812846FFF73CFFA0B363787BBB2378A1
:10A0B0000133DBB2082B237002D1404613F096F92E
:10A0C0002378092B02D1404613F088F92378092B15
:10A0D0001DD94FF48573238053F01CFB02221021FD
:10A0E00053F0D0F88BF022FF6368C01A47F2305368
:10A0F000984209D905F54F50144A0221283056F0EC
:10A1000055FC8BF013FF60602846FFF75FFF637814
:10A11000FB73C3E72378002BF9D0013B6278DBB2F5
:10A120002370002AF3D0002BF1D1667053F0F2FABD
:10A130003246102153F0A6F82846FFF771FFE6E7F4
:10A14000008C0020B08F00205D900020089D0D083D
:10A1500010B500F5A044D4F85C35042B01D10120E2
:10A1600010BD00F5C140383008F042F90028F6D1A2
:10A1700094F88805F4E7000073B500F58045019276
:10A18000A5F8381F04468BF0D1FEC5F83C0FD5F872
:10A19000200F03685B68984785F8360FD5F8200FC5
:10A1A00003685B689847019A182818D8DFE800F020
:10A1B0000D170D0D0D0D0D0D0D175217591759597E
:10A1C00017414141171717415900334B93F80A348F
:10A1D00003B304F59841043120460CF0F1FFD5F8A3
:10A1E000200F95F8366F03685B68984704F54F5465
:10A1F000864204F1280447D0D5F8200F03689B68F5
:10A200009847264A03460421204602B0BDE8704024
:10A2100056F0CCBB04F5005393F91432022BD8D07E
:10A22000042B0BBF04F5984104F59641203174319D
:10A23000D2E704F5C043D3F87C33D90203D504F543
:10A2400099412C31C8E704F59B419B064CBF303146
:10A250001431C1E720460192FFF77AFF019A0028E6
:10A26000BDD104F50056019296F91432002BB6D0F8
:10A27000D5F8200F03685B68984785F8360F96F984
:10A280001432019A022BCAE7054A0421204602B083
:10A29000BDE8704056F08ABB908B0020189D0D08D9
:10A2A0003A9D0D08F0B5044604F5804685B00F468A
:10A2B00015465EF0A3FBD6F8200FA6F8387F03689A
:10A2C0005B68984718281ED8DFE800F00D0D0D0DCB
:10A2D0000D0D0D0D0D1D607D0D0D6C6C1D4E4E4E4A
:10A2E0001D1D1D4E0D003B4BD3F85C25012A21D1CD
:10A2F00004F5005393F81532023B012B1AD904F5EB
:10A30000405383F8E423D6F8200F334A334B052D0E
:10A3100018BF1346026803939268904704F54F54A0
:10A3200028340090039B2E4A0421204656F03EFB21
:10A3300005B0F0BD2B4B93F80A343BB104F59841BE
:10A340002A46043120460CF03BFFDCE704F50053BD
:10A3500093F91532032BD6D0022BEFD0042B2DD13D
:10A360002A4604F59941EDE704F5C043D3F87C3360
:10A37000DA0223D49B0604D504F59B412A463031EA
:10A38000E0E704F59B412A461431DBE72046FFF75E
:10A39000DFFE0028B7D104F5C140383007F0C4FA19
:10A3A0000028EED104F5005393F91532032BAAD0FF
:10A3B000022BC3D0042BD3D0012BA4D104F5994197
:10A3C0002A462C31BEE704F5005393F91532042BCD
:10A3D00099D1C5E7907B0020509D0D0838810D086C
:10A3E000589D0D08908B002070B500F54F55044620
:10A3F0002835124A0421284604F5804656F0D6FA3C
:10A400000023A6F8383F04F5005393F85C31032B82
:10A4100012D196F8361F302220460CF0A9FFD6F84C
:10A42000200F03689B689847054A03460621284683
:10A43000BDE8704056F0BABA70BD00BF6C9D0D0803
:10A44000839D0D0800F5405310B5002205290446F0
:10A4500000F54F5083F8E42300F128000CBF054AB3
:10A46000054A042104F5804456F0A0FA0023A4F81C
:10A47000383F10BD9C9D0D08AD9D0D08013A38B5C3
:10A480000446052A3ED8DFE802F04A1B86113D0348
:10A4900000F5C04393F8CC3143B100F59B41042251
:10A4A0006C314148BDE838400CF08ABE04F5C04329
:10A4B00093F8CC3123B104F59B4104221431F0E729
:10A4C00004F58043D3F8202F04F59B4314339A42BC
:10A4D00025D004F59B436C339A4220D004F5A04369
:10A4E000D3F85C35042B1AD0304D95F8513FB3B1F9
:10A4F0002F4905F5AC5030F015F920B12D4B012254
:10A5000083F8882538BD2A4905F5AC5030F00AFC9F
:10A5100028B1042204F59941A5F58040C2E704F56D
:10A520008043D3F8202F04F59B4314339A42E9D09B
:10A5300004F59B436C339A42E4D004F5A04304F540
:10A54000C1403830D3F85C5507F052FF0028D9D10C
:10A55000042DD7D004F5005393F9DF31022B0DD031
:10A5600004F59941204604222C310CF029FE04F513
:10A5700006501F30BDE8384048F086B90B4890F8C7
:10A58000513F002BECD00A4900F5AC5030F0CAF82E
:10A590000028B3D1E4E700F5C040BDE8384001220F
:10A5A00014217030F7F7F4BA902B0020906B002044
:10A5B000748B0020907B002070B52DED068B044637
:10A5C0008BF0ACFC414BB4F8BE101A88404E8A4266
:10A5D0000546404A06D01980002330601370BDEC58
:10A5E000068B70BD33683C49C31A8B4265D9012381
:10A5F00013705EF003FB5EF0BBF935605EF0FEFAAF
:10A600005EF0B6F95EF0DCF90428E8D95EF0F6F900
:10A61000204600210BF00CF820460021B0EE40AAA5
:10A620000BF010F820460121F0EE409A0BF0D4F91F
:10A6300000212046B0EE408A0BF00EF804F5C04031
:10A640007030F0EE408A79F0C9FB9FED249A002823
:10A65000B0EE4A0A4FF0040008BFB0EE498A5FF03E
:10A66000DDFDB0EE690A13205FF0D8FDB0EE680A98
:10A6700015205FF0D3FDB0EE680A1A205FF0CEFD22
:10A68000B0EE480A46205FF0C9FD0121084660F09F
:10A69000D1F8B0EE490A02205FF0C0FDB0EE490AE1
:10A6A00003205FF0BBFD20460BF0C4FBBDEC068B26
:10A6B0002046BDE870400CF00FBB1278002A8ED007
:10A6C00044F6206293428AD993E700BFBC8F0020F2
:10A6D000C08F0020BE8F0020400D0300000000004E
:10A6E00000F5804200F59943D2F8202F9A4204D118
:10A6F00000F5A04090F88805E8B10F4B93F85C0195
:10A7000003F58043A0F12702012A93F818340FD9EA
:10A710002C2809D00A2809D0A0F13102504250411A
:10A720000A2B18BF002070470120F9E7012070476D
:10A730000A3B584258417047904B002008B500F53D
:10A74000005393F8A02042B193F8DC302BB1FFF70F
:10A75000C7FF80F00100C0B208BD0120FCE7000087
:10A760002DE9F04700F50055AF4F95F8DC80044621
:10A7700000F5C0408AB0703079F026FBD7F85C3520
:10A78000042B064642D1012104F50257DFF8ACA2A2
:10A790002037384668F0BCFB9AF818340A2B8146FB
:10A7A00004D1002E54D100238AF8183495F8A03033
:10A7B000002B59D195F9A6309C4D012B03D0063BB7
:10A7C000DBB2012B11D895F85C310A2B0DD104F5C1
:10A7D0008046D6F8200F03681B6A984728B1D6F840
:10A7E000241F2B2220460CF0EBFC9AF818340A2B7D
:10A7F00004BF37238AF8183495F85C310A2B02D14C
:10A80000372385F85C310AB0BDE8F0870028BAD05C
:10A8100004F58043B7F8BE95D3F8200F03685B6852
:10A8200098471428AFD004F5C140383007F02EFC0B
:10A830000028A8D14946A7F5A040FFF721FA014614
:10A840000028A1D097F884154B1E594259419BE727
:10A8500040EA0803DBB2002BA8D1AAF5C04000F003
:10A86000EFF800289FD0A1E7002ECCD004F5BE4021
:10A87000143087F025FC0028C5D12046FFF730FFB3
:10A880000028C0D1B9F1000F00F0BD8068494A46E8
:10A89000384667F015FF95F9A680B8F1010F06D08C
:10A8A00040F38580A8F10603DBB2012B7FD85FFA65
:10A8B00088F8B8F1010F4DD104F5804204F59943B1
:10A8C000D2F8202F9A4209D104F5A04393F8883595
:10A8D00023B195F8DF31013B012B94D904F599415F
:10A8E0000A222C31204606AE0CF06AFC304618F0E5
:10A8F000EFFC95F9B92092BBB8F1010F2FD004F508
:10A90000A048B5F9BA30D8F8D01FDFED4A5AD1EDDA
:10A91000017A002BF8EEE77A52DD07EE103AF8EEF6
:10A92000C76AE6EEA57A3046FDEEE77A17EE901A92
:10A9300018F0D4FC00233846CDE9043368F084FBDA
:10A9400004A969F0C5F8002857D0049B0893059B1B
:10A95000099317E004F599410A226431C2E72046C1
:10A96000FCF7F2FB07EE900A6F4604F5BF42643233
:10A9700021463846B8EEE70AFDF742FD97E80F009A
:10A9800086E80F0095F9A630012B10D031462046FD
:10A99000FDF768F831462046FDF718FC95F9A6301A
:10A9A000072B04D104F54054012384F8E23352F01C
:10A9B000B1FE4A4609210AB0BDE8F04752F062BC38
:10A9C000D5ED2A6A95ED2D5A95ED2B7A35EE076A6D
:10A9D00036EEC57AB4EEC67AF1EE10FA89BF37EEDC
:10A9E000067A95ED907A27EE257AF6EE006A94BF06
:10A9F000E7EE257AE7EE267A95E7D8F8D03F9A6811
:10AA00000892DB68A4E7B8F1000F3FF4FCAE95F8BC
:10AA1000DC30002B7FF4F7AE04F54F50064A0521D9
:10AA2000283055F0C3FFC2E7907B0020904B0020F8
:10AA3000C89D0D080000C842D19D0D08908B0020D4
:10AA400010B5044600F5C040703079F0C7F998B1F0
:10AA500004F5C140383008F0C1F960B904F5AA44E2
:10AA600094ED187ADFED087AB4EEE77AF1EE10FA99
:10AA7000ACBF0120002010BD04F5AA4494ED187A63
:10AA8000DFED027AF0E700BFCDCCCC3D6666663FD5
:10AA900070B500F5804600F59C43D6F8202F0833AA
:10AAA0009A42044600F5A04502D195F85805D0B960
:10AAB00004F5C140B5F8BE15383006F049F998B92B
:10AAC000D6F8203F04F59944A3420CD195F85835A7
:10AAD0004BB1D5F85C35032B05D1B5F8BE05A0F117
:10AAE00016035842584170BD0020FCE72DE9F74F8E
:10AAF00000F5804200F59943D2F8202F9A4204468F
:10AB000000F5A04504D100F5005B9BF9B8313BB9D5
:10AB10000023C5F84C3585F8493503B0BDE8F08F02
:10AB20008BF004FAD5F80465804636B1861B40F6F2
:10AB3000C3139E4294BF002601262046FFF780FFE4
:10AB4000019028B1002785F848754FF0000A46E0CB
:10AB500004F5C040703079F037F981460028F1D013
:10AB600004F5BE4A0AF1140A504687F0A9FA0746CE
:10AB7000002845D095F848A5BAF1000F3BD156B34F
:10AB800004F5805041F27071D0F8B824002AB8BFA3
:10AB900052428A4206DCD0F8BC24002AB8BF524296
:10ABA0008A422BDD04F5AB4104F5BF4044316430EB
:10ABB00018F0F0FEDFED487AC5F84C85B4EEE70AF0
:10ABC000F1EE10FA4FF000024CBF4FF0010A4FF0C7
:10ABD000000AC5F85025012285F84825374604F5B6
:10ABE0009070F7F727F9022832D9002F44D10023BB
:10ABF000C5F84C3591E7019EB246ECE75646EAE7C8
:10AC0000504687F045FA824648B1002E9DD04FF459
:10AC1000FA73C5F850354FF0000A4F46DFE7D5F814
:10AC20005C25012A07D0032AD9D12046FFF730FF3F
:10AC300000288AD1E9E7DBED967AF5EEC07AF1EEED
:10AC400010FA82DD95F85835002B7FF47EAFDEE7F1
:10AC500004F5F75604F50059083699F836103046D1
:10AC600010F06EFB0028C2D099F83610304610F074
:10AC70005FFC0028B9D1BAE7D5F84C0510B9C5F882
:10AC80004C854AE7D5F85025A8EB00089045FFF41D
:10AC900044AF95F84925002A7FF43FAF012285F89B
:10ACA00049259BF8B811CB0705D504F5C0400C2108
:10ACB0007030F6F76DFF04F54F502830BAF1000FF1
:10ACC00006D0064A022103B0BDE8F04F55F06EBE33
:10ACD000034A5146F7E700BF00009642E89D0D0881
:10ACE000FE9D0D082DE9F04F2DED028B044685B039
:10ACF000002304F5005903938BF018F9D9ED6D7A10
:10AD0000F5EEC07AF1EE10FAC4BF9FEDC37A67EE9C
:10AD1000877A04F5907BC8BFFCEEE77A80465846F8
:10AD2000CCBF17EE907A9627F7F784F8022840F206
:10AD3000018194F8E4339FEDB97AB02202FB03431A
:10AD4000D3ED777A67EE877AFCEEE77A17EE903AE2
:10AD50009F428CBF00270127B9F9A831022BB8BF49
:10AD6000022307EE903AB8EEE78A03A9F6EE087AD6
:10AD700004F5965028EE278A12F0FEFB054640B1F6
:10AD8000DDED037AF4EEC87AF1EE10FAACBF0125DE
:10AD900000255846F7F74EF8012804F5A0461AD8C2
:10ADA00004F5C040703079F00FF8A0B19DB906F5F8
:10ADB000AC6393ED007ADFED9A7AB4EEE77AF1EEC8
:10ADC00010FA08DDDDED037AF4EEC87AF1EE10FA40
:10ADD000ACBF0125002504F5C140383005F012FA5A
:10ADE0008246002840F0F78004F5C040703078F0CB
:10ADF000EBFF002800F0FD8094F8E43304EB03132C
:10AE0000D3F890317BB158460193F7F713F8012836
:10AE100000F29280019BA8EB030041F28733984235
:10AE20008CBF00230123D6F8002502B11BB9002DE9
:10AE300040F084803D4604F5804204F59943D2F801
:10AE4000202F9A4219D199F9E031002B7ED10023AD
:10AE500086F84A35D6F85C35042B00F0A880072B1D
:10AE600000F0BB80032B08D12046FFF711FE20B174
:10AE7000002586F84955C6F8045596F84A3503B1B9
:10AE80008DB907EE905A9FED677AF8EE677A06F56E
:10AE9000AC6367EE877AD3ED006A9FED637AE6EEE6
:10AEA000877AC3ED007A2046FFF7CAFD0546A0B1B8
:10AEB00096F86415C6F8008509B9C6F8688504F5E2
:10AEC000804204F59943D2F8202F9A4205D1D6F852
:10AED000043503B109B9C6F8048586F8645571F0E4
:10AEE00003FF294671F0DCFE504B20465D71FFF7F1
:10AEF000FDFD2046FAF77EFB35B199F85E311BB9AE
:10AF00008BF014F8C9F8600189F85E512046FFF70C
:10AF100097FD00287ED104F5C040703078F05EFFC8
:10AF200080F00100C0B286F86C0505B0BDEC028B64
:10AF3000BDE8F08F00270FE7534674E728F096FC32
:10AF400027F0E4FD00287FF475AF74E75B4207EE5D
:10AF5000903A04F69803F8EEE77A93EDDB7AF4EE94
:10AF6000C77AF1EE10FA13DD012386F84A35C6F8E8
:10AF7000548506F5AC63DFED2E7A93ED007AB4EEDE
:10AF8000E77AF1EE10FA7FF765AFC3ED007A61E77B
:10AF900096F84A35002B3FF45DAFD6F8543540F6AD
:10AFA000B832A8EB030393423FF651AF52E704F5E2
:10AFB000BE40143087F06CF800283FF45EAF06F511
:10AFC0009E6393ED007ADFED1A7AB4EEE77AF1EE44
:10AFD00010FA7FF752AF01254FE706F59E6393ED18
:10AFE000007AFEEE007AB4EEE77AF1EE10FAF2D4CF
:10AFF00043E7D6F85C35002D18BF3D46012B01D143
:10B0000000253AE704F5BE40143087F037F80028F1
:10B01000F6D132E7002086E70000B4420000C842C3
:10B020009A99993E9A99193E9A99593F5D900020B4
:10B03000CDCC4C3E00207047002070470120704767
:10B04000034BD3F85C05431E58425841704700BF7C
:10B05000907B002030B587B002A818F039F93D4840
:10B0600087F00CF820B13C493C48FCF70DFD1FE08F
:10B07000384887F00DF8E8B1394C04F1240523462F
:10B0800004F11002A4F11001A4F1D000009587F0A2
:10B0900025F8CDE90045A4F6EC2292ED000A3149ED
:10B0A00004F11003A4F11002A4F1D00086F0D8FF3F
:10B0B00007B030BD274802A987F028F808B102A9D7
:10B0C000D2E7294CD4F8D03B002B0CDD94F8703B30
:10B0D0004BB1A4F500502249FCF7D6FCA4F5005072
:10B0E000FCF71AF9E4E71D4804F07EF90028BAD10C
:10B0F0001E4D95F8F43F5B0724D41D4CA368002B2C
:10B10000B1D0A4F10C02A4F12C01A4F11C0018F0A0
:10B11000ADFB0028A7D105F2FC45D5ED007AB7EECE
:10B12000000AA4F10C01A4F5C04030EE670AFCF758
:10B13000D9FCA4F12C02A4F10C01A4F5C040FCF749
:10B140002FF8B5E7A5F5A040FCF742FD0028AFD1E8
:10B15000D3E700BFA48A0020848B0020902B00201E
:10B16000748B0020E0570020904B0020907B002043
:10B17000908B002008B50A4890F85132013B012B12
:10B1800003D8A0F50050F8F709F90648F7F7CCFF07
:10B190000448F8F7C3F8BDE808400248F8F724BCB3
:10B1A000904B0020902B002010B5044607480CF06F
:10B1B000FDFE50B1064B93F8F90130B123682046EB
:10B1C0009B6B984780F00100C0B210BD808E0020BC
:10B1D000908B0020124B984210B5044601D10020FC
:10B1E00010BD03F11C029042F9D003F138029042E5
:10B1F000F5D003F174029042F1D0D4339842EED0EE
:10B2000003681B6A984720B1064B93F8E233002B82
:10B21000E5D1206907F006F980F00100C0B2DFE750
:10B2200020770020905B0020174B984210B5044611
:10B230000ED003F11C0290420AD003F13802904272
:10B2400006D003F17402904202D0D433984206D162
:10B250000E4B93F90902B0FA80F0400910BD036863
:10B260001B6A984718B10A4B93F8E23343B9206937
:10B2700007F0D8F830B12069BDE8104009F07CBC77
:10B280000020EBE70120E9E720770020904B002029
:10B29000905B002073B50F4E0D46114696F9842140
:10B2A0001AB90124204602B070BD036801915B69A0
:10B2B000984704460028F4D1D6F87C33019913F45A
:10B2C000802FEED00448054B00682A46C06A25F05E
:10B2D0007BFCE7E7908B00208C2B0020109E0D0854
:10B2E000084A0260084A4260111F816002F10801A9
:10B2F000C160A2F1380102F59C724261034A01610A
:10B30000826170475C9E0D08808C0020503E0020BA
:10B3100008B503681B6E98470648D0F8202F00F642
:10B3200064439A4205D0BDE80840A0F58040FEF78E
:10B33000A1BD08BD906B00202DE9F3415B4C04F5E5
:10B340009B6300221A60A4F56073C11A4B42A4F5F6
:10B3500000584B4188F8783604F59D63002584F841
:10B36000BC54A4F8125584F8165584F8D45484F8C3
:10B37000495584F84A55C4F83C55C4F83855C4F8C2
:10B380003455C4F844551A608369D3F8FC31A4F8E5
:10B390000C3504F6E47306460FCB04F6D47787E841
:10B3A0000F0084F8155584F82455C4F8B05F8AF06E
:10B3B000BDFD44F8D80C336830465B6998474FF0C0
:10B3C000FF3384F8195588F8E45344F8A83C84F80E
:10B3D0001805306906F0B2F904F5805384F8175562
:10B3E0005D7333683046DB6D9847A4F5805705469A
:10B3F000002857D0336830469B6B984784F858052F
:10B40000D8F804060368DB6B9847A4F5E4507AF09B
:10B4100075FEA4F5A0400AF05DF8A7F5FB5067F0B3
:10B42000DDFD94F88835C3B1A4F5A040FFF708FB13
:10B4300098B91F4878F0D2FC78B9D7F8200F036884
:10B440005B6B984748B95CF02DF91A4A062155F014
:10B45000ADFA04F5B0602FF011FA1748F6F7C8FFFF
:10B46000336993F9CC206AB1586801A912F084F8C5
:10B4700034699DED010A014604F18800FBF710FCD8
:10B4800084F84101336830465B69984750B13369AD
:10B4900093F93C22002A02DD93F8A03213B900236D
:10B4A00087F82D3F284602B0BDE8F081907B002050
:10B4B000008C00201C9E0D08902B002070B50368A6
:10B4C0005B6E0E4615469847044650B995F9003014
:10B4D0003BB90548054B00683246C06A294625F04D
:10B4E00073FB204670BD00BF8C2B0020409E0D08D2
:10B4F00010B50E4C20467AF0FDFB04F5AC707AF0E6
:10B5000075F904F52C707BF0A3F8094B03F5A04204
:10B51000002182F8D41402F59B62002103F5005348
:10B520001160012283F8A82E10BD00BFEC5A002044
:10B53000902B002008B52DED028B1520B0EE408A2F
:10B540005EF06CFEB0EE480ABDEC028B1A20BDE83E
:10B5500008405EF063BE000008B5084890F9093263
:10B560000121A0F5005033B10AF036FABDE80840D9
:10B5700046205EF053BE0AF057FAF7E7904B0020E2
:10B58000012070470120704701207047012070475B
:10B59000012070471920704700487047C49E0D086D
:10B5A00000487047D49E0D0884B038B505AC84E8D7
:10B5B0000E00054614210C48FCF7FAF92A696423A9
:10B5C000B2F9C01068B103225943204617F086FE35
:10B5D00005482146FCF7FAFDBDE83840012004B0DB
:10B5E00070470122F0E700BF902B002013B50F49F0
:10B5F00001AAA1F1100017F059FF40B1DFED0C7A5C
:10B600009DED017AB4EEE77AF1EE10FA0CD8094C10
:10B61000D4F8040603689B6B984728B106492E228C
:10B62000A4F540500BF0CCFD02B010BD848B00207F
:10B63000000000B4905B00202479002030B51D4C40
:10B640000546D4F8240F036887B05B69984738B182
:10B6500019491A482F220BF0B3FD012007B030BD65
:10B66000174806F0DFFE0028F2D1A4F58054D4F884
:10B67000040603689B6B984728B1D4F80406036856
:10B680001B6C984798B10F4B0FCB02AC84E80F00AE
:10B69000284601F06DF82868059B009394E80E0099
:10B6A000446C2846A0472846FFF7A0FFD5E7064B85
:10B6B000EAE700BF906B002024790020902B002047
:10B6C000488C0020748B0020848B002010B5044629
:10B6D000FFF78CFF2046BDE8104001F085B8000060
:10B6E0000420704700487047C9A40D0800487047FF
:10B6F000C9A40D08037F73B1D0ED087AFDEEE77A97
:10B7000017EE903A084AC2F87035437F3BB1436A5E
:10B71000C2F8743570478369D3F8F831F2E783696A
:10B72000D3F8FC31F4E700BF907B002008B500237C
:10B73000838300F12801806911F034FF012008BDE6
:10B7400070B56E4E2DED048B06F59E430446012127
:10B75000304693ED1C9ADFED6A9A09F069FF0121EA
:10B76000B0EE408A304609F06DFFC8EE297A06F542
:10B770000055A069B5F92C3204F1280108EE903A81
:10B78000F8EEE88AB5F92E3268EEA78AC0EE297A7B
:10B7900008EE103AB8EEC88A28EE278A11F002FFA8
:10B7A00095F9323263B39FED577AF0EEE87AF4EE12
:10B7B000C77AF1EE10FA23D5227FA369002A55D16A
:10B7C000012222770022226294ED087ADFED4E7A80
:10B7D000D3F8F8314D4A4E4867EEC77A9FED4D7A5F
:10B7E00067EE877AB0EE490AFDEEE77A17EE901A17
:10B7F0000B44C2F87035002301227AF00BFA08E0FE
:10B80000002343482377F0EE490AB0EE680A7AF045
:10B81000FDF904205EF002FD95F9323243B19FED4F
:10B82000397AF0EEC87AF4EEC77AF1EE10FA28D43D
:10B83000002339486377F0EE490AB0EE480A79F000
:10B840003FFE13205EF0EAFCB5F93032002B03DD39
:10B85000324E96F9223263BB28482021F7F7FEF8D2
:10B86000002843D1254809F005FD42E0D3EDC56A23
:10B8700096ED467AD4ED087AE6EE877AC4ED087A3A
:10B88000A2E7637F2BB901236377A369D3F8FC3167
:10B8900063621E4B616AC3F87415A369D3F8FC0197
:10B8A0000023091A1A461C48B0EE490A79F0EEFE48
:10B8B000C7E70121A6F5405009F0CEFE80EE297AB7
:10B8C000B5F93032002106F5037007EE903AF8EE34
:10B8D000E77AF0EE490A27EE870A7AF0B9FDBDEC67
:10B8E000048B2046BDE87040FFF724BE0348F7F7FD
:10B8F000E7FE07EE900AB8EEE70AF0E7902B00208B
:10B9000000A08C4500000034E02E6542907B0020B2
:10B91000EC5A00200000C842445C0020905B0020EC
:10B920002DE9F04F2DED0C8BDFF8A8A39FEDDEDAAB
:10B930009FEDDE9A97B00AF59E4300F12805044674
:10B940000121504693ED1CBA09F072FE01215046C8
:10B95000F0EE408A09F076FE01215046B0EE408AB2
:10B9600009F07AFEDFEDD27A88EEA77A0AF5005662
:10B9700001A8B6F92C320AF5A04B0AEE903AF8EE7F
:10B98000EAAAB6F92E32DFEDCB8A6AEE87AA88EEF4
:10B99000277A0AEE103AB8EECAAAB6F930329FED0D
:10B9A000C68A2AEE07AA80EE277A09EE903AF8EEC8
:10B9B000E99A6AEE8D7A69EE879AF0EEEACAF4EEB9
:10B9C000C8CACDED017AB0EECACA6AEE0D7AF1EEC0
:10B9D00010FAF0EEE9BAB4EEC8CACDED027A58BF5B
:10B9E0004FF0010969EE8D7A48BF4FF00009F1EE82
:10B9F00010FAF4EEC8BA9AED460ACDED037A54BFB8
:10BA00004FF001084FF00008F1EE10FA54BF012783
:10BA100000272BF0BFFD01A928462BF065F828462A
:10BA20002BF05CF928462BF0CBF820EE090A2846CB
:10BA300020EE280ABDEEC00A10EE103ACBF87035A1
:10BA40002BF0D8F820EE090A20EE280ADFED9B8AB9
:10BA5000BDEEC00ACDED0D8A10EE103ACBF874356C
:10BA60000DF1280B4FF07E535946A0690A93CDED96
:10BA70000C8ACDED0B8A11F095FD0021504609F09E
:10BA8000ABFFB0EEC00AB4EEC80AF1EE10FA16D55C
:10BA90005046FEF7D5FF90B9F4EEC8CAF1EE10FAA1
:10BAA0000DD5B4EEC8CAF1EE10FA08D5F4EEC8BA56
:10BAB000F1EE10FA44BF9BE80F0085E80F000AA8DA
:10BAC0002BF070F9294612A88DED141A8DED120A8B
:10BAD000CDED130ACDED151A2BF076F90DF1100A04
:10BAE00051460EA88DED101ACDED048ACDED058AD4
:10BAF000CDED068A8DED0E0ACDED0F0ACDED111AB2
:10BB00002AF02CFFB6F92C32DFED6D7A01EE103AF7
:10BB1000B6F92E3209EE103AB6F9303208EE903A04
:10BB2000B8EEC11AB8EEC99AF8EEE88A21EE271AE3
:10BB300029EE279A68EEA78AF4EEC8CAF1EE10FA49
:10BB400021EE0D1A29EE0D9A68EE8D8A07D594F82C
:10BB50003830DFED5A7A002B18BFB0EE671AB4EE1A
:10BB6000C8CAF1EE10FA07D594F83930DFED537AF0
:10BB7000002B18BFB0EE679AF4EEC8BAF1EE10FAD7
:10BB800007D594F83A30DFED4D7A002B18BFF0EE70
:10BB9000678A9AE807000DF11C0B8BE80700F1EEAD
:10BBA000410AC2209DED070A28F09CFBC3208DEDC1
:10BBB000070AB0EE491AF1EE490A9DED080A28F08D
:10BBC00091FBB0EE681AF1EE680A8DED080AC42008
:10BBD0009DED090A28F086FB514658468DED090A6D
:10BBE0002BF06EFC12A928468DED120ACDED130A3A
:10BBF0008DED141A06F576662AF076FF28462BF0AE
:10BC00006DF8DDED076A96ED007A2E4B9FED270A61
:10BC1000C6EE877A5846DDED086ACDED077AD3ED9A
:10BC20002E7A86EEA77ADDED096A8DED087A86EE2A
:10BC3000A77A8DED097A2BF0ADFCB9F1000F01D098
:10BC4000CDED07AAB8F1000F01D08DED08AA0FB114
:10BC5000CDED099AF0EE4B0A9DED070A1A4879F0EE
:10BC6000D5FF04205EF0DAFAF0EE4B0A9DED080AEB
:10BC7000164879F025FC13205EF0D0FA0021F0EE92
:10BC80004B0A9DED090A12487AF0E2FB2046FFF7C5
:10BC900051FC84F8389084F8398084F83A7017B0F1
:10BCA000BDEC0C8BBDE8F08F35FA8E3CE02E654282
:10BCB00000A08C450000C8420000003400000000D5
:10BCC000CDCC4C3E905B0020EC5A0020445C002020
:10BCD0009C5D0020902B002010B50446FFF73CFC33
:10BCE0000B4B93F93222022A0DD1B3F93022002AEC
:10BCF00009DD03F5805393F9223223B12046BDE8D4
:10BD00001040FFF70DBE2046BDE81040FFF718BDFC
:10BD1000904B00200A2070470048704792C40D08DD
:10BD20000048704792C40D080120704701207047F9
:10BD30000120704701207047034BD3F85C05031FB7
:10BD400058425841704700BF907B002070B50546AF
:10BD50002D48D0F8242F00F6E4439A4215D12B69E0
:10BD600093F844318BB100F5AC502EF051F90446F4
:10BD700058B95BF097FC254A032154F017FE2B6954
:10BD8000012283F84321204670BD214A92F8CC312C
:10BD900023B192F984319A1E534253411D4D85F8C7
:10BDA000183505F6E4730FCB05F6D47405F6F47672
:10BDB00084E80F0086E80F0005F5B0602EF09EFFC6
:10BDC000154B1C68E66A336830465B689847B0B12B
:10BDD00096F84D309BB1E36A9B8F83B15BF062FCB8
:10BDE000E36A0E4A9B8F062154F0E0FDE36A05F5F5
:10BDF000B060998F2EF06EFDE36A00229A870848A2
:10BE000087F0BEF80124BEE7906B0020BC9F0D08B0
:10BE1000908B0020907B00208C2B0020D69F0D085B
:10BE20007855002038B50D4C94F88435012B10D18D
:10BE300004F5B0602CF048F8B4F8BE55084829461F
:10BE400005F0E0FC28B9152D03D104F6147086F036
:10BE5000F5F90023C4F8043538BD00BF907B0020FD
:10BE6000488C002008B511F0B7FD90F87C32DB0754
:10BE700004D5BDE8084002482EF0DCBD08BD00BF77
:10BE80001081002038B5344C94F88435012B0ED045
:10BE9000A4F555710822A4F5A0400BF091F95BF0D0
:10BEA00001FCBDE838402D4A062154F07FBD2C48E6
:10BEB000B4F8BE5505F0CAFC20B1BDE838402848AA
:10BEC00008F004BE162D05D0152D36D1D4F85C35FA
:10BED000072B0AD123480CF089FF22480DF0D2F835
:10BEE000BDE838401F480CF0E3BFA4F5A040F7F7C9
:10BEF0000BFFA4F5A040F7F7E7FDA4F54053D4F8F5
:10BF0000701593F9702264235A4304F6147086F076
:10BF1000F1F8C4F8700504F6147086F02DFA30B10B
:10BF2000BDE838409FED100A46205EF077B9A4F5D1
:10BF3000A040BDE83840F7F7ABBB1E2D18BF4FF04F
:10BF4000FF33084818BFC4F8D034F7F7DDFE0548C2
:10BF5000F7F7BAFD0348ECE7907B0020F09F0D084F
:10BF6000488C0020902B00200000000070B5134882
:10BF700090F984310E46154613B90124204670BD50
:10BF8000D0F87C335B0311D5A0F58053B830B3F8FB
:10BF9000BE1504F0DDFE044640B9094B09480068AF
:10BFA00032462946C06A24F00FFEE7E706482EF025
:10BFB0002FF804460028E0D1044BEFE7908B0020D7
:10BFC0001CA00D088C2B00201081002030A00D0833
:10BFD00010B5144BB3F8BE35532B04461ED10AF0EE
:10BFE000FFF89FED110A46205EF018F99FED0E0A4A
:10BFF00049205EF013F99FED0C0A4A205EF00EF91D
:10C0000046205EF0EBF949205EF0E8F94A205EF048
:10C01000E5F92046BDE81040FFF76ABABDE81040D8
:10C02000FFF7A8B8907B00200000000008207047B0
:10C0300000487047BCA00D0800487047C8A00D0814
:10C040000120704708B50248FDF7B4FE012008BD85
:10C05000902B0020014800F061B900BF94770020C8
:10C0600010B50446FFF786F82046BDE81040FFF7FC
:10C0700073BA0000012070470048704740A10D08C6
:10C080000048704748A10D08012070470120704703
:10C0900010B5054B03F6F47403F6E4730FCB84E894
:10C0A0000F00012010BD00BF907B002008B50B4899
:10C0B00000F5A04200F500530321D3F8403C93FB68
:10C0C000F1F3C2F87035F7F763FD0448F7F7FCFCAD
:10C0D000BDE808400148F7F7DBBA00BF902B00200D
:10C0E0000720704700487047F5820D0800487047E8
:10C0F000C0A10D0801207047012070470120704742
:10C100007047000008B5002303774362034886F0B8
:10C1100037FF0348FBF778FC012008BD7855002065
:10C12000902B002010B5194CD4F8283CB3F90830F6
:10C1300023B9D4F8343CB3F90830F3B100230377C2
:10C140004362D4F8280C5CF049FE04F54463D3ED57
:10C15000007A0F48F8EEE77A27EE800ABDEEC00AB3
:10C1600010EE103AC0F87035A0F5A040F7F710FDBA
:10C17000BDE81040074803F037B8037F002BE0D03C
:10C18000A4F50050F7F7C0FDF2E700BF904B002088
:10C19000907B0020902B002070B54E4DDFED4E7A45
:10C1A00095F8E4339FED4D7A2DED048BB02606FB18
:10C1B000035393ED788A9FED4A9A28EE278A05F576
:10C1C000A653BDEEC88A93ED030AF8EEC87A04467A
:10C1D00067EE897A97EE870A28F070F8237FF0EEF1
:10C1E000408A002B62D105F50053D3F8283CB3F9FF
:10C1F0000830002B5AD1284609F03CF8002855D1C8
:10C2000095F8E43395F8281406FB035393F8C121FD
:10C2100000294BD1012A49D993ED777AF0EE087ABB
:10C22000B4EEE77AF1EE10FA40DBDFED2E7AB0EEF5
:10C23000E80AB4EEE70AF1EE10FA37D5636A93B371
:10C2400089F074FE636AC01AB0F5FA7F32D8237F92
:10C25000002B3CD0244DA5F1200696E80F0085E880
:10C260000F0094ED088AA5F110013046B8EEC88A97
:10C2700017F090FB28EE098ADFED1C0A284670EEC5
:10C28000200AB0EE480A17F02BFC194B9FED190A53
:10C29000D3F80406BDEC048B03682A4631469B6A3A
:10C2A000BDE87040184789F041FE6062636A002B68
:10C2B000CDD0C5E7104D84ED088A012323770023F4
:10C2C000636205F110030FCB85E80F00BFE7BDECFB
:10C2D000048B70BD902B00200000C84235FA8E3CC4
:10C2E0000AD7233CDB0FC93F848B002000007A442F
:10C2F000905B002000000000648B0020036A0B604C
:10C30000007F7047052070470048704738A20D082D
:10C310000048704748A20D080120704738B54B4DC2
:10C320002DED028BD5F8280C9FED498A5CF056FD67
:10C33000D5F8403C07EE903AF8EEE77A05F5405420
:10C3400027EE800AA5F50050BDEEC00A10EE103AA7
:10C35000C4F87035F7F71CFCD5F82C0C5CF03EFDEA
:10C36000B5EEC00AF1EE10FADABF05F64443D3ED9C
:10C37000007AD5ED707A3748CBBF20EE270A20EE41
:10C38000270A20EE080A28EE400ABDEEC00A10EE89
:10C39000103AC4F87435F7F7C7FB95ED707AD4F806
:10C3A000740505F6444327EE087AD3ED007A27EEAC
:10C3B000888AFDEEC77A17EE902AFDEEC87A17EE4E
:10C3C000901A28F02FF8C4F874052248FDF77EFD76
:10C3D00020B1D4F874355B42C4F874351E4B93F821
:10C3E000343F63B195F91432022B08D100230121A7
:10C3F0004620C4F87035C4F874355EF073FA5CF00A
:10C40000FDFB5F215DF0BCFBE8B15DF089FB02281C
:10C4100019D194F81535B3B904F59D6393ED007AFD
:10C42000D5ED987AB4EEE77AF1EE10FA0BD5012348
:10C4300084F81535BDEC028B084A0948BDE8384040
:10C44000042154F0B3BABDEC028B38BD904B0020F0
:10C450000000C842902B0020906B002050A20D08D5
:10C46000785F002010B50446FEF784FE2046BDE844
:10C470001040FFF771B80000062070470048704771
:10C48000D0A20D0800487047E0A20D0801207047B7
:10C49000012070470120704701207047704700005D
:10C4A00008B5044886F06CFD0348FBF7ADFA01209F
:10C4B00008BD00BF78550020902B002038B50F4CE8
:10C4C00004F50055D5F8280C5CF088FC04F53152D1
:10C4D000D2ED007AF8EEE77A04F5A04327EE800A61
:10C4E0002046BDEEC00A10EE102AC3F87025F7F7FB
:10C4F0004FFB2046BDE8384002F076BE902B00206E
:10C500000F2070470048704758A30D080048704737
:10C5100060A30D080120704701207047012070477B
:10C5200001207047012070470120704730B5184B3B
:10C530002DED028B002283F8E22303F53F532433D1
:10C5400005460FCB85B06C4684E80F00114804F017
:10C55000BDFB90B1A86900F57F702AF04BFE0D4835
:10C56000B0EE408A04F01AFCF0EE400A9FED0A0A91
:10C57000204628EE000A17F0B3FA00230748EB61C3
:10C580002146FBF723FE012005B0BDEC028B30BD38
:10C59000905B0020488C0020E02E6542902B00200C
:10C5A00038B5424C94F819354BB104F5805393F8E3
:10C5B000CC3123B1BDE838403D4808F057BAD4F833
:10C5C0003435002B18DC3B48F7F79EFBD4F83835A0
:10C5D000002B29DC3748F7F777FA374890F8E23331
:10C5E000002B46D00121A0F5405009F0F5F9BDE837
:10C5F000384046205DF012BE89F098FCD4F83435FE
:10C60000C01A40F6B7339842DDD82C4DD4F828052F
:10C61000D5F8402C514227F005FFC4F87005A5F568
:10C620000050F7F7B5FAD1E789F080FCD4F8383537
:10C63000C01A40F6B7339842CCD8204BDFED206AC1
:10C6400093ED707AD4F82C0503F64443D3ED007AC9
:10C6500027EE267A67EEA67ABDEEC77AFDEEE77A78
:10C6600017EE102A17EE901A27F0DCFEC4F87405B6
:10C67000B3E7A0F5805090F99F31012B04DCBDE8B1
:10C6800038400C48F7F704B8D4F84435002BF6D0FE
:10C6900089F04CFCD4F84435C01A40F6B7339842C0
:10C6A000EDD804F5A86494ED000AA0E7907B002083
:10C6B000488C0020902B0020905B0020904B0020A5
:10C6C0000000C842D0ED077A0348FCEEE77A17EE87
:10C6D000903A99B202F086BF902B002084B010B53A
:10C6E00003AC84E80E000B4821466F22FBF7B4FC34
:10C6F0009DF80C1011F0040102D1204616F0B2FE94
:10C7000004482146FBF762FDBDE81040012004B05B
:10C71000704700BF902B0020B0EEC00AFDEEC07A3B
:10C7200038B54FF6FF7205460C4617EE900A002109
:10C7300027F078FE07EE900A002CF8EEE77A054B1A
:10C74000C5ED077A14BF4FF0FF32012283F8AC2FFA
:10C7500038BD00BF907B0020FEF77CBC0C207047EA
:10C760000048704739A60D080048704702D90E08E6
:10C7700008B50C48FCF776FA0A480B49FBF772F942
:10C780000848F6F7F1FB40B106484FF48051F6F740
:10C7900065F910B10348FBF737F9024802F0FCF9DC
:10C7A000012008BD902B0020848B002008B50D4887
:10C7B000F7F7AAFA0B48F6F7D7FB50B109484FF440
:10C7C0008051F6F74BF920B1BDE80840054802F06A
:10C7D0000BBD0448F7F778F9BDE808400148F6F7C3
:10C7E00057BF00BF902B002008B509484FF4805177
:10C7F000F6F734F928B10748002241680C3816F0E2
:10C800006DFDBDE808400248002102F0EBBE00BF0C
:10C81000902B0020908B0020881A10B527F02AFD5D
:10C82000104BD3F8A82F0028B8BF4042002AB8BF49
:10C83000524248F6A041B2FBF1F24FF47A7102FB8A
:10C84000011188420CDC93F8F42FD20606D503F6CA
:10C85000F47403F6E4730FCB84E80F00012000E0CA
:10C86000002010BD907B002013B504468069019123
:10C8700000F57F702AF0BEFCDFED0A7A20EE270A71
:10C8800027F09AFCDFED087A019920EE270A20466E
:10C89000FDEEC07A17EE902A02B0BDE81040FFF717
:10C8A000BBBF00BFE02E65420000C84284B070B537
:10C8B0002DED048B86B00FAC84E80E004E4BDFEDFF
:10C8C0004F8A0546D3F8040603F5005603F53F5397
:10C8D00093ED000A0368B0EEC00A5B6A9847B4EEB5
:10C8E000E80AF1EE10FAB0EE408A07DA012006B04D
:10C8F000BDEC048BBDE8704004B070474049204651
:10C9000016F054FF02A8CDED030A8DED020A2AF0BD
:10C9100041FD04A88DED040AB0EE480ACDED050AEC
:10C920002AF0F4FB13A920468DED000ACDED010A93
:10C9300016F03CFF02A88DED020ACDED030A2AF0A5
:10C94000A3FCB4EEE80AF1EE10FACFDBB4EEC08A35
:10C95000F1EE10FA9FED2B9ADFED2B8ADFED2B9A8B
:10C960002BD802A869462AF0C1FB04A88DED040A61
:10C97000CDED050A2AF03EFC684620EE098A2AF031
:10C9800039FC96F9AC3F07EE903AF8EEE77A28EEDC
:10C99000288AA7EEA90A27F091FC20EE090ABDEE2D
:10C9A000C88A20EE280A18EE101AFDEEC07A284632
:10C9B00017EE902AFFF730FF99E738EE400A38EE7D
:10C9C000088A80EE080AB0F0F5FC02A8B0EE408AB2
:10C9D0002AF010FC96F9AC3FF0EE007AB0EE697ADE
:10C9E000A8EE677A07EE903AF8EEE77AA7EE270A04
:10C9F00027F064FCC0E700BF905B0020000000341B
:10CA0000748B0020E02E65420000C842DB0FC93F56
:10CA100010B504460848F6F7A7FA20B92046BDE845
:10CA20001040FEF717BB04484FF48051F6F716F894
:10CA30000028F3D010BD00BF902B002000207047CD
:10CA40000048704748A40D080048704750A40D08DE
:10CA500000207047036993F8140118B1D3F8C40299
:10CA6000C0F380107047000038B5154C0546002112
:10CA7000204608F0DDFD04205DF0D0FB00212046BB
:10CA800008F0E0FD13205DF0C9FB0021204608F00E
:10CA9000E3FD2846FEF74EFD2046012108F09CFFED
:10CAA00046205DF0BBFBAB6904F5A044D3F8F83138
:10CAB000C4F87035AB69D3F8FC31C4F8743538BDAF
:10CAC000902B0020FEF714BD1720704700487047D8
:10CAD000C8A40D0800487047D0A40D080120704775
:10CAE000012070470120704710B50369002283F8C8
:10CAF000402103690446D3F83C0103689B689847CA
:10CB0000A36818687FF000FE206904F059FE03490D
:10CB1000A06910F047FD012010BD00BF8077002004
:10CB20001FB50D4C9FED0D0A04F5C04304F5A0445C
:10CB3000D3F8EC006C302AF0D9FCFDEEE00ABDEE33
:10CB4000C00A10EE903AC4F8743510EE103AC4F8EA
:10CB5000703504B010BD00BF902B00209F0CB34572
:10CB600030B52DED028B83B0044689F0DFF9014624
:10CB7000206900F50E700BF063F938B1204603B060
:10CB8000BDEC028BBDE83040FEF7F4BA206990F8A6
:10CB90004031BBB1012104F099FDA368DFED400AEB
:10CBA0001868036801215B6EB0EE600A984720693F
:10CBB00003F0ECF93B4803B0BDEC028BBDE830401C
:10CBC000FFF78AB8384DDFED398A022104F07EFD87
:10CBD000D5F82C0C5CF002F92369D3ED390A93F9EE
:10CBE0003C2220EE200A002A60EE280A3FDD93F85E
:10CBF000A032002B3BD0D5F8340CCDED000A5CF010
:10CC0000EDF82369D5F8280C93ED3A8A20EE080A4E
:10CC100020EE288A5CF0E2F8236993ED381A20EEC2
:10CC2000410A20EE281ADDED000A2069CDED010A47
:10CC30008DED001A03F0E6F9A36895F93222186821
:10CC40009DED001ADDED010A0368F0EE408A2AB37B
:10CC50001B6CB0EE480A9847A36818680368F2EEA8
:10CC6000040A5B6E0021B0EE680A9847A2E7D5F887
:10CC7000280CCDED000A5CF0B1F82369D5F8340C2E
:10CC800093ED388A20EE080A20EE288A5CF0A6F898
:10CC9000236993ED3A1A20EE010AC2E7DB6BD8E76D
:10CCA0000000000058770020904B00200000C84290
:10CCB000122070470048704748A50D08004870478B
:10CCC00050A50D08012070470120704701207047D2
:10CCD00038B52DED028B43689FED1C8A1D68044614
:10CCE000006904F091F9236993ED131AD3ED110A49
:10CCF000434200EE103A21EE081A60EE880AB8EEC0
:10CD0000C00A284680F0BAFE636820691D6804F0F6
:10CD10007BF9236993ED131AD3ED110A434200EE18
:10CD2000103A21EE081A60EE880AB8EEC00A2846CA
:10CD300080F01EFF9FED060A206903F053F9206979
:10CD400005F000FFBDEC028B012038BD0000C84299
:10CD500000000000014800F079BE00BFCC78002040
:10CD600013B5044600698830FAF7FAF889F0DEF85E
:10CD70000146206900F50E700BF062F828B12046DC
:10CD800002B0BDE81040FEF7F5B9206990F84031D7
:10CD90003BB3012104F09AFCA368DFED170A186881
:10CDA0000368B0EE600A5B6E01219847206903F0CA
:10CDB000EDF863689FED100A186882F089F80F4853
:10CDC000F6F7B2F90D48F6F7A9FA20469FED0A0AE0
:10CDD000FEF7B0FB2069883002B0BDE81040FAF7DA
:10CDE0007DB9074804F0D6FD2069019004F072F97E
:10CDF000019806F0B3FAE2E700000000902B002053
:10CE0000488C00201420704700487047CE9E0D08C3
:10CE10000048704715D90E08012070470020704760
:10CE200070B504460E4800F03BF82369002583F8EE
:10CE30004051206904F08CFF6069052103F048FD32
:10CE4000084826690221FAF78BFC86EDB70A2369A8
:10CE5000C3F848512369C3F84C51012070BD00BF8D
:10CE600004790020902B0020014800F0EFBD00BFA6
:10CE7000CC780020014800F069B800BF0479002098
:10CE8000132070470048704738A60D0800487047C7
:10CE900040A60D080120704701207047012070470F
:10CEA00038B52DED028BDFED240AC3689FED238A90
:10CEB0000446B0EE600A18687CF0A8FFE3681868C2
:10CEC0007DF082F8636820691D6804F09DF823698D
:10CED00093ED131AD3ED110A434200EE103A21EEFE
:10CEE000081A60EE880AB8EEC00A284680F0C6FD2F
:10CEF000636820691D6804F087F8236993ED131AAD
:10CF0000D3ED110A434200EE103A21EE081A60EE0A
:10CF1000880AB8EEC00A284680F02AFE206905F08B
:10CF200011FE256989F002F8C5F86C01BDEC028B91
:10CF300000230120E36138BD000000000000C8426A
:10CF4000014800F083BD00BFCC78002030B52DED46
:10CF5000048B0446006985B08830FAF701F838B1CF
:10CF6000B64805B0BDEC048BBDE83040FFF7F8BE15
:10CF700088F0DCFF05462069294600F50E700AF0AE
:10CF80005FFF38B1204605B0BDEC048BBDE83040F2
:10CF9000FEF7F0B8206990F8403163B3012104F046
:10CFA00095FBA368DFEDA60A186803680121B0EEBF
:10CFB000600A5B6E9847206902F0E8FF63689FEDA6
:10CFC000A00A186881F084FFDFED9D0AE368B0EEE7
:10CFD000600A18687CF01AFFE36818687CF0F4FFB8
:10CFE0009848F6F7A1F8974805B0BDEC048BBDE86A
:10CFF0003040F6F793B9C36A93F8CB3013B992482F
:10D00000FFF74EFF206903F027F918B1E3681868AD
:10D010007CF0F8FE2369D3F86C31EB1AB3F5FA7F94
:10D020000BD9E368DFED860A1868B0EE600A7CF081
:10D03000EDFEE36818687CF0C7FF23699FED838AE3
:10D04000C3F86C510221206904F040FB6368206939
:10D050001D6803F0D9FF236993ED131AD3ED110A6C
:10D06000434200EE103A21EE081A60EE880A284684
:10D07000B8EEC00A80F002FDD4E9033518687CF0F0
:10D080002FFFA368186803689B6EF0EE408A9847EC
:10D0900003AAF0EE400A02A9B0EE680A284602F0A0
:10D0A000F5FFE368DDED030A18689DED020A7CF0E8
:10D0B000ADFE6368186880F0D3FC18B9636818681F
:10D0C00081F0C4FBE368624D186801217DF0E8F847
:10D0D000E36860481B689B68D3EDCF7AFDEEE77A82
:10D0E00017EE903AC5F87035E3681B689B68D3ED7E
:10D0F000D07AFDEEE77A17EE903AC5F8743504F071
:10D1000049FC2369D3F83C01036805F274525B6B58
:10D1100005F5AE61984748B163681B68D3F888236A
:10D12000C3F89423D3F88C23C3F898232069DFED48
:10D130004A9A04F03FFBD5F87035206907EE903A23
:10D14000012105F27453F8EEE78A93ED009A06F098
:10D150009FF8A368B8EEC99A186820EE290A0368F8
:10D1600068EEA98A29EE299ADB6A20EE081A69EE90
:10D17000080A28EE880A9847384BD3F8202F03F680
:10D1800094518A4248D1636993F86430062B0AD8D7
:10D19000206903F0ADFC30B16069072103F098FB12
:10D1A000206904F0D5FD27480221FAF7D9FA206951
:10D1B00003F07EF8636993F86430072BB0EE408A81
:10D1C00008D12369D3F8C4329B0403D4A069012198
:10D1D00010F0AEFE6368B5EEC08AF1EE10FA186882
:10D1E000CCBF01210021B1EE480A80F0CDFC2069BE
:10D1F00007F0CCFD206903F025FF1248F5F794FFF6
:10D200001048F6F78BF89FED0E0A2046FEF792F9CC
:10D2100005B0BDEC048B30BD03F6E4439A422069AF
:10D2200007D190F8423123B19FED050A02F0DAFEF2
:10D23000E0E7019003F04EFF0198F7E7E87800205F
:10D2400000000000902B0020047900200000C8425C
:10D25000907B0020488C00200AD7233C906B002054
:10D260001520704700487047B8A60D080048704761
:10D27000B8A60D08012070470120704700207047B4
:10D28000C369012B06D1044B93F88C02431E58420C
:10D290005841704700207047908B00200E4BB3F927
:10D2A000D221B3F9043207EE102A07EE903AB8EE15
:10D2B000C77AF8EEE77AB0EEC77AF0EEE77AB4EE26
:10D2C000677AF1EE10FAC8BFF0EE477AB7EE080AB7
:10D2D00027EE800A704700BF904B00202DE9F047F1
:10D2E0002DED048B864C94F8FCA18AB00546BAF16A
:10D2F000000F0BD083493122A4F5C04009F060FF34
:10D3000001200AB0BDEC048BBDE8F0870123C361A6
:10D31000A4F11C0696E80F00A4F12C0787E80F0083
:10D320002B6954F8302CB3F8C070DB6A526893F85C
:10D33000A0306421022BA4F5805817FB012740F090
:10D34000B78007EE907A3246B8EEE70AA4F5C041FE
:10D3500006A8FBF755F806A9304616F01BFB284631
:10D36000F0EE408AFFF79AFF2B69B3F9C020D3EDA6
:10D37000310A01EE102AB3F9C220B0EE409A00EE55
:10D38000102AB8EEC11A1A20B8EEC00A26F0AAFF79
:10D390002B69B3F9C030F4EEC98A07EE903AF1EE8A
:10D3A00010FA54BFF0EE686AF0EE496AB8EEE77A18
:10D3B000C8EEA67A2B6828465B68B0EE408A67EE16
:10D3C000877AB4EE670AF1EE10FA48BFB0EE678ACA
:10D3D00098470146A4F5C040FAF7EAFA0821024648
:10D3E0008146A4F5C040FAF76DF9DFED477A38EED3
:10D3F000408AB4EEE78AF1EE10FA32DBC5F81CA0E1
:10D4000096E80F000C3C84E80F009FED409AB9F1BC
:10D41000000F14D005AA0321304615F095FF70B116
:10D42000DDED057AF8EEE77A0322E8EE097A204688
:10D43000FDEEE77A17EE901A15F050FF60E708F658
:10D44000E873D3ED008A3248F8EEE88A15F070FFF1
:10D45000E8EE098A02462F48FDEEE87A17EE901AA8
:10D46000EAE7F4EEC98AF1EE10FA21D505AA514691
:10D47000304615F069FF18B1059B9F42A8BF1F46B3
:10D480005AF010F9044619EE100AF3F73DF8CDE909
:10D49000020118EE900AF3F737F81F4ACDE90001B0
:10D4A0000621204653F082FA6869032103F010FA3E
:10D4B00039461A48FAF75AFF286903F08FFC1448D6
:10D4C00005AA002115F040FF78B96A69D8F8E83F4D
:10D4D000D8F8F81F8B4292F82010D4BF0023012304
:10D4E00063F3000182F820100AE70A4806AA002127
:10D4F00015F02AFF0028E8D0DDE905316A69E9E77F
:10D50000908B002024790020000000340000C842E5
:10D51000748B0020848B0020C0A60D08902B002067
:10D52000014800F093BA00BFCC780020F0B52DED93
:10D53000028B99B0044688F0F9FC0146206900F599
:10D540000E700AF07DFC054638B1204619B0BDECDE
:10D55000028BBDE8F040FDF70DBEE36983B1012BFE
:10D5600000F01D81A048F5F7DFFD9F48F5F7D6FED6
:10D570009D4819B0BDEC028BBDE8F040F6F734BA17
:10D580009FED9A8A60688DED098A8DED0A8A8DED8E
:10D590000B8A8DED0C8A0BAA09A901230068944D12
:10D5A00080F082F92069B0EE480A03F0DBF8636886
:10D5B00090481B68D3EDCF7AFDEEE77A17EE903AEC
:10D5C000C5F8703563681B68D3EDD07AFDEEE77A55
:10D5D00017EE903AC5F8743504F0DCF92369D3F8F6
:10D5E0003C01036805F274525B6B05F5AE61984728
:10D5F00048B163681B68D3F88823C3F89423D3F831
:10D600008C23C3F89823206904F0DAF8A368206912
:10D610001E683368DF6AD5F8703507EE903AD5F8A2
:10D620007435F8EEE78A07EE903AF8EEE70ACDEDAA
:10D63000050A05F0A1F8DDED050AB0EE401A304606
:10D64000B0EE680AB8472069C36B93ED070A02F091
:10D65000C9FC206903F0F6FC63688DED0D8A8DED41
:10D660000E8A8DED0F8A18680FA980F06FFC0D9B54
:10D6700014930E9B159302220F9B169314A910A8C6
:10D6800016F0FEF95C4907AA10A815F00FFF48B183
:10D69000DFED5A7A9DED077AB4EEE77AF1EE10FAF3
:10D6A000FFF660AF0123E36105F6E4730FCB05F6E7
:10D6B000D47686E80F00D5F8D03F22695B68B2F8CF
:10D6C000C0604949642216FB023607EE906A4C4A54
:10D6D000B8EEE70A14A8FAF793FE494814A916F021
:10D6E00059F92046B0EE408AFFF7D8FDB4EEC08A63
:10D6F000F1EE10FAF0EE408A21D53F4808AA002149
:10D7000015F022FE18B1089B9E42A8BF1E4659F094
:10D71000C9FF074618EE900AF2F7F6FECDE90201BE
:10D7200018EE100AF2F7F0FE364ACDE900010621A4
:10D73000384653F03BF96069032103F0C9F83146DC
:10D740002948FAF713FE206903F048FB2A4907AA83
:10D75000A1F1100015F0AAFE636988B19DED077A6A
:10D76000DFED267A93F82020B4EEE77AF1EE10FA96
:10D77000ACBF0121002161F3000283F82020F1E613
:10D78000D5F8E82FD5F8F81F8A4293F82010D4BFB7
:10D790000022012262F3000183F82010E2E62069F2
:10D7A00006F046F8636993F86430042B08D91048F2
:10D7B000D0F8D03F2A46596800F6F47015F08EFD77
:10D7C000636993F86430032B02D9206907F01EFBCC
:10D7D000236993F8D431013B012B3FF6C3AE0248D5
:10D7E000F5F7DCFDBEE600BF902B00200000000036
:10D7F000907B0020488C0020848B002000000034A7
:10D80000748B0020C0A60D0830B5C369012B85B00C
:10D8100004D1414A92F88C32012B04D005B0BDE806
:10D820003040FDF717BCA2F58043B2F97821B3F977
:10D83000D211DFED3A6A3A4D9FED3A0A07EE101A1F
:10D84000B3F9041207EE901AB8EEC77AF8EEE77A49
:10D85000B0EEC77AF0EEE77AB4EE677A00EE902A7F
:10D86000F1EE10FAC8BFF0EE477AB8EEE07AD3EDE9
:10D87000900A03F6085270EEC70A92ED007A27EE7E
:10D88000267AF5EEC00AF7EE006AF1EE10FAB4EE71
:10D89000E67A48BFDFED230AF1EE10FAD8BFB0EE0A
:10D8A000667AF3EE046A77EEA71A67EEA67AC0EE00
:10D8B000876A05F59F626C4693ED6B7A92ED001ACC
:10D8C000B0EE612AA6EE872AF4EE427AF1EE10FA63
:10D8D00048BFB0EE672AF4EE421AF1EE10FAC8BF64
:10D8E000B0EE612A26F030FC05F6F4730FCB07EE9C
:10D8F000901A9FED0D7AF8EEE77A84E80F00E0EEDB
:10D90000077A2146A5F5A040FDEEE77ACDED017A34
:10D91000FAF7BAF805B030BD908B00209A99193FFC
:10D92000907B0020000000000000C84211207047DA
:10D930000048704750A70D08004870475CA70D08C5
:10D940000120704701207047012070470120704777
:10D950000369002283F8402101207047174B1849C2
:10D9600093EDC87AB3F9C020D3F8F401B5EEC07ACC
:10D97000F1EE10FA07EE902AC8BFDFED126AF8EE5A
:10D98000E77ACABF27EE267A20EE270A27EE000A9A
:10D9900067EEA07ABDEEC00AFDEEE77A10EE102A1F
:10D9A000C1F8702517EE902AC1F87425036801F2BA
:10D9B00074525B6B01F5AE61184700BF908B00207D
:10D9C000907B00200000C8421E4BDFED1F6AB3F9B8
:10D9D000C010A3F58050A3F58043F5EEC00AD3F83C
:10D9E000402C8A42A8BF0A4607EE902AF1EE10FAB0
:10D9F000F8EEE77AD6BF03F6444393ED707A93EDE1
:10DA0000007A27EE800A07EE901ACCBF27EE267A1E
:10DA100027EE667AF8EEE77ABDEEC00AB4EEE77A52
:10DA2000F1EE10FA58BFB0EE677A60EE870A10EE9A
:10DA3000102AFDEEE00AC0F8702510EE903AC0F80A
:10DA400074357047908B00200000C84237B52C4CCD
:10DA5000D4F8283CB3F908201B8B07EE102A07EEF8
:10DA6000903AD4F82C3CB8EEC77AB3F908201B8B57
:10DA7000F8EEE77A054687EE270A224807EE102AD5
:10DA800007EE903AB8EEC77AF8EEE77A8DED010A24
:10DA9000C7EE270ACDED000A09F082FFDDED000A8E
:10DAA0009DED010A28B1284603B0BDE83040FFF7DC
:10DAB00055BF04F58043D3F87C23520405D428468F
:10DAC00003B0BDE83040FFF77FBFB3F9C03007EEC9
:10DAD000903AF8EEE77A04F5405427EE800A67EEB4
:10DAE000A00ABDEEC00AFDEEE00A10EE103AC4F83E
:10DAF000703510EE903AC4F8743503B030BD00BFF5
:10DB0000904B0020808E002010B5044688F00EFA5D
:10DB10000146206900F50E700AF092F920B1204606
:10DB2000BDE81040FDF726BB114803F033FF206924
:10DB300090F9D0304BB102F0EFF90E48F5F7F4FA56
:10DB4000BDE810400B48F5F7E9BB02F05BFA20692D
:10DB500005F0BEFB0748F5F7E7FA0648F5F7DEFBE8
:10DB600020469FED050ABDE81040FDF7E3BC00BF6D
:10DB7000488C0020902B0020000000000B207047F4
:10DB80000048704776AA0D0800487047D4A70D08D2
:10DB90000120704701207047012070470020704726
:10DBA00038B53148F6F7B0F82F48F5F78DFF2E4815
:10DBB000F5F76EFD2C481021F4F750FFF0B12B4A19
:10DBC000D2F8E83FD2F8F82F9342D4BF00230123C4
:10DBD000274C94F8682082B9A4F5805573B3A4F15A
:10DBE0001C030FCBA4F12C0585E80F00A4F5C04061
:10DBF000F9F7B8FC012384F8683038BD1D4AB2F942
:10DC00000C1C0029F9DD02F540529FED1B7AD2F879
:10DC1000E83FD2F8D82F9B1A07EE903AF8EEE77A51
:10DC200067EE877A07EE101AB8EEC77AF4EEC77A75
:10DC3000F1EE10FACCBF01230023C9E7A4F580441C
:10DC4000642394F97022D5F8700512FB03F2D4F81E
:10DC5000403C9A42A8BF1A465142C4F8402C26F0D4
:10DC6000E1FBC5F87005C8E7902B0020907B0020F1
:10DC7000908B0020904B00200AD7233CF0B52F4C0E
:10DC80002DED028B04F11005074695E80F0083B0D7
:10DC900084E80F002A48F9F757FA04F12C060146E8
:10DCA0002748FAF763FBA6F50052002386F8683090
:10DCB000C2F8483F96F8CC31002B39D096F8FC31A9
:10DCC0003BB13122A4F59251A6F5C04009F078FA93
:10DCD0002EE096F98631032B03D11A4918482C22DD
:10DCE000F4E7013BDBB2012B22D83B69DB6A93F8F6
:10DCF000A030022B1CD104F12001284615F04AFE69
:10DD00001048B0EE408AFFF7C9FAB4EEC08AF1EECF
:10DD100010FA0DD501AA0121284615F015FB38B1DE
:10DD2000B6F87831642213FB02F3019A9342D4DCF3
:10DD3000012003B0BDEC028BF0BD00BF648B00205E
:10DD4000902B00204079002010B52DED028B244B44
:10DD500093F98621012A03D00020BDEC028B10BD6F
:10DD6000A3F58043B3F90442002CB8BF6442A4B2C7
:10DD70002CB9B3F9D241002CB8BF6442A4B2194BFC
:10DD8000D3F8040603689B6B984730B116491748CF
:10DD9000272209F015FA0120DFE7154AA2F1200138
:10DDA00001F1100015F062FD0028EFD1114B03F5D1
:10DDB0003C6093ED008A02F0F1FF07EE904AF8EE26
:10DDC000E77AB4EEE70AF1EE10FA44BF07EE904AA4
:10DDD000B8EE670AB4EEC08AF1EE10FABCD5D5E70A
:10DDE000908B0020905B002040790020902B002039
:10DDF000848B00208880002070B5474C94F8CC318B
:10DE000088B0054693BB454DB5F9043283EAE3710A
:10DE1000A1EBE37189B205F54054002955D1404882
:10DE200001F0E0FB94F81635002B3ED195F9DF3177
:10DE3000022B52D13B4D95F8513F9BB13A4905F524
:10DE4000AC502CF06FFF68B1012384F8B93528225B
:10DE500005F54861A5F5804009F0B2F928BB00231B
:10DE600084F8B935012384F816351EE094F986311B
:10DE7000022BA4F500561AD103AD284615F028FA56
:10DE8000A4F10C030FCB85E80F0001A9A4F5C04055
:10DE9000FBF736F9D6F8483F052B06D1272206F5C1
:10DEA0005B61A4F5C04009F08BF908B070BD88F043
:10DEB0003DF8D6F8283FC01AB0F57A7FA3D9284696
:10DEC000FFF742FF00289ED0EFE7002BB4BF4FF0D2
:10DED000FF33012384F8AC3FA1E7012B0CD110489C
:10DEE00001F082FA40B10E48F9F7FCFA0028B8BFF9
:10DEF0004042B0F57A7F9DDB95F9DF31042BD4D118
:10DF0000084D95F8513F002BACD0074905F5AC50B2
:10DF10002CF084FF97E700BF908B0020904B0020EF
:10DF2000902B0020906B0020748B00200220704703
:10DF30000048704751A70D0800487047FCD80E08EC
:10DF4000034B0022C3F87025C3F87425704700BF47
:10DF5000907B002038B5094D04462846F5F7E4F8D3
:10DF60002846F5F7DBF92046F5F7F0F92846F5F7EE
:10DF70003BFD2046BDE83840FDF7EEBA902B00206F
:10DF80000D20704700487047BCA80D080048704736
:10DF9000C4A80D0801207047012070470120704778
:10DFA000002380F8273080F83830012070470000C7
:10DFB0000148002101F016BB902B0020F0B5BA4CAF
:10DFC000D4F8F02FD4F8EC3F2DED088B1343D4F8A0
:10DFD000E82F134389B005460FD1B448F5F794FEF6
:10DFE000B248F5F771FD9FEDB20A462009B0BDECCD
:10DFF000088BBDE8F0405CF011B90FF0EDFC90F833
:10E000007C32DB07E9D5B5F91C3095F8271009EE0D
:10E01000103AB5F9243008EE903AB8EEC99AF8EE05
:10E02000E88A002940F0DD809FEDA2AA29EE0ABA15
:10E030000122FDEECB7AA4F5A04017EE903AC4F889
:10E04000E034F9F73FFBA86900F57F700790B0EE68
:10E05000408A29F0CFF8DFED987A20EE270A26F0E3
:10E06000ABF80798F0EE409A29F00EF9A4F5A0401D
:10E07000F0EE40AAFCF7E4FC00287CD104F6E4763C
:10E0800096E80F0005F1280787E80F0096E80F00D3
:10E0900004F6D47787E80F0004F6F47787E80F00DA
:10E0A000D4F8F83F854807EE903AF8EEE77AF0EEBC
:10E0B000680A77EE8B7AB0EE690AFDEEE77A17EE22
:10E0C000903AC4F8F83F15F00BFD002384F8493569
:10E0D00095F92630754803EB830303EB83039B001C
:10E0E0000121A4F80E35F4F751F994F85875002F72
:10E0F00077D1734B9FED737AB3F9A83107EE903A5D
:10E10000F8EEE77A67EE877AF4EEE7AAF1EE10FA16
:10E1100067DD59F0C7FA064619EE900AF2F7F4F9EE
:10E12000CDE9040118EE900AF2F7EEF9CDE902010B
:10E1300019EE100AF2F7E8F9634ACDE90001062169
:10E14000304652F033FC87F0F1FEC4F8CC74C4F8CA
:10E15000B80487F0EBFE0123C4F8C80429EE8A0A4C
:10E1600085F8273026F052F8BDEEC00A10EE103ABE
:10E17000C4F8D03435E087F0D9FED4F86835C01A39
:10E1800042F2107398427FF679AFF0EE087AF4EE1F
:10E19000E7AAF1EE10FA7FF771AFBCEEC88A04F679
:10E1A000F47718EE103A9BB208EE103AB8EEC88A2F
:10E1B00004F6E476B4EEC89AF1EE10FA48D859F0B5
:10E1C00071FA424A062152F0F1FB96E80F0087E807
:10E1D0000F00012385F827300321A4F5A040F4F7B0
:10E1E000D5F832480BF08EF830B130480321F4F7FF
:10E1F000CDF8002385F82730D4F85C35012B40F0AA
:10E20000B880D4F8E83FEA6A9FED2AAA9B1A07EE85
:10E21000903AD4F8D0340133F8EEE79A5ED0DFEDCF
:10E220002C7AE9EE0A7AF4EEE79AF1EE10FA0ADABD
:10E23000284905F1280015F0ADFBF4EEC08AF1EE97
:10E2400010FA00F2968019480321F4F79FF890E045
:10E2500059F028FA204A062152F0A8FB96E80F0050
:10E2600005F1280C8CE80F0096E80F0087E80F00F6
:10E27000D4F8F83F07EE903A39EE488AF8EEE77A9C
:10E28000F0EE680AE8EE0A7A3846B0EE690AFDEE6A
:10E29000E77A17EE903AC4F8F83F15F021FC012117
:10E2A00085F8271099E700BF907B0020902B002075
:10E2B000000000000000C842E02E6542848B002070
:10E2C000904B00209A99993E0DA90D08CCA80D08F5
:10E2D000000048C3748B0020E8A80D08B5F91E3073
:10E2E00007EE903AF8EEE77A05F1280667EE8A7AAB
:10E2F000F4EEE79AF1EE10FA55DB4449304615F09A
:10E3000019FADFED437AB6EE008AA0EE278A96E886
:10E310000F00BDEEC88A9FED3F0AB8EEC88A04F62A
:10E32000F47728EE008A87E80F00F0EE680A3A4892
:10E33000B0EE480A15F0D4FBD4F8F83F07EE903A57
:10E34000F8EEE77A28EE0A0AE9EE0A7AFDEEE77AB5
:10E3500017EE903AC4F8F83F25F058FFBDEEC00A1A
:10E3600010EE103AC4F8D034D4F85C35012B3FF4E9
:10E3700056AF2A480AF0A6FF18B128480321F4F73F
:10E3800005F8D4F85C35012B17D124480AF02EFD8E
:10E3900022480AF077FE214809B0BDEC088BBDE8A1
:10E3A000F0400AF085BD1949304615F0F3FAF4EE55
:10E3B000C08AF1EE10FAA0D9D6E795F838302BB91B
:10E3C000174864F03FFA012385F838301348F5F711
:10E3D0009BFC1248F5F778FB1048F5F759F91148FE
:10E3E00090F8E4336BB1002380F8E4333322022148
:10E3F000A0F5405009B0BDEC088BBDE8F040FBF73C
:10E4000051BF09B0BDEC088BF0BD00BF748B00207C
:10E41000A00CB3450AD7233C848B0020902B00200E
:10E42000304C0020905B002010B50446FCF758FFEC
:10E430002046054B40F8283B14F04AFF204603498C
:10E4400044F04CF9204610BDC0A90D0858A90D088C
:10E45000182070470048704728AA0D0800487047E8
:10E4600030AA0D0801207047012070470120704735
